:020000040800F2
:1080000000800120195A0108110201081302010819
:1080100015020108170201081902010800000000FA
:108020000000000000000000000000001B0201082A
:108030001D020108000000001F020108DD81000888
:10804000655A0108655A0108655A0108655A010810
:10805000655A0108655A0108655A0108655A010800
:10806000FF8D0008655A0108655A0108655A010824
:10807000655A0108655A0108655A0108655A0108E0
:10808000655A0108655A0108655A0108F593000808
:108090008D92000841930008655A0108D98E0008A6
:1080A000655A0108655A0108655A0108655A0108B0
:1080B000655A0108655A0108655A0108655A0108A0
:1080C000655A0108655A0108655A0108655A010890
:1080D000655A0108655A010819910008655A010896
:1080E000655A0108655A0108655A0108655A010870
:1080F000655A0108655A0108655A0108655A010860
:10810000655A0108655A0108655A0108655A01084F
:10811000655A0108655A0108655A0108A98E0008C8
:10812000655A0108655A0108655A0108655A01082F
:10813000655A0108655A0108655A0108655A01081F
:10814000655A0108655A0108655A01080BB700080D
:10815000655A0108655A0108655A0108655A0108FF
:10816000655A0108655A0108655A0108655A0108EF
:10817000655A0108655A0108655A0108655A0108DF
:04818000655A010833
:1081880010B5054C237833B9044B13B10448AFF349
:1081980000800123237010BDC005002000000000EE
:1081A8006865010808B5064B1BB106480649AFF3D8
:1081B80000800648036813B1054B03B1984708BD12
:1081C8000000000068650108C4050020BC05002007
:1081D80000000000684620F007018D4601B5124BEB
:1081E80019781A4679B15B68013353600F4B1968E7
:1081F800013119600E4B196811B1196801391960FC
:108208000023137001E001221A700A4B1A683AB170
:108218001A68013A1A601B6813B9074B01221A70D1
:10822800BDE8014085467047DC050020E054002089
:10823800C44A0020C84A0020CC4A0020074B41F617
:108248004B525A60064AF02182F8231000229A60A5
:1082580007221A606FF004000AF070BC10E000E01A
:1082680000ED00E0014B5868704700BFDC050020B6
:108278002DE9F341684F012001460024022509F049
:10828800E5F90F2338466946012600938DF8044026
:108298008DF806408DF8074048F210088DF8055013
:1082A80009F02AF838466946CDF800808DF806406E
:1082B8008DF807408DF804608DF8055009F01CF81A
:1082C800A7F818804FF480733846694600938DF8F4
:1082D80006408DF807408DF804508DF8055009F0D8
:1082E8000BF821464FF4800007F5806709F006F97E
:1082F8002846314609F0AAF940F6FC733846694623
:1083080000938DF804408DF806408DF807404FF42F
:1083180080588DF8055008F0EFFF38466946CDF8CB
:1083280000808DF806408DF807408DF804608DF8C0
:10833800055008F0E1FFA7F81880314607F5806777
:10834800042009F083F938464AF2C233694600939B
:108358008DF804408DF806408DF807408DF80550DB
:1083680008F0CAFF384644F20803694600938DF8BE
:1083780006408DF807408DF804608DF8055008F028
:10838800BBFF4FF4804308203B833146788307F5D1
:10839800806709F05BF94FF68C733846694600939D
:1083A8004FF010088DF804408DF806408DF807400E
:1083B8008DF8055008F0A0FF384669468DF806404C
:1083C8008DF80740CDF800808DF804608DF80550D1
:1083D80008F092FF40463146A7F81A8009F036F9AE
:1083E8008DF806408DF8074004F1804404F5043404
:1083F8004FF6FF732046694600938DF804608DF8A8
:10840800055008F079FF4FF47F436383FF232383EC
:1084180002B0BDE8F08100BF00000240C90802F0C8
:10842800FFBE07281ED8DFE800F004070A0D101366
:1084380016194FF4807213E04FF4007210E04FF4F5
:1084480080620DE04FF400620AE04FF4805207E0CA
:108458004FF4005204E04FF4804201E04FF4004230
:10846800014B5A83704700BF0010024007281ED8EE
:10847800DFE800F004070A0D101316194FF4807294
:1084880013E04FF4007210E04FF480620DE04FF4F7
:1084980000620AE04FF4805207E04FF4005204E013
:1084A8004FF4804201E04FF40042014B1A837047B9
:1084B8000010024038B50546002445FA04F3DB07EE
:1084C800E0B202D5FFF7D2FF01E0FFF7AAFF0134BF
:1084D800082CF2D138BD08B507282ED8DFE800F0FF
:1084E80004060B10151E232800200FE0144B1869F2
:1084F800C0F3802008BD124B1869C0F3C02008BD26
:108508000F4B1869C0F3003008BD042001F01CFCB3
:10851800B0F5006F34BF0020012008BD084B186972
:10852800C0F3403008BD064B1869C0F3803008BD61
:10853800034B1869C0F3C03008BD002008BD00BF58
:10854800000C024007282DD8DFE800F004090E13BC
:10855800181D2227144B5869C0F300207047124B8E
:108568005869C0F3402070470F4B5869C0F380200A
:1085780070470D4B5869C0F3C02070470A4B5869C3
:10858800C0F300307047084B5869C0F3403070475B
:10859800054B5869C0F380307047034B5869C0F3E6
:1085A800C03070470020704700100240144B5869D3
:1085B8005A69C0F3002091055A6944BF40F002008F
:1085C800C0B252055A6948BF40F0040011055A6903
:1085D80048BF40F00800D2045A6948BF40F0100074
:1085E80091045A695B6948BF40F02000520448BFB3
:1085F80040F040001B0448BF40F08000704700BFB7
:1086080000100240034B202208B15A8370471A8396
:10861800704700BF0010024008B5082001F094FB25
:10862800592804D9064B1A784AB9012206E00820CD
:1086380001F08AFB542802D8014B00221A7008BDA9
:10864800E4050020034B1878013801288CBF00206E
:1086580001207047E4050020034B1878012806BF65
:1086680002221A7000207047E405002001280CD06F
:1086780006D302280ED1084B1869C0F3C0207047F2
:10868800054B1869C0F340207047034B1869C0F3C5
:10869800802070470020704700040240022808B577
:1086A80012D80A4B1A5C0A4BC00018442AB9D0E900
:1086B8000023100C40EA034008BD03C842F21072C0
:1086C80000230CF0BFFE08BD002008BDBE4A0020F4
:1086D800404C0020022830B524D872B60A46CB1781
:1086E8001149012801EBC001C1E90023D1E9004586
:1086F8004FEA054343EA14434FEA0442C1E9002321
:108708000A4A4FF0000342F82030094A42F8203064
:1087180003D0022803D0074A02E0074A00E0074ACC
:10872800536262B630BD00BF404C0020F44B0020BD
:10873800084D00200004014000080040000C0040E3
:108748000020704702289CBF014B43F82010704757
:10875800344C0020012837D002D3022868D0704753
:108768004D4B11F0040F9A680BD0C80602D542F0A1
:10877800040208E022F004029A60DA6842F0040277
:1087880005E022F004029A60DA6822F00402DA6056
:1087980001F0080202F0FF00404B12B101221A70EA
:1087A80000E0187001F0200202F0FF003C4B12B10B
:1087B80001221A7000E0187011F00101394B1ABF3C
:1087C80001221A7019707047334B11F0040F9A6820
:1087D8000BD0C80602D542F4807208E022F48072F9
:1087E8009A60DA6842F4807205E022F480729A6036
:1087F800DA6822F48072DA6001F0080202F0FF0001
:10880800264B12B101225A7000E0587001F0200284
:1088180002F0FF00224B12B101225A7000E058709A
:1088280011F001011F4B1ABF01225A70597070478D
:10883800194B11F0040F9A680BD0C80602D542F004
:10884800200208E022F020029A60DA6842F0200252
:1088580005E022F020029A60DA6822F02002DA604D
:1088680001F0080202F0FF000C4B12B101229A70CD
:1088780000E0987001F0200202F0FF00084B12B1EE
:1088880001229A7000E0987011F00101054B1ABF9F
:1088980001229A7099707047003C0140BB4A002041
:1088A800BE4A0020B84A00202DE9F047C94D8CB0D7
:1088B800002402264FF0C00A284602A9CDF808A0D5
:1088C8008DF80C608DF80E408DF80D608DF80F4016
:1088D80008F012FD28460621032208F089FD03222C
:1088E8002846072108F084FDA5F582350121304688
:1088F80008F0DCFE284609F0A1F909A809F086FA73
:108908004FF6FF79284609A9CDF82890ADF82440FC
:10891800ADF82C40ADF8264009F03AFA2346224635
:108928002846032109F0AFFE06A84FF0080809F011
:10893800E2FC284606A90427ADF8208009F052FD7C
:10894800284606A9ADF8187009F04CFD284641F6EE
:108958005F6109F0F4FD6C622846012105F5803558
:1089680009F0ABFA0DEB08012846CDF808A08DF800
:108978000C608DF80E408DF80D608DF80F4008F0F2
:10898800BBFC28463246062108F032FD324628460E
:10899800072108F02DFDA5F5FE350121384608F020
:1089A80079FE284609F04AF909A809F02FFA28465D
:1089B80009A9CDF82890ADF82440ADF82C40ADF8C1
:1089C800264009F0E5F9234622462846032109F006
:1089D8005AFE06A809F08FFC284606A9ADF82080A3
:1089E80009F000FD284606A9ADF8187009F0FAFC50
:1089F800284641F65F6109F0A2FD6C622846012114
:108A080005F5FC3509F059FA4FF0030A0DEB08019A
:108A18002846CDF808A08DF80C608DF80E408DF82A
:108A28000D608DF80F4008F067FC28462146324655
:108A380008F0DEFC32462846012108F0D9FCA5F5ED
:108A4800FA350121404608F025FE284609F0F6F8D7
:108A580009A809F0DBF9284609A9CDF82890ADF84E
:108A68002440ADF82C40ADF8264009F091F9224693
:108A780023465146284609F006FE06A809F03BFCA5
:108A8800284606A9ADF8208009F0ACFC284606A9BE
:108A9800ADF8187009F0A6FC284641F65F6109F0A8
:108AA8004EFD6C622846012109F007FA3146012083
:108AB80009F066F80497484F012504A88DF8158039
:108AC8008DF814408DF8165008F03EFBBB6801A8DD
:108AD80023F00403BB60FB684FF0200923F0040374
:108AE800FB6006238DF805308DF804808DF806406C
:108AF8008DF8075009F0D6FF4146284609F040F89E
:108B08004FF4807304A804938DF815808DF81440F1
:108B18008DF8165008F018FBBB68052123F4807304
:108B2800BB60FB68284623F48073FB6009F028F8D3
:108B380004A88DF81580CDF810908DF814408DF8A4
:108B4800165008F001FBBB68DFF8988023F020037B
:108B5800BB60FB6801A823F02003FB6017238DF896
:108B6800043007238DF805308DF806408DF807503E
:108B780009F098FFD8F81010184F21F07F432046CD
:108B8800090E3B60FFF7E6FDD8F83010284621F0C3
:108B98007F43090E7B60FFF7DDFDD8F850103046A3
:108BA80021F07F43BB60090E0D4FFFF7D3FD294627
:108BB800484608F06FFD384609F040F841F27073F6
:108BC800384609A90A93ADF82440ADF82C40ADF811
:108BD800264009E000080240003C0140344C0020D7
:108BE80000140040A84C002009F0D2F82A46384664
:108BF800294609F093FC3846294609F05EF93723DF
:108C080001A88DF804308DF805608DF806508DF8B0
:108C1800075009F047FF0CB0BDE8F0870128F0B510
:108C28003E4C0CD002D3022812D019E03C4B1A78E3
:108C38003C4B5B6A0AB1C3F58033236010E0384BC4
:108C48005A78394B5B6A0AB1C3F58033636007E031
:108C5800334B9A78354B5B6A0AB1C3F58033A3600E
:108C6800334954F8202051F820302C4D9A4255F8B9
:108C7800202051F820301EDDD31A2E4EB3F5004FB8
:108C88004FEAC0031E442C4FD6E9002308DA55F8F2
:108C980020C051F8205057F82070C5EB0C0532E081
:108CA80051F820C055F8205057F82070C5EB0C0536
:108CB80005F5803518E09A422BDA51F8202055F84E
:108CC80020301C4ED31AB3F5004F4FEAC0031E44A0
:108CD800194FD6E900230CDA51F820C055F8205076
:108CE80057F82070C5EB0C057D43521B63EBE57309
:108CF8000DE055F820C051F8205057F82070C5EB0A
:108D08000C0505F580357D43521943EBE573C6E93B
:108D1800002354F8203041F82030F0BDF44B0020F7
:108D2800B84A00200004014000080040000C004040
:108D3800084D0020404C0020344C0020164B186988
:108D48001B6980F00800DA06144BC0F3C0001B69E9
:108D58005CBF40F00200C0B21B04114B58BF40F08A
:108D680004001A6951071A691B6958BF40F00800C6
:108D7800120758BF40F010001906094B58BF40F0C1
:108D880020001A691B69D20558BF40F040009B05B6
:108D980058BF40F0800070470004024000080240BD
:108DA800000C0240034B08B1034A00E0034ADA60B2
:108DB800704700BF00ED00E00400FA050100FA0565
:108DC80000239A0002F16042013302F561424FF03C
:108DD800FF31082BC2F88010C2F88011F1D10023AE
:108DE80003F16042013302F561420021F02B82F861
:108DF8000013F5D17047684620F007018D4601B58C
:108E0800042008F007FA0E4B002119600D4B0E489C
:108E1800196000220023C0E900230C4B59620C4B57
:108E28001B7843B90B4B9A6822F004029A60DA68FF
:108E380022F00402DA60BDE801408546704700BFB1
:108E4800F44B0020084D0020404C00200004014055
:108E5800BB4A0020003C014001280CD006D3022860
:108E68000ED1084B1869C0F380007047054B18698C
:108E7800C0F3C0007047044B1869C0F30020704766
:108E8800002070470000024000080240034B4FF4E6
:108E9800804208B15A8370471A837047000802401D
:108EA800684620F007018D4601B50121074809F001
:108EB80055FB0020FFF7B2FE0120FFF7AFFE0220AE
:108EC800FFF7ACFEBDE8014085467047001400403E
:108ED800684620F007018D4601B54FF4807008F010
:108EE8008BF9D8B14FF4807008F094F91D4B00212C
:108EF80059601D4B1D48596000220023C0E9022318
:108F08001B4B59621B4B5B7843B91B4B9A6822F485
:108F180080729A60DA6822F48072DA60202008F0A1
:108F28006BF9D0B1202008F075F90E4B002199603B
:108F38000D4B0E48996000220023C0E904230F4B13
:108F480059620C4B9B7843B90B4B9A6822F020026C
:108F58009A60DA6822F02002DA60BDE801408546AE
:108F6800704700BFF44B0020084D0020404C002003
:108F780000080040BB4A0020003C0140000C0040B3
:108F8800C0B202F079BAC0B202F068BA704770474E
:108F9800704700BF70B5064688B0584809F0A0FB76
:108FA8004FF40030012108F075FB0820012108F07A
:108FB8004DFB022500242023514802A902938DF875
:108FC8000C508DF80E408DF80D508DF80F4008F0BC
:108FD80093F940234A4802A902938DF80C508DF862
:108FE8000E408DF80D508DF80F4008F085F9444873
:108FF8000521072208F0FCF941480621072208F05C
:10900800F7F904A809F018FC0B2E25D8DFE806F0BC
:109018002406090C0F1215181B1E20224FF4615349
:109028001CE04FF4964319E04FF4E14316E04FF487
:10903800164313E04FF4614310E04FF496330DE00C
:109048004FF4E1330AE04FF4613307E02D4B05E0BC
:109058002D4B03E02D4B01E04FF4165304A927488C
:10906800049309F091FB2623002401258DF8043090
:1090780001A806238DF805308DF806408DF80750B5
:1090880009F010FD1D4840F2FF3109F0D5FC2246D9
:109098001A48282109F0B2FC2A46184840F22771DC
:1090A80009F0ACFC2A46154840F2266109F0A6FCF6
:1090B8002A46124840F2255109F0A0FC22460F48E2
:1090C80040F2244109F09AFC22460C4840F6460139
:1090D80009F094FC2246094840F66A1109F08EFC12
:1090E80022460648602109F089FC054B10225A8364
:1090F8000248294609F0C1FB08B070BD0044004091
:10910800000C024090D0030020A1070040420F004D
:10911800684620F007018D46294919B50B889C0639
:109128001AD5284B5B69D80601D58B8814E0264BE5
:109138001A6858680132202A08BF0022824205D0E6
:109148001C6888881919C0B208721A601F4A0A2157
:1091580011609A6A1E4B1A60194803881A061BD5B3
:109168001B4B1A68C2B9184BDC6A196B8C420FD0BA
:10917800144910240C83196B4C1C1C63194491F876
:109188003410C9B28180196B202905D11A6303E014
:1091980040F2277109F032FC094803885B060BD5B9
:1091A80040F2266109F06CFC074B1A6BDB6A9A42A5
:1091B80002D1044B10225A83BDE8194085467047F6
:1091C80000440040000C0240E8050020C84A002086
:1091D800C44A00200A4BDA6A196B0132202A08BFF8
:1091E80000228A420AD0D96A194481F83400DA6226
:1091F800044840F22771012209F000BC704700BF03
:10920800E8050020004400400A4B59681A6891425A
:109218000BD05A68511C59601A44127A02705A6865
:10922800202A04D100225A6001E000207047012062
:10923800704700BFE8050020014B9862704700BFE7
:10924800E8050020044B1A7802F0FF0012B1002252
:109258001A700120704700BFCC4A002072B6034B39
:1092680000225A601A6062B6704700BFE805002005
:1092780010B5441E14F8010F10B1FFF7ABFFF9E762
:1092880010BD00BF684620F007018D4631B5264C59
:10929800264B25681B680135082D08BF00259D420F
:1092A80086B023484FF0000137D001AA07F001FC2F
:1092B8009DF80C302268042B1E4B03EB021206D1DA
:1092C800012151702168029A03EB011105E0002188
:1092D80051702168019A03EB01114A609DF80D2035
:1092E800022A226808BF012103EB021218BF0021DD
:1092F800917022689DF80E1012019954002221687D
:1093080001A8104403EB01111144C07A0132082A64
:109318000872F4D1044B1D6001E007F013FC06B09D
:10932800BDE83140854670475C4B0020D04A00209C
:1093380000640040DC4A0020684620F007018D46A2
:1093480031B5264C264B25681B680135082D08BF0A
:1093580000259D4286B023484FF0010137D001AA6D
:1093680007F0A7FB9DF80C302268042B1E4B03EB7B
:10937800021206D1012151702168029A03EB0111F2
:1093880005E0002151702168019A03EB01114A6040
:109398009DF80D20022A226808BF012103EB021262
:1093A80018BF0021917022689DF80E10120199547F
:1093B8000022216801A8104403EB01111144C07A6E
:1093C8000132082A0872F4D1044B1D6001E007F04D
:1093D800B9FB06B0BDE83140854670475C4B0020BC
:1093E800D04A002000640040DC4A0020684620F093
:1093F80007018D4631B52B4B2B4A1968126886B088
:10940800914205D129480121002207F01EFC44E0C1
:109418001A68274901EB0212507800F0FF0248B1A0
:1094280004228DF80C20002201921A6801EB021226
:10943800526806E018688DF80C2001EB00104068AF
:10944800019002921A6801EB0212927802F0FF0072
:109458001AB102228DF80D2001E08DF80D001A686E
:1094680012018A5C8DF80E2000221C680D4801EB61
:1094780004141444257A01AC14440132082AE57214
:10948800F3D1036801A9013303600368082B04BF03
:1094980000230360054807F072FA06B0BDE83140C2
:1094A80085467047D84A0020D44A0020006400400E
:1094B800604B0020F0B501388BB00F4615460223EB
:1094C80007282AD8DFE800F0211917110F0D0B041F
:1094D800ADF80C300B238DF81030012324E0032362
:1094E8001CE006231AE00C2318E00F22ADF80C202C
:1094F8008DF8102018E01E2310E03C23ADF80C3046
:109508000F238DF8103007230EE07823ADF80C30C8
:109518000C238DF81030032306E00823ADF80C3037
:109528000F238DF8103002238DF81130884800235E
:109538008DF80F3007F0CAF84FF00070012108F0DD
:10954800A9F80820012108F081F8032300240193D9
:109558000820022301218DF808308DF809308DF894
:109568000A408DF80B4008F071F87A4801A907F015
:10957800C3FE78482146092207F03AFF75480121C1
:10958800092207F035FF0126714803A98DF80E401E
:109598008DF812408DF813608DF814408DF8154041
:1095A8008DF816608DF8176007F0AAF8B7F5006F08
:1095B8008DF822408DF823408DF824600FDA7B0166
:1095C800ADF818304FF6FF73ADF81A40ADF81C30FF
:1095D800ADF81E30ADF820408DF825600DE04FF64F
:1095E800FF73ADF81840ADF81A40ADF81C30ADF86F
:1095F8001E30ADF820408DF8254006A807F0EBF89E
:10960800012300228DF822308DF823208DF8243094
:1096180095B1B5F5006F0FDA6901ADF81A204FF66C
:10962800FF72ADF81810ADF81C20ADF81E20ADF88B
:1096380020308DF825300DE04FF6FF71ADF8182079
:10964800ADF81A20ADF81C10ADF81E10ADF820309A
:109658008DF8252006A807F0BEF802238DF82230E1
:109668007B13FF0047F0040700260124ADF81A70A9
:1096780006A84FF6FF77ADF818308DF823608DF8FF
:109688002440ADF81C70ADF81E70ADF820608DF860
:10969800254007F0A0F80323B5428DF822308DF855
:1096A80023608DF8244010DD6B13ED0045F00405B0
:1096B800ADF81830ADF81A50ADF81C70ADF81E7042
:1096C800ADF820408DF825400CE00423ADF8186073
:1096D800ADF81A30ADF81C70ADF81E70ADF820402A
:1096E8008DF8256006A807F076F8012407260025DE
:1096F800142368468DF800308DF801608DF802500B
:109708008DF8034009F0CEF9152368468DF800302E
:109718008DF801608DF802508DF8034009F0C2F908
:10972800132368468DF800308DF801608DF80250DB
:109738008DF8034009F0B6F922460548022107F0E2
:1097480084FA03481021224607F07FFA0BB0F0BDD7
:1097580000640040000C0240F0B5437887B004462E
:10976800426833B104238DF80C3000230292019330
:1097780003E08DF80C3001920293A37803B1022321
:109788008DF80D3023788DF80E300023E11801AAEA
:109798001A44097A0133082BD172F7D1114801A96B
:1097A80007F0EDF8042817D10F4F104B3D681B68E0
:1097B8000135082D08BF00259D420FD03E680C4B8F
:1097C80003EB061694E80F0086E80F000121054810
:1097D8000A463D6007F039FA012000E0002007B092
:1097E800F0BD00BF00640040D44A0020D84A0020E1
:1097F800604B002030B50D4B0D4C054622681B68A8
:109808009A420ED023685A1C22600A4A02EB0313BC
:109818000FCB85E80F002368082B04D100232360B1
:1098280001E0002030BD012030BD00BF5C4B0020AE
:10983800D04A0020DC4A00202DE9F0474FF4805040
:1098480088B0012107F032FF694D0120002402266B
:10985800E023014601938DF80A408DF80B408DF8FE
:1098680008608DF8096007F0F1FE284601A907F0A5
:1098780043FD052128460A4607F0BAFD5D4F2846F4
:109888000621052207F0B4FD05222846072107F026
:10989800AFFD012520234FF482794FF40078384634
:1098A80003A9ADF81830ADF80C40ADF81040ADF88C
:1098B8001A40ADF81C40ADF80E90ADF81260ADF846
:1098C8001450ADF8168007F0F7FF3846294608F01F
:1098D80090F829464FF4804007F0DCFE07F554471E
:1098E8004FF460433046294601938DF80A408DF8BD
:1098F8000B408DF808608DF8096007F0A7FE384620
:1099080001A907F0F9FC38460D21052207F070FD82
:1099180038460E21052207F06BFD052238460F2137
:10992800A7F5E63707F064FD4FF0100A384603A99B
:10993800ADF80C40ADF81040ADF81A40ADF81C4039
:10994800ADF80E90ADF81260ADF81450ADF8168071
:10995800ADF818A007F0B0FF3846294608F049F8D6
:1099680029464FF4004007F095FE07F5E8374FF415
:10997800E0532946042001938DF80A408DF80B40E6
:109988008DF808608DF8096007F060FE384601A977
:1099980007F0B2FC38460A21062207F029FD3846AE
:1099A8000B21062207F024FD062238460C2107F079
:1099B8001FFDADF80C40ADF81040ADF81A40ADF8F9
:1099C8001C400D4C03A92046ADF80E90ADF812606E
:1099D800ADF81450ADF81680ADF818A007F06CFF7C
:1099E8002046294608F005F808B0BDE8F08700BF12
:1099F8000000024000300140003C004070B50446C1
:109A08000D461646042878D8DFE800F003090D1241
:109A1800060002223A4B09E00122394B01E0394B9A
:109A280010225A8309E0384B4FF480525A8315E0CC
:109A3800344B4FF400425A8321E03448022108F0A5
:109A480068F80028F9D03148294608F02DF82F4841
:109A5800012108F05EF80028F9D021E02C48022105
:109A680008F057F80028F9D02948294608F01CF8CA
:109A78002748012108F04DF80028F9D010E02548C2
:109A8800022108F046F80028F9D02248294608F0B3
:109A98000BF82048012108F03CF80028F9D016E01E
:109AA800DEB1042C29D8DFE804F003090D13060001
:109AB8000222134B09E00122114B01E0114B102245
:109AC8001A8311E0104B4FF480521A830EE07EB1D6
:109AD8000C4B4FF400421A830AE0042C0DD8DFE83F
:109AE80004F0050305070300084802E0084800E001
:109AF800084807F0D6FFC0B270BD002070BD00BF97
:109B08000010024000000240000402400030014002
:109B180000380040003C0040F8B50BF055FA0AF058
:109B280037FE00222E4B0AF087FE21A3D3E900233B
:109B38000AF082FE04460D4622462B461CA1D1E9B6
:109B480000010AF0C5FC1CA3D3E9002306460F4612
:109B5800204629460AF09AFF02460B463046394607
:109B68000AF094FF0BF02AF90AF012FE00221D4BAE
:109B78000AF08CFF0CF0F2F811A3D3E900230AF0E5
:109B88005BFE11A3D3E900230AF0A4FC02460B46AE
:109B98000FA1D1E900010AF079FF0FA3D3E900234F
:109BA8000AF096FC0BF00AF90BF02CFCF8BD00BF8C
:109BB8006666666666660A409A9999999999014017
:109BC800C3F5285C8FA272400000000000FEAA4086
:109BD8009A999999FD6F2F41C3F5285C8F127140AE
:109BE8000000303F000024402DE9F0414FF4800090
:109BF8009CB0012107F02AFD4FF480700121002458
:109C080007F054FD0326332301A94A4801938DF830
:109C18000B408DF8086007F06FFB01A94648DFF894
:109C280024818DF80B4001968DF8086007F064FBDD
:109C38004FF48000012107F009FD01214FF48070E5
:109C480007F034FD404607F0D9F83C4B01250E9348
:109C58003B4B06270F934FF4806313934FF4006335
:109C680014934FF4005315934FF4807316934046A2
:109C78004FF400330DA917930D941094129418946F
:109C88001A941B941197199507F03EF929464046F6
:109C980007F075F903A8039404940594069406F054
:109CA80093FB079409940A940B9404F1804404F5F7
:109CB8009034204607A98DF820508DF821508DF852
:109CC800307006F052FB2046294606F045FC204637
:109CD8002A462B460A2106F0C3FB20462B460E21B6
:109CE800022206F0BDFB204632462B460F2106F025
:109CF800B7FB20462B460821042206F0B1FB20467C
:109D08002B460921052206F0ABFB3A462B46204696
:109D18000B2106F0A5FB2046294606F026FC204626
:109D2800294606F06BFB204606F0E2FB1CB0BDE8B6
:109D3800F08100BF00080240000402404C200140AE
:109D48003C060020106402400B2821D8DFE800F010
:109D580006202020092020200D15181B0D4B1888DF
:109D680001E00C4B588880B270470A4B588940F282
:109D7800712380B2584300137047064B988804E05B
:109D8800044BD88801E0034B188980B2FFF7C4BEA2
:109D9800002070473C0600200C4BC0EBC000184464
:109DA80090F800380B7090F801384B7090F8023832
:109DB8008B7090F80338CB7090F804380B7190F8DA
:109DC80005384B7190F806388B71704748060020AB
:109DD80038B54FF40063254A002199540133B3F58F
:109DE800804FF8D14FF40064002006210122FFF7CC
:109DF80005FE002005210246FFF700FE002001466F
:109E08000122FFF7FBFD8307F3D50020022102465C
:109E1800FFF7F4FD0020C4F307210246FFF7EEFD2B
:109E28000020E1B20246FFF7E9FD0025B5F13F0E3B
:109E3800DEF100024FF0000052EB0E020146013540
:109E4800FFF7DCFD402DF1D1002005210246FFF788
:109E5800D5FD002001460122FFF7D0FDC307F3D44A
:109E68004034B4F5804FBFD138BD00BF480600204C
:109E7800F7B5C0EBC00000F5006500200C460246AF
:109E88000321FFF7BBFD0020C5F307210246FFF7BA
:109E9800B5FD0020E9B20246FFF7B0FD00200146FB
:109EA8000246FFF7ABFD0746002001460246FFF7D2
:109EB800A5FD0646002001460246FFF79FFD054620
:109EC800002001460246FFF799FD8DF803000020A7
:109ED80001460246FFF792FD8DF804000020014676
:109EE8000246FFF78BFD8DF8050000200146012290
:109EF800FFF784FD23788DF80600BB420DD1637807
:109F0800B3420AD1A378AB4207D1DDF80300D4F8F5
:109F18000330C31A5842584100E0002003B0F0BD96
:109F280038B51B4B04460D46195500200621012261
:109F3800FFF764FD002005210246FFF75FFD0020C2
:109F480001220146FFF75AFD8207F3D500200221BE
:109F58000246FFF753FD0020C4F307210246FFF72E
:109F68004DFD0020E1B20246FFF748FD00202946DA
:109F78000122FFF743FD002005210246FFF73EFDC1
:109F8800002001460122FFF739FDC307F3D438BD8D
:109F98004806002038B5C0EBC0050C4605F5006042
:109FA8000978FFF7BDFF05F601006178FFF7B8FFF4
:109FB80005F60200A178FFF7B3FF05F60300E17884
:109FC800FFF7AEFF05F604002179FFF7A9FF05F6B4
:109FD80005006179FFF7A4FF05F60600A179BDE841
:109FE8003840FFF79DBF2DE9F041002304460F4696
:109FF8001646B34205D03D4AF95C2244D154013398
:10A00800F7E7002006210122FFF7F8FC00200521D0
:10A018000246FFF7F3FC002001460122FFF7EEFCA1
:10A028008507F3D5002002210246FFF7E7FC002050
:10A03800C4F307210246FFF7E1FC0020E1B2024623
:10A04800FFF7DCFC0025B54242D0013414F03F088C
:10A05800795D04D0721EA81A4242424100E00122F2
:10A068000020FFF7CBFCB8F1000F2FD1731E9D42E3
:10A078002CD2002005210246FFF7C0FC0020014633
:10A088000122FFF7BBFC10F00100F2D106210122EA
:10A09800FFF7B4FC002005210246FFF7AFFC0020C3
:10A0A80001220146FFF7AAFC8207F3D5002002210E
:10A0B8000246FFF7A3FC0020C4F307210246FFF77E
:10A0C8009DFC0020E1B20246FFF798FC0135BAE793
:10A0D800002005210246FFF791FC002001460122DD
:10A0E800FFF78CFCC307F3D4BDE8F08148060020D5
:10A0F800014B185C704700BF4806002010B50023CC
:10A10800934205D0034C0444E45CCC540133F7E794
:10A1180010BD00BF4806002073B500200321024689
:10A12800FFF76CFC002001460246FFF767FC0020A1
:10A1380001460246FFF762FC002443F6FF72A51AA7
:10A148006A424FF000006A410146FFF757FC404B56
:10A1580018550134B4F5804F1D46EED10020052175
:10A168000246FFF74BFC002001460122FFF746FCA0
:10A1780010F07104F2D1FEF775F80646FEF772F892
:10A18800801B0028B8BF4042B0F5FA6F07DA3CB927
:10A1980095F8FF47B4F142035C425C41EEE71CB11D
:10A1A8002C4B1B78002B3CD040F2FF700021FFF7AE
:10A1B800B7FEFFF70DFE002027494022FFF713FFE7
:10A1C8000024B42202FB04F0244900F58070FFF754
:10A1D8000AFFA01C4001224920220134FFF703FF97
:10A1E800032CEED1002301934FF4C364204601A948
:10A1F80004220434FFF7F7FEB4F5FF6FF6D100230D
:10A2080001934FF4A764204601A904220434FFF700
:10A21800EAFEB4F5C36FF6D140F2FF704221FFF7B2
:10A228007FFE00200C494022FFF768FF40200D49BF
:10A238002022FFF763FF60200B492022FFF75EFF13
:10A2480080200A492022FFF759FF02B070BD00BFE5
:10A2580048060020304C002004000020C462010899
:10A26800A4620108A84C0020C84C0020E84C00203B
:10A278002DE9F843144612788046C2F34115EFB22F
:10A28800032F0E462DD0484901EB451101F1080373
:10A29800187930BBD00724D45F2A22D84348405DC0
:10A2A800F8B912F0970F1CD1DFF8089119F80520BA
:10A2B80062B9C97F384619B1FEF7B0F8032303E045
:10A2C8005978FEF7ABF8022309F80530DFF8E89073
:10A2D80019F805302BB1384601F0CEF8002309F8FB
:10A2E8000530217800220420FFF788FB3070617860
:10A2F80000220420FFF782FB7070A178002204205E
:10A30800FFF77CFBB07001220420E178FFF776FBB1
:10A31800F0702378DA0744D45F2B42D803F01E028A
:10A32800082A13D0142A31D0062A3AD1242202FB53
:10A3380008F85B090C2202FB03831D4AA178134429
:10A34800E27842EA01225A60BDE8F883242101FB41
:10A3580008F15B090C2000FB0313A678E578144A82
:10A3680045EA0625D550A3781B071AD594F800802E
:10A378004FEA581800FB081852F808306FEA0353E0
:10A388006FEA135342F80830BDE8F883242101FB33
:10A3980008F85B090C2101FB03830549E2780B44AB
:10A3A8001A72BDE8F88300BFA84C0020604D002059
:10A3B800584C00205D4D0020634D002007B51378F0
:10A3C8008DF800108DF80130537801A98DF802300E
:10A3D80093786A468DF80330FFF74AFF03B05DF8BB
:10A3E80004FB07B58DF802309DF810308DF8001089
:10A3F8008DF8012001A96A468DF80330FFF738FF70
:10A4080003B05DF804FB07B500238DF800108DF844
:10A4180001308DF80320131201A96A468DF8023025
:10A42800FFF726FF03B05DF804FB5F292DE9F34130
:10A4380005460E46144658D811F01E07C1F34112BE
:10A4480002D0022F1DD050E000EB40031A443049DF
:10A458001201881843688C50C3EB040EBEF1000F3C
:10A46800B8BFCEF1000EBEF5000F08DB9C42CCBF92
:10A47800284C294C0A441C440123137335E0077304
:10A4880033E000EB4007224B17443F01D91924F071
:10A498007F4EC1F808E04C6001F10800D959984690
:10A4A800C4EB010EBEF1000FB8BFCEF1000EBEF531
:10A4B800000F18DBA142CCBF164B174B52012344A7
:10A4C8008DF800201A148DF801201A128DF8022038
:10A4D800284601A96A468DF803304744FFF7C8FEAD
:10A4E80001233B7301E00023037123148DF801302D
:10A4F8002846231201A96A468DF800608DF80230BB
:10A508008DF80340FFF7B4FE02B0BDE8F08100BF4C
:10A51800A44D0020FFFF7F00010080FF07B511F068
:10A528001C0202D1FFF781FF0CE000238DF8001018
:10A538006A4601A98DF801308DF802308DF8033094
:10A54800FFF796FE03B05DF804FB012104200A46DC
:10A55800FFF754BA13B541F0010114468DF8041001
:10A5680001AA6946FFF784FE9DF801309DF80000B6
:10A5780023709DF8023063709DF80330A37002B019
:10A5880010BD07B541F001018DF8041001AA694614
:10A59800FFF76EFE9DF803309DF8020043EA0020A5
:10A5A800030544BF6FEA00506FEA105003B05DF82E
:10A5B80004FB73B54901CCB244F01503164601A952
:10A5C8006A4605468DF80030FFF752FE9DF80530C3
:10A5D80044F014048DF801309DF80630284601A98E
:10A5E8006A468DF800408DF802308DF80360FFF759
:10A5F8003FFE02B070BD73B54901CCB244F01503FB
:10A60800164601A96A4605468DF80030FFF730FE68
:10A618009DF8053044F014048DF801309DF807309A
:10A62800284601A96A468DF800408DF802608DF829
:10A638000330FFF71DFE02B070BD2DE9F34740015E
:10A64800C7B2C1F30A06002047F0180101AAFFF7B4
:10A6580081FF9DF8058030464FEA181908F00F0869
:10A66800C8450FDB0AF072F8C9EB08080446012058
:10A6780000FA08F00D460AF079F80022344B0AF087
:10A68800DBF810E00AF062F8C8EB0908044601207C
:10A6980000FA08F00D460AF069F802460B46002059
:10A6A8002B490AF0F3F902460B46204629460AF0E0
:10A6B800EDF90AF083FB0AF06BF823A3D3E9002332
:10A6C8000AF0BAF80AF07AFB0AF062F80022214B85
:10A6D8000AF0B2F84FF0FF3904460D46CA464FF06B
:10A6E8000008012000FA08F00AF040F802460B467C
:10A6F800204629460AF0A0F80AF038FBA0F18002AB
:10A70800802A38BFC14608F1010828BF5046B8F171
:10A718000E0F01D08246E4E700248DF8050047F0CB
:10A728001201204601AA8DF804408DF80690FFF723
:10A7380045FE204647F00C013246FFF764FE2046EE
:10A7480002B0BDE8F08700BF04560E2DB29DEF3F62
:10A75800000060400000204073B54C0804EB44043E
:10A76800B42304F5807403FB0044054620460E46D6
:10A77800FFF7BEFC8DF80400601CFFF7B9FC8DF8EC
:10A788000500A01CFFF7B4FC46EA45118DF8060049
:10A79800C9B2002001AAFFF711FE02B070BD37B59B
:10A7A8000C46640841EA401101AA0546C9B20020D6
:10A7B80004EB4404FFF7CEFE04F58074B42303FBD6
:10A7C80005449DF804102046FFF7AAFB601C9DF87D
:10A7D8000510FFF7A5FBA01C9DF80610FFF7A0FBCE
:10A7E80003B030BD10B5C4B221466401E4B2002004
:10A7F8000222FFF7DEFE44F008010020FFF78EFE7C
:10A8080044F00A010020BDE81040FFF787BE37B5C5
:10A81800400140F01604E4B20D4601AA214600208A
:10A82800FFF798FE9DF8053015F0010F14BF43F0AF
:10A83800400323F040038DF805309DF8053015F0EE
:10A84800020F14BF43F0100323F010030020214629
:10A8580001AA8DF805308DF80600FFF7AFFD03B0AB
:10A8680030BD37B5400140F01604E4B20D4601AAE8
:10A8780021460020FFF76EFE9DF8053015F0010F08
:10A8880014BF63F07F0303F07F038DF805309DF854
:10A89800053015F0020F14BF43F0200323F0200306
:10A8A8000020214601AA8DF805308DF80600FFF733
:10A8B80085FD03B030BD07B5400140F0160101F039
:10A8C800F60101AA0020FFF745FE9DF80530C3F305
:10A8D8008010DB0648BF40F0020003B05DF804FBBF
:10A8E80007B5400140F0160101F0F60101AA002069
:10A8F800FFF730FE9DF80530D8099B0648BF40F0A9
:10A90800020003B05DF804FB70B50F4C000123187A
:10A918009A68914209DD8A1AC2F18075AA425E6876
:10A9280001DC324409E0751B0AE00ADA521AC2F166
:10A938008075AA425E6802DCB21A5A6001E03544AA
:10A948005D602044816070BDA44D002037B541F0A2
:10A9580001030C4601AA69468DF804300546FFF745
:10A9680087FC9DF802309DF801201B0243EA024350
:10A978009DF8032043EA02010B0248BF41F07F41E2
:10A988005F2C19D8C4F3411214F01E040ED0022C07
:10A9980012D105EB45051544E8B221F07F41FFF7D8
:10A9A800B3FF074B03EB0515696805E005EB4505A3
:10A9B8002A44034B12019958084603B030BD00BF22
:10A9C800A44D002038B50C4668210546FFF7BEFFA8
:10A9D80014B140F0010201E020F00102284668218C
:10A9E800BDE83840FFF721BD73B51C4B587E10F009
:10A9F800010004D00020682140F2211202E0682101
:10AA08004FF49072FFF711FD0020022300937E217E
:10AA180002460346FFF7E5FC00240025E6B2E9B24A
:10AA280030460135FFF798FE1D2DF7D17501EDB2BF
:10AA380045F00C010020FFF789FF01463046FFF77B
:10AA4800FCFD0134002045F0160143F2FF12FFF728
:10AA5800DAFC032CE1D102B070BD00BF0400002075
:10AA6800F0B5450185B0044645F0030303AA00206C
:10AA780002A98DF80C30FFF7FBFB9DF80A109DF832
:10AA88000930090241EA03419DF80B302046194379
:10AA9800154EFFF739FF2301F21802F10801087972
:10AAA80000B312480C2707FB0404207AD0B9F358E6
:10AAB80052689C1A002CB8BF6442B4F5000F05DB3D
:10AAC8009342CCBF0A4B0B4B134400E00871DAB237
:10AAD80000920020C3F3074205F0E001C3F3072307
:10AAE800FFF77FFC05B0F0BDA44D0020584C0020B6
:10AAF800FFFF7F00010080FFF8B50F4B0D461E5C7D
:10AB0800C1F3074100223046FEF778FF0B4C0702DD
:10AB1800C5F30721002230462760FEF76FFF384350
:10AB28000702E9B2304601222760FEF767FF384383
:10AB380007092760F8BD00BFF462010848460020F5
:10AB480038B5484C0B2303FB004203FB0043117943
:10AB58000433032984BF032111719A78032A84BF1F
:10AB680003229A700B2303FB004203FB0043117A74
:10AB780004320F2984BF0F2111715A7A0433072A2E
:10AB880084BF07225A710B2303FB004203FB0043D7
:10AB9800917A04320F2984BF0F2191715A7B0C33AB
:10ABA8000F2A84BF0F225A700B2202FB004302FBBC
:10ABB8000042997B0C330F2984BF0F2199701379B8
:10ABC8005279DB0343F40021A1621AB1254943F409
:10ABD80004238B620B2101FB0041C979214B19B178
:10ABE800996A41F4005199620B2372B903FB00433F
:10ABF800197A9A79C90141EAC2210433A26A5B79B8
:10AC08000A4342EA0312A2621AE003FB00431B7BD9
:10AC1800144A1BB1936A43F4805393620B2202FBDC
:10AC28000042917B557BA26A0E4B42EAC51201F0A5
:10AC3800070542EA0512090748BF42F400629A6212
:10AC48000B2202FB0042D17A064B043219B99179E2
:10AC58009A6A0A439A62A16AFFF74EFFA36AE362FF
:10AC680038BD00BF4846002010B5134C0023A3622E
:10AC7800C300E21892F8352012B14FF40072A262B4
:10AC8800E11891F836100C4A19B1916A41F48071B3
:10AC98009162E21892F8371023440F2984BF0F21DC
:10ACA80082F8371093F83710A36A1943A162FFF7A7
:10ACB80023FFA36AA36410BD4846002038B5224C80
:10ACC8004FF46023A362C300E21892F8532012B134
:10ACD8004FF47022A262E21892F84D1092F84C508C
:10ACE800090341EA853192F84E20A56A012A41EA12
:10ACF8000501A16203D1144A41F480619162E1180F
:10AD080091F84F50A26A91F8501042EA05220129A1
:10AD1800A26203D10C4942F080028A62E11891F8DC
:10AD28005110094A012903D1916A41F04001916209
:10AD3800234493F85210A36A43EA0111A162FFF772
:10AD4800DBFEA36A636638BD4846002038B52A4C46
:10AD580043001A18224492F9691068323F29C4BF87
:10AD68003F2151701A18224492F9691068323F3114
:10AD7800BCBFC12151701A18224492F86A10683277
:10AD88001F2984BF1F2191704FF44022A2621A1814
:10AD9800224492F86820012A03D1174A4FF450211F
:10ADA800916204EBC00191F85310134A51B9191874
:10ADB800114491F86950916A05F07F0541EA05212F
:10ADC80091620CE01D18154495F8695001F00301D3
:10ADD80005F07C052943956A45EA012595620344F7
:10ADE800234493F86A10A36A1943A162FFF784FE0B
:10ADF800A36A636738BD00BF4846002010B58300CA
:10AE0800254C1A18224492F87810012984BF012190
:10AE180082F878101A18224492F8791078320329A7
:10AE280084BF032151701A18224492F87A1078329C
:10AE38000F2984BF0F2191701A18224492F87B10B1
:10AE48007832032984BF0321D1701A18224492F85A
:10AE58007C1003440F2988BF0F2102F1780288BFB4
:10AE68001171234493F87C1003F1780293F8783039
:10AE780041F4202141EAC331537841EA43319378C0
:10AE880041EA0321D37841EA4311A162FFF734FE76
:10AE9800A36AC4F8883010BD4846002000202C4A18
:10AEA800F8B5054604462B4E0327A6F11C016F543E
:10AEB800331929444FF0050E4FF0010C04F806C071
:10AEC80081F805C083F801E04FF0020C83F802E036
:10AED80000234F708B70CB700B7181F806C0CB715B
:10AEE8003C4406F11001383E43542E440144092CD9
:10AEF80082F800C05370D370937082F804C0577101
:10AF080082F806E0D3711372977253724B708B708C
:10AF1800CB700B717371B371F37105F1080570444F
:10AF280002F10B02BFD11D46ECB22046FFF766FFC7
:10AF38002046FFF70BFF2046FFF7C0FE2046FFF72D
:10AF480093FE01352046FFF7FBFD032DECD1F8BD3C
:10AF58004C460020B0460020064B042903EBC003F2
:10AF680018BF002283F8371018BF83F83520FFF781
:10AF78007BBE00BF48460020054B03EBC00383F8A7
:10AF8800351011B1042283F83720FFF76DBE00BFDA
:10AF980048460020034B03EBC00383F83610FFF745
:10AFA80063BE00BF48460020024B03EBC00090F888
:10AFB8003700704748460020024B03EBC00090F86A
:10AFC8003500704748460020024B03EBC00090F85C
:10AFD8003600704748460020034B0B2202FB003323
:10AFE8001971FFF7ADBD00BF48460020034B0B2287
:10AFF80002FB00335971FFF7A3BD00BF484600208C
:10B00800034B0B2202FB0033D971FFF799BD00BF38
:10B0180048460020034B0B2202FB00339971FFF7CF
:10B028008FBD00BF48460020034B0B2202FB0033B4
:10B038001972FFF785BD00BF48460020034B0B225D
:10B0480002FB00335972FFF77BBD00BF4846002062
:10B05800034B0B2202FB00339972FFF771BD00BF4F
:10B0680048460020034B0B2202FB00331973FFF7FD
:10B0780067BD00BF48460020034B0B2202FB00338C
:10B088005973FFF75DBD00BF48460020034B0B22F4
:10B0980002FB00339973FFF753BD00BF48460020F9
:10B0A800024B0B2202FB0030007970474846002013
:10B0B800024B0B2202FB00304079704748460020C3
:10B0C800024B0B2202FB0030C07970474846002033
:10B0D800024B0B2202FB0030807970474846002063
:10B0E800024B0B2202FB0030007A704748460020D2
:10B0F800024B0B2202FB0030407A70474846002082
:10B10800024B0B2202FB0030807A70474846002031
:10B11800024B0B2202FB0030007B704748460020A0
:10B12800024B0B2202FB0030407B70474846002050
:10B13800024B0B2202FB0030807B70474846002000
:10B14800034A00EB8003134483F87810FFF756BED8
:10B1580048460020034B00EB800213445970FFF768
:10B168004DBE00BFC0460020034B00EB80021344D5
:10B178009970FFF743BE00BFC0460020034B00EBA9
:10B1880080021344D970FFF739BE00BFC0460020C3
:10B19800034B00EB800213441971FFF72FBE00BF69
:10B1A800C0460020034B00EB8000184490F878005C
:10B1B800704700BF48460020024B00EB800018444F
:10B1C80040787047C0460020024B00EB80001844CE
:10B1D80080787047C0460020024B00EB800018447E
:10B1E800C0787047C0460020024B00EB800018442E
:10B1F80000797047C0460020034A00EB400313441F
:10B2080083F86810FFF7A2BD48460020034B00EB07
:10B21800400213445970FFF799BD00BFB0460020A3
:10B22800034B00EB400213449970FFF78FBD00BF3A
:10B23800B0460020034B00EB4000184490F868002B
:10B24800704700BF48460020034B00EB40001844FD
:10B2580090F90100704700BFB0460020024B00EB98
:10B268004000184480787047B0460020034B03EB39
:10B27800C00383F84C10FFF721BD00BF48460020EB
:10B28800034B03EBC00383F84D10FFF717BD00BF56
:10B2980048460020034B03EBC00383F84E10FFF72A
:10B2A8000DBD00BF48460020034B03EBC00383F8E5
:10B2B8004F10FFF703BD00BF48460020034B03EBC8
:10B2C800C00383F85010FFF7F9BC00BF48460020C0
:10B2D800034B03EBC00383F85110FFF7EFBC00BF2B
:10B2E80048460020034B03EBC00383F85210FFF7D6
:10B2F800E5BC00BF4846002010B5064B044603EBEA
:10B30800C00383F85310FFF7D9FC2046BDE810406E
:10B31800FFF71CBD48460020024B03EBC00090F825
:10B328004C00704748460020024B03EBC00090F8E1
:10B338004D00704748460020024B03EBC00090F8D0
:10B348004E00704748460020024B03EBC00090F8BF
:10B358004F00704748460020024B03EBC00090F8AE
:10B368005000704748460020024B03EBC00090F89D
:10B378005100704748460020024B03EBC00090F88C
:10B388005200704748460020024B03EBC00090F87B
:10B3980053007047484600202DE9F0472E4D1E46C1
:10B3A8002B1893F88C3004468A469146DDF82080A5
:10B3B800099F042B1AD8DFE803F003080D121700C1
:10B3C800FFF7BEFB2B19012212E0FFF777FC2B19C0
:10B3D80002220DE0FFF712FD2B19032208E0FFF708
:10B3E800B5FC2B19042203E0FFF73EFC2B190022C1
:10B3F80005EBC40483F88C2094F85220164B012ADC
:10B4080012D002D3022A14D020E0BAF1000F03D0E0
:10B418001B689B0C8AF80030B9F1000F16D02B6816
:10B428009B0A89F8003011E086B11B689B0A3360DB
:10B438000CE01EB11B68DB0B5B013360B8F1000F39
:10B4480004D02B68C3F3842388F800300FB12B682D
:10B458003B70BDE8F08700BF48460020054B0B2233
:10B4680002FB0033DA7A04331AB90122DA71FFF7E2
:10B4780067BB704748460020054B0B2202FB003390
:10B48800DA7A04331AB10022DA71FFF759BB704730
:10B498004846002006281BD8DFE800F004070A0DFC
:10B4A800111417000B4B1B6811E00A4B9B6C0EE044
:10B4B800084BDB6A0BE0074BD3F8883007E0054BF5
:10B4C8005B6F04E0034B5B6E01E0024BDB7A0B60C1
:10B4D800704700BF48460020704770477047704764
:10B4E80070477047704712230B800148704700BFB0
:10B4F8004400002004230B800048704756000020B9
:10B5080000207047002070470020704770B5084C35
:10B51800002223688A4207D03F2B03D8865CE518AF
:10B528002E7101330132F5E72360002070BD00BFA2
:10B53800D846002010B5044C0A460448214607F0B6
:10B54800BDFF204610BD00BF9B610020E0630108DD
:10B5580010B5044C0A460448214607F0AFFF2046C0
:10B5680010BD00BF9B610020F863010810B5044CB2
:10B578000A460448214607F0A1FF204610BD00BF37
:10B588009B6100201064010810B5044C0A46044869
:10B59800214607F093FF204610BD00BF9B610020A5
:10B5A8001864010810B5044C0A460448214607F0FF
:10B5B80085FF204610BD00BF9B6100202364010861
:10B5C800202811D0212821D1114B9A69100A0A701C
:10B5D8004870100C120ECA701A7F88700A715A7F50
:10B5E8009B7F4A718B7111E08A784878120442EA8D
:10B5F80000220878064B0243C87842EA00629A6142
:10B608000A791A774A795A778A799A77002070479F
:10B6180044000020F7B5274C4FF4C05300260327F9
:10B6280000932046022369468DF804308DF8057092
:10B638008DF806608DF8076005F05EFE20460B2148
:10B648000A2205F0D5FE20460A220C2105F0D0FE7C
:10B6580001254FF400732046694600938DF8057064
:10B668008DF804608DF806508DF8076005F044FEEB
:10B6780020460A22092105F0BBFE4FF480632046CC
:10B68800694600938DF806508DF807508DF80570BF
:10B6980005F032FE0A210A46204605F0A9FE294691
:10B6A8004FF4804006F002F88020294605F0DAFFC2
:10B6B80003B0F0BD0000024007B54FF4C06007F0CA
:10B6C800E7F943238DF804300322012301A88DF8FC
:10B6D80005308DF806208DF8073007F0E3F903B040
:10B6E8005DF804FB782358430722B0FBF2F00023EF
:10B6F80001338342FCD970474FF47A735843FFF7FC
:10B70800F1BF684620F007018D4601B5034808F0EF
:10B71800AFFCBDE801408546704700BFD44D00200E
:10B72800F0B500238B420ED0074A084E15686C1CF2
:10B738001460C75CB4F5006F28BF0024775528BF94
:10B7480014600133EEE7F0BD9C4A00209B590020AD
:10B75800074B10B51A684AB1002305490C1D1C5D3A
:10B76800C45401339342F8D100230B60104610BD36
:10B77800D8460020084B1B68082B0BD90023064A23
:10B78800111D595CC1540133092BF8D100231360F2
:10B798000120704700207047D846002007B5064AA8
:10B7A800064802F13C03009301212032044B07F0C4
:10B7B800EBFA03B05DF804FB44000020D44D0020F0
:10B7C80058010020014808F026BC00BFD44D0020D5
:10B7D80037B5D04DA8782C46022800F2E3826B7862
:10B7E800A52B00F06F8200F28280852B00F02D815E
:10B7F80027D8072B00F05B810FD8032B00F0258199
:10B8080005D8012B00F0FB8040F2F48002E1052B03
:10B8180000F0368140F220813BE1812B00F0EF807F
:10B8280009D80D2B00F06581802B00F0E3800C2BEC
:10B8380040F0F68249E1832B00F00E8140F27D81D1
:10B84800E8E0952B00F0A18127D88C2B00F092819D
:10B8580014D8872B00F07C81C0F012818A2B40F02D
:10B86800DF82400140F0140101F0F401002001AA38
:10B87800FEF770FEEB788DF8063070E1932B00F040
:10B88800388100F222818D2B40F0CA82400140F0BD
:10B898001A0101F0FA01002055E1A12B00F0F7810F
:10B8A8001AD89A2B00F08581A02B00F0EA81992BF9
:10B8B80040F0B682400140F0180101AA002001F0D2
:10B8C800F801FEF747FEEA789DF8053002F00F020E
:10B8D80023F00F0313437CE1A32B00F0DE8100F279
:10B8E800E281D5F80310C9B2FFF776FB9BE2B62BCD
:10B8F80000F0608236D8AD2B00F0288214D8A92B2E
:10B9080000F00B8205D8A72B00F0FB8140F2EA81FA
:10B91800FDE1AB2B00F0078200F20B82D5F8031093
:10B92800C9B2FFF721FC7EE2B12B00F021820AD8D0
:10B93800AF2B00F0118200F21582D5F8031049B23E
:10B94800FFF764FC6FE2B32B00F01E82C0F0168292
:10B95800B52B40F06582704B03EB4010D5F80330EF
:10B96800836160E2C82B00F0518114D8C12B00F02C
:10B978003A8108D8B82B00F03982C0F03082C02B49
:10B9880000F095804CE2C32B00F03981C0F0318182
:10B99800C72B7ED044E2D22B00F0338215D8CC2BB3
:10B9A80000F04481D12B00F02782C92B40F0388267
:10B9B800594BE97803EB40131A6922F07F4242EAB7
:10B9C80001621A61FCF7C6FE2DE2D52B00F0358125
:10B9D80009D8D42B40F024824F4B03EB4010D5F804
:10B9E800033043611FE2D62B00F02E81FE2B00F0BE
:10B9F800328115E2410101F0E001002005E040013B
:10BA080040F0020101F0E2010020D4F80320FEF723
:10BA18000CFD08E2400140F0080101F0E8010020B7
:10BA2800D4F80320FEF7EFFCA178D4F803204901ED
:10BA380041F0060101F0E6010020002AB8BF524299
:10BA4800FEF7E1FCA378012117E0400140F00A016C
:10BA580001F0EA01002076E0400140F0060101F023
:10BA6800E601D4F803200020FEF7CDFCA378D4F833
:10BA780003102A4A42F823100021294AD154D2E15E
:10BA8800D4F80310FEF7D9FDA378D4F80310254A9B
:10BA9800F0E7254B01221A541F4BE17803EB4013C2
:10BAA8005972224B1B5C022B40F0BD8194E11E4B66
:10BAB80001221A54184BE17803EB401399721B4B7F
:10BAC8001B5C002B40F0AF8186E1400140F014017F
:10BAD80001AA002001F0F401FEF73CFDD4F8032090
:10BAE8009DF8053012B143F0020323E023F002036E
:10BAF80020E0400140F0140101AA002001F0F40107
:10BB0800FEF728FDD4F803209DF8053082B143F0F4
:10BB180001030FE0C8530020A84C0020FC58002067
:10BB28001C470020F0540020584D00205D4D002097
:10BB380023F001038DF8053011E0400140F00401C5
:10BB480001F0E4010020D4F80320FEF75CFC6AE170
:10BB5800400140F00E0101F0EE010020F3E7A1786A
:10BB68000020490141F0140101F0F40101AAFEF797
:10BB780025FC58E1AD4BE97803EB4013D972C1F1CC
:10BB88000801C9B2FFF7E8F94DE1400140F014019E
:10BB980001AA002001F0F401FEF7DCFCD5F803202F
:10BBA8009DF8053012B143F00403C3E723F0040302
:10BBB800C0E7400140F0180101AA002001F0F80197
:10BBC800FEF7C8FC9DF80530EA7803F00F0343EA56
:10BBD8000213A1788DF80530490141F018010020C1
:10BBE80001F0F801C2E7914B03EB4010EB780372C8
:10BBF80019E1D5F803208D4B40011A5013E18B4B06
:10BC080003EB4010D5F8033043600CE1884B012268
:10BC18001A54864BD5F8032003EB4013DA77854B8B
:10BC28001B5C032B40F0FF80E978D5E07F4B03EBEA
:10BC38004010D5F80330C381F5E07C4B03EB40108E
:10BC4800D5F803308377EEE0784B03EB4010D5F856
:10BC580003308383E7E0D5F80330744A052B4FEAB5
:10BC680040130AD874491344C97801221973704BD8
:10BC78001A540846FDF70AF9D5E0134400221A734E
:10BC8800D1E0D5F80310C9B2FFF776F9CBE0D5F8C3
:10BC98000310C9B2FFF77EF9C5E0D5F80310C9B2A1
:10BCA800FFF7A4F9BFE0FFF703FAD5F8031020B9AE
:10BCB800A878C9B2FFF7AEF9B5E0A878C9B2FFF71E
:10BCC800D1F9B0E0FFF7F4F9AB78D5F8031020B953
:10BCD8001846C9B2FFF7A8F9A5E01846C9B2FFF798
:10BCE800D5F9A0E0FFF7E4F9D5F8031020B9A87852
:10BCF800C9B2FFF7A3F996E0A878C9B2FFF7BCF973
:10BD080091E0D5F80310C9B2FFF7A2F98BE0D5F896
:10BD18000310C9B2FFF714FA85E0D5F80310C9B2C9
:10BD2800FFF718FA7FE0D5F80310C9B2FFF726FA33
:10BD380079E0D5F80310C9B2FFF72AFAAA783F4B81
:10BD480003EBC203D5F803205A716CE0D5F8031051
:10BD5800C9B2FFF751FA66E0D5F80310C9B2FFF788
:10BD680085FA60E0D5F80310C9B2FFF789FA5AE0FE
:10BD7800D5F80310C9B2FFF78DFA54E0D5F80310CF
:10BD8800C9B2FFF791FA4EE0284B03EB40135A7AF9
:10BD98000833A72A02D89B78A72B05D9D4F8031013
:10BDA800012904D004223CE0D5F80310C9B2FFF7FA
:10BDB8008FFA38E0D5F80320204B43F8302022B919
:10BDC80003EBC0035979FFF7E3F9A078194B1B5C23
:10BDD800012B28D1184BD978FCF720FB23E0174B0F
:10BDE80003EBC000D5F8033003711CE0D5F803104D
:10BDF800C9B2FFF705F916E0D5F80310FCF76AFC9D
:10BE080011E00A4BD5F8031003EB40131A6921F02F
:10BE18007F4102F07F420A431A61FCF793FC02E07B
:10BE28000322074B1A7003B030BD00BFA84C002096
:10BE3800584D00205D4D0020C8530020044C0020C0
:10BE4800E454002073B5CE4ECE4CB0783546022867
:10BE580000F28A827378A42B00F02D8200F2A5806C
:10BE6800842B00F04E8136D8082B00F06B8115D852
:10BE7800032B00F0508105D8012B00F0398140F2E6
:10BE880032813EE1052B00F04F81C0F04B81062B3B
:10BE980000F04E81072B00F0508163E20D2B00F07B
:10BEA8005A8109D80A2B00F08C81C0F063810B2BD2
:10BEB80000F076810C2B35E0812B00F0198103D836
:10BEC800802B00F010814DE2822B00F08681832BBD
:10BED80000F0288146E2952B00F0998132D88A2B10
:10BEE80000F082810ED8862B00F01E81C0F01381ED
:10BEF800872B40F03782400140F00E0101F0EE013F
:10BF0800002004E18D2B00F07B8107D88C2B40F0BA
:10BF18002982FFF749F8C0F10800FAE0932B00F0F6
:10BF28001A81942B40F01E82400140F0140101F068
:10BF3800F401002001AAFEF70DFB9DF80530C3F3BC
:10BF4800400315E19D2B00F0FD801BD89A2B00F0D3
:10BF58006C8110D8992B40F00582400140F01801FF
:10BF680001F0F801002001AAFEF7F4FA9DF8053067
:10BF780003F00F03FCE09B2B00F012819C2B00F0D8
:10BF88002081EFE1A12B00F0908105D8A02B40F093
:10BF9800E981FFF711F8BCE0A22B00F08981A32BFF
:10BFA80040F0E081FFF784F8B3E0B72B00F0CE81D2
:10BFB8003ED8AD2B00F0B08119D8A82B00F0A08195
:10BFC80005D8A62B00F08E8140F2818195E1AA2B3D
:10BFD80000F09C81C0F09781AB2B00F09A81AC2BCC
:10BFE80040F0C081684B03EBC0004379C0E0B22B3E
:10BFF80000F09E810DD8AF2B00F09481C0F08F81A6
:10C00800B02B00F09281B12B40F0AC81FFF794F98E
:10C018007FE0B42B00F09281C0F08D81B52B00F049
:10C028009081B62B40F09E81574B53F830309FE0FB
:10C03800CC2B00F0168129D8C32B00F0088112D828
:10C04800C02B7AD005D8B82B40F08C81FFF738F890
:10C058005FE0C12B00F0F680C22B40F083814B4B90
:10C0680040011B5884E0C72B62D004D8C42B40F091
:10C078007981474B59E0C82B00F0EE80C92B40F07E
:10C088007181424B03EB4010C37C71E0D22B00F06E
:10C09800628111D8CF2B00F0E98004D8CE2B40F074
:10C0A80061813C4B41E0D02B00F0F380D12B40F074
:10C0B8005981FCF7F3FA2CE0D52B00F0EC8007D877
:10C0C800D42B40F04F81314B03EB401043694FE0D4
:10C0D800D62B00F0E580FE2B40F044812B4B03EB80
:10C0E8004010037B44E0410101F0E001002005E03D
:10C0F800400140F0020101F0E2010020FEF726FCB9
:10C1080007E0400140F0080101F0E8010020FEF7D7
:10C1180038FA60602AE1400140F00A0101F0EA01C2
:10C128000020F4E71C4B00E01C4B53F820301FE0C4
:10C13800164B03EB4010437A1AE0144B03EB401004
:10C14800837A15E00020FEF700FAAB785B0018410F
:10C1580000F001030CE0400140F0140101F0F4018B
:10C16800002001AAFEF7F6F99DF8053003F0010357
:10C178006360FBE00130C0B2FCF7ADF9C9E700BF6E
:10C18800C8530020E4540020044C0020A84C002090
:10C19800E44B0020244C0020FC580020F0540020E0
:10C1A80001AA00207C21FEF7D5F9AA7802235200C3
:10C1B80003FA02F29DF806301A420CBF002301234D
:10C1C800D6E701AA00207C21FEF7C4F9AB789DF8D8
:10C1D80006205B0042FA03F3C8E7400140F004017F
:10C1E80001F0E401002092E7400140F0140101F061
:10C1F800F401002001AAFEF7ADF99DF80630B7E773
:10C20800400140F01A0101F0FA0100207FE74001E7
:10C2180040F0140101F0F401002001AAFEF79AF998
:10C228009DF80530C3F38003A2E7400140F01801F0
:10C2380001F0F801002001AAFEF78CF99DF80530FD
:10C248001B0995E7524B03EB4010037A90E7504BDC
:10C2580003EB401043688BE74D4B03EB4010C37F63
:10C2680086E74B4B03EB4010C38981E7494B00221B
:10C27800195C626011B1484901254D601A54474B59
:10C288001A5C1AB1626842F00202626000221A5413
:10C298006CE0434B53E03E4B03EB4010837F67E772
:10C2A8003B4B03EB4010838B62E7FEF78DFE30E7D4
:10C2B800FEF7F6FE2DE7FEF7FBFEB37818B9184631
:10C2C800FEF706FF25E71846FEF722FF21E7FEF7EF
:10C2D800EFFE18B9B078FEF703FF1AE7B078FEF75B
:10C2E80027FF16E7FEF7E4FE18B9B078FEF700FF5F
:10C2F8000FE7B078FEF714FF0BE7FEF701FF08E73A
:10C30800FEF750FF05E7FEF757FF02E7FEF75CFF71
:10C31800FFE6FEF761FFFCE6FEF78CFFF9E6FEF7A5
:10C3280093FFF6E6FEF7F8FFF3E6FEF7FDFFF0E60B
:10C33800FFF70AF8EDE6FFF717F8EAE6194B1B5C7A
:10C3480016E7134B03EB4010836911E7164B03EB19
:10C35800C00003790CE70E4B03EB4010036923F090
:10C368007F4305E7032300E0042323700F4B1B786A
:10C3780063B10F4B62681A600E4B1AB91A6842F023
:10C38800080202E01A6822F008021A6002B070BDC2
:10C39800A84C0020A04C0020E45400201F4C002092
:10C3A800A34C0020004C0020044C0020DF54002047
:10C3B800D0540020D053002038B5934A93781446BF
:10C3C800022B00F01A81032B00F02C81002B40F087
:10C3D800B18153784D2B00F0B18031D8452B7BD0FB
:10C3E80018D8422B6BD009D8402B64D0412B40F091
:10C3F8009F81D178854B0020197064E0432B66D06B
:10C40800442B40F09581D2F8033080491C2041F834
:10C418001C3F6CE0482B6FD00CD8462B61D0472BC3
:10C4280040F08681794DD2F80330294641F8083F1B
:10C438000820B1E04B2B71D07BD8492B62D077E133
:10C44800542B00F0B3801BD8512B00F08F8009D8F3
:10C458004F2B78D0502B40F06B81D1786B4B162046
:10C46800997530E0522B00F09080532B40F060819A
:10C47800664DD2F80330294641F8103F10208BE072
:10C48800832B00F0AB800BD8552B00F09B80572BEB
:10C4980040F04E81D3785D49272001F8273F8FE08F
:10C4A800852B00F0A580C0F09E80FF2B40F04081D6
:10C4B800D278574B40E140F2FF70D17803E0D17851
:10C4C800524B01205970BDE83840FDF729BDD1789D
:10C4D8004E4B04201971F6E7D1784C4B0520597161
:10C4E800F1E7D2F8033049490C2041F80C3F042207
:10C4F800BDE83840FDF777BDD3784449262001F8D8
:10C50800263F5DE0D278414B0AB9DA7503E041492C
:10C518000122DA754A601720D97DD4E73B4CD178DF
:10C528000320E170FDF7FCFCE078BDE83840FCF73B
:10C5380083BED178354B02209970C4E7D178334B4C
:10C5480015205975BFE7D2F80310304CC9B219202D
:10C558006176FDF7E5FC607EBDE8384010F001002B
:10C568001ABF002001210146FEF72CBA274B1A7D7D
:10C578001D4612F0010F04D0E378DB0701D4FDF764
:10C5880027FCE178142029759DE7D2F803301F496C
:10C59800202041F8203FAAE70422FDF724FD68790E
:10C5A800A9682A69BDE83840FCF784BFD2F803308F
:10C5B800012B00F2BF80D37814491A2001F81A3FE2
:10C5C800012295E7D2F80330012B00F2B3800E4B1D
:10C5D8000E49DB781B2001F81B3FF1E7D2F8032056
:10C5E8000D4B5A6038BDD2F803200C4B1A6038BD89
:10C5F800D2F80320084B9A6038BD5178084BD2F81E
:10C60800032043F8212038BDC8530020040000202F
:10C61800DE540020E45400201C470020E054002091
:10C62800FC54002053782E2B00F28280DFE803F0C0
:10C6380018212A80808080808033383D80808080E7
:10C6480080808080808080808080804244464D4FFA
:10C6580051808080808080585D62676C71767B0035
:10C66800364BD4F803201A60FBF7FCFD344BD86036
:10C6780038BD324BD4F803205A60FBF7F3FD304B3A
:10C68800186138BD2D4BD4F803209A60FBF7EAFDFA
:10C698002B4B586138BDD4F80320284BDA6038BDDD
:10C6A800D4F80320254B1A6138BDD4F80320234B56
:10C6B8005A6138BD002002E000200BE00120D4F8C8
:10C6C8000310BDE83840FEF7A2B8012002E00220BE
:10C6D800F5E70220D4F80310BDE83840FEF7C1B8EA
:10C6E800D4F80320154B9A6138BDD4F80320134BB6
:10C6F800DA6138BDD4F80320104B1A6238BDD4F87B
:10C7080003200E4B5A6238BDD4F803200B4B9A62B3
:10C7180038BDD4F80320094BDA6238BDD4F80320B9
:10C72800064B1A6338BDD4F80320044B5A6338BD4E
:10C73800032200E00422034B1A7038BD144D002078
:10C748001C470020E45400202DE9F8430446154610
:10C758000E4600294AD0002848D0814246D04FEAE8
:10C7680042185FFA88F848F0060739460020FEF7B5
:10C77800EDF848F00C0181460020FEF7E7F8804606
:10C78800204608F021FC0446304608F01DFC01460E
:10C79800204608F025FD0646484608F015FC3146B7
:10C7A80008F01EFD08F02EFE0446404608F00CFC7A
:10C7B800314608F015FD08F025FE002C08BF0124BD
:10C7C8000B49002814BF80464FF00108304608F096
:10C7D800F1FD18B128464146FDF72FFF22460020FB
:10C7E8003946FDF722FE034B01225A55BDE8F8836E
:10C7F8000000A0411C47002070B50C4D04462B5C7E
:10C808009BB1C6B20A4B710141F0060153F82420CE
:10C81800002001F0E601FDF7F6FD064B304653F81F
:10C828002410FDF70AFF00232B5570BD1C4700207C
:10C83800FC580020F05400202DE9F043C54FDFF8E4
:10C8480028833B78D7F803606422222B85B088F8C8
:10C85800013088F80020C8F804603D46444601F0DD
:10C8680093835CD80F2B00F0E08727D8072B00F0C4
:10C878006B8311D8032B00F0368107D8012B00F009
:10C88800BE80022B00F0FA8001F0DCBD052B00F021
:10C89800538340F2E88053E30B2B00F01B8706D844
:10C8A800092B00F0E88540F2818400F0E8BD0D2BEB
:10C8B80000F0448740F22C8700F090BF192B01F05C
:10C8C800F48014D8152B01F0498007D8132B00F0F9
:10C8D800E887142B01F0208001F0B4BD172B9E4B84
:10C8E80001F0C98001F2D480DE6101F0ADBD1E2BDC
:10C8F80000F001870CD81B2B01F0F980C1F0E6800D
:10C908001C2B41F09F85944B00221A7601F09CBDA8
:10C91800202B01F0818241F2328201F0E1BA812BB1
:10C9280001F0CD8335D8412B01F0B78317D8252BDB
:10C9380001F0748307D8232B01F02D83242B01F0F9
:10C94800318301F07FBD272B01F09683C1F06F83FF
:10C95800402B41F0778502F0E3FA01F075BD452BD5
:10C9680001F0A48308D8432B01F09A8301F29B833A
:10C9780002F0DFFA01F068BD472B01F09D83C1F09A
:10C988009883802B41F05E85734B00221A7601F064
:10C998005BBD882B01F012841BD8842B01F0C18366
:10C9A8000DD8822B01F0A083832B41F04B856A4B75
:10C9B800002183F8441083F82C1101F099BB862BD1
:10C9C80001F0C18301F21C84634B00221A7601F046
:10C9D8003BBD8C2B01F0868406D88A2B01F0668437
:10C9E80041F2358401F079BCF22B01F0E584FF2B8C
:10C9F80001F01F858D2B41F0258501F09ABCBB788D
:10CA0800022B37D80024AB789C4209D0534A02EB5A
:10CA180043139B7F13B302EB4412927F9A421DD1BA
:10CA28004D4B0122E2544E4B0026E654E7B24D4BE3
:10CA380039467F01E65430460222FFB2FDF7B9FDC0
:10CA4800304647F0060140F2FF72FDF7DCFC304645
:10CA580047F00801D5F80320FDF7D5FC0134032C75
:10CA6800D1D101F0F1BCB878022868D9394B5B788C
:10CA7800022B64D00423237001F0E6BCBB78022BA0
:10CA8800F8D80024AB789C4209D0344A02EB43130F
:10CA98009B7F1BB302EB4412927F9A421ED12E4B0E
:10CAA8000122E2542E4B0026E654E7B22D4B3946BC
:10CAB8007F01E65430460222FFB2FDF77AFD304688
:10CAC80047F0060140F2FF72FDF79DFCD5F8032000
:10CAD800304647F008015242FDF795FC0134032C1B
:10CAE800D0D101F0B1BCBB78022BC3D80024AB78FD
:10CAF8009C4209D0194A02EB43139B7FD3B102EB46
:10CB08004412927F9A4215D1154B0026E654154BD4
:10CB1800E7B23846E65402F0CDFC394630460222E8
:10CB28007F01FDF746FD47F00801304601F0E801B6
:10CB3800FDF7F4FC0134032CD9D101F085BC6B78E6
:10CB4800032B00F2F581DFE813F011005F00C1004C
:10CB5800CD0100BFC85300201C470020A84C00206E
:10CB6800A04C00201F4C0020E4540020FFF744FE96
:10CB7800A978BB4B00245C54BA4BBB4E5C540123D0
:10CB88008B403278490122EA0303204601F0E00194
:10CB9800D5F803203370FDF748FC2046A9782246D3
:10CBA800FDF707FDB14FAB7807EB43139B7F002BD5
:10CBB80001F04A84AB789C4221D007EB441207EB82
:10CBC8004313927F9B7F9A4219D12046FFF714FEA8
:10CBD8000123A34032785FFA84F822EA0303337012
:10CBE800A34B4FEA4811002001F0E001D3F80320DD
:10CBF800FDF71BFC002041460246FDF7DAFC013434
:10CC0800032CD7D101F020BCFFF7F6FDAB78944A8E
:10CC18000026D654934A3046D6545B0143F00201AD
:10CC280001F0E201FDF792FEA97801238B408E4FB7
:10CC3800D5F803803A788044490122EA0303304654
:10CC4800424601F0E0013B70FDF7EFFB324630460B
:10CC5800A978FDF7AEFC854BAA78C4F8048003EBED
:10CC68004212927F9846002A01F0EE833446A87853
:10CC7800844226D008EB441208EB4013927F9B7F36
:10CC88009A421ED1E6B24FEA46195FFA89F9FFF7D0
:10CC9800B3FD49F002010020FDF758FE744B3978C6
:10CCA800D3F803200123A340024421EA0303002010
:10CCB80049463B70FDF7B9FB002031460246FDF7B7
:10CCC80078FC0134032CD2D101F0BEBB10F0C007B0
:10CCD80027D102283FF6CEAE142E3FF7CBAE654BD8
:10CCE80006EB4606064453F82640FFF785FDA9786B
:10CCF80001228A405A4B5F545A4B5F545A4B4901A0
:10CD0800187801F0E00120EA02021A70384622463B
:10CD1800FDF78BFB3846A9783A46FDF74AFC01F047
:10CD280093BB402F40F0A880142E3FF7A3AE0024F9
:10CD3800019402940394234640FA03F2D10706D5DE
:10CD480004AA22440134032C02F8103C02D0013317
:10CD5800032BF1D10027A7421DDA1DF807804046B2
:10CD6800FFF74AFD4FEA481141F00201002001F0A7
:10CD7800E201FDF7EBFD06EB460398443D4B01AAA3
:10CD880053F82830C01A80EAE073A3EBE07342F846
:10CD980027300137DFE7012C35DD022C019E029C8C
:10CDA80008D1A64201DD304628E0204631469DF8EC
:10CDB800002026E0A642039F0EDDBE4207DD304676
:10CDC80021469DF80120FFF7BFFC30460DE03846AC
:10CDD80031469DF800200EE0BC429DF8002008DD99
:10CDE80020463146FFF7B0FC204639469DF8022020
:10CDF80007E038463146FFF7A7FC38469DF8012082
:10CE08002146FFF7A1FC0024AB7843FA04F2D207CD
:10CE180020D5174A1749D2F80320002602EB420210
:10CE2800224451F822200E49E7B2CE540D49CE547F
:10CE38000121A1400C4B187820EA010119707901F1
:10CE4800304601F0E001FDF7F0FA30463946324647
:10CE5800FDF7AFFB0134032CD6D101F0F5BA00BFC2
:10CE68001F4C0020A04C0020F14B0020A84C0020B3
:10CE7800C8530020D4530020802F41F0E582142E9F
:10CE88003FF7F8AD0024AB78D44E2341DF0724D513
:10CE9800D6F80330D24A03EB43032344204652F822
:10CEA8002380FFF7A9FCB378CE4A0026D654CE4A91
:10CEB800E7B2D6540122A240CC4B3046197821EA79
:10CEC800020279011A7001F0E0014246FDF7ADFA5D
:10CED800304639463246FDF76CFB0134032CD2D17B
:10CEE80001F0B2BA040601F1AF82BD4B06EB46066B
:10CEF800064453F82660FFF77FFCA97801228A4090
:10CF0800B84B00245C54B84B5C54B84B49011878B2
:10CF180001F0E00120EA02021A7020463246FDF7CD
:10CF280084FA2046A9782246FDF743FB01F08CBA23
:10CF38000323237001F088BAFEF74AFC01F084BA93
:10CF4800FEF780FF01F080BABB78022B3FF692AD66
:10CF58007A789A2A2ED8992A80F0AB80822A00F013
:10CF68008E800BD8062A6ED003D8042A65D0052AED
:10CF78000BE0072A75D00C3A012A13E08C2A00F03E
:10CF880084800AD8832A58D0862A40F00B81184614
:10CF98000C21FDF704FC01F057BA8D2A00F08380BC
:10CFA800933A022A00F2FE8018461421FDF7F7FB97
:10CFB80001F04ABAC82A00F0AF8010D8C12A00F0A0
:10CFC8008C8004D8B52A7AD0C02A4AD0EAE0C32A8D
:10CFD80000F09780C0F08B80C72A34D0E2E0D42AD2
:10CFE80000F0B68013D8CC2A00F0A480D22A40F0F2
:10CFF800D980580100F110027D49101A02331144FA
:10D0080000EB43100422FCF7EEFF01F01DBAD62A0C
:10D0180000F0BA80C0F0AA80FE2A40F0C380744AAB
:10D02800580111180C311044081A023300EB431050
:10D038000122FCF7D8FF01F007BA18460621FDF7D0
:10D04800AEFB01F001BA6A4A5901501809300A4486
:10D05800801A023300EB4310517AFCF761FF01F0AC
:10D06800F3B9634A590150180A300A44801A023346
:10D0780000EB4310917AFCF753FF01F0E5B918462D
:10D088000421FDF78CFB01F0DFB9594A580111184A
:10D098000B311044081A023300EB43100122FCF74D
:10D0A800A2FF01F0D1B918461A21FDF778FB01F06B
:10D0B800CBB918461821FDF772FB01F0C5B9580124
:10D0C80000F118024A49101A0233114400EB4310C8
:10D0D8000422FCF788FF01F0B7B9454A580102EB72
:10D0E80043124830117AFCF71BFF01F0ADB94049F3
:10D0F800981C400101EB43110422FCF774FF01F076
:10D10800A3B93B49580101EB4311443004310422CF
:10D11800FCF769FF01F098B9354A580111181F3119
:10D128001044081A023300EB43100122FCF75BFF9E
:10D1380001F08AB92E4A580111180E311044081A04
:10D14800023300EB43100222FCF74DFF01F07CB9DB
:10D15800274A5801111814311044081A023300EBF9
:10D1680043100422FCF73FFF01F06EB9204A580132
:10D1780011181E311044081A023300EB4310012223
:10D18800FCF731FF01F060B9194A580111181C3138
:10D198001044081A023300EB43100222FCF723FF65
:10D1A80001F052B90323237001F04EB9BB780B4E3E
:10D1B800022B3FF65FAC72789A2A51D8992A80F0F0
:10D1C800F680822A00F0D0801AD8062A00F0B080B3
:10D1D80010D8042A00F09680052A18E0C8530020C9
:10D1E800D45300201F4C0020A04C0020F14B0020FD
:10D1F800A84C0020072A00F0A9800C3A012A27E051
:10D208008C2A00F0B7801ED8832A7BD0862A40F06B
:10D218002E8118460C21FDF79FFAAC780020610199
:10D2280041F00C0101F0EC01FDF7ABF9C94BCA4A1A
:10D2380043F82400A8780021115453F82010FDF772
:10D24800FCF901F001B98D2A00F0AB80933A022A6B
:10D2580000F20D8118461421FDF77EFA01F0F4B8AA
:10D26800C72A65D01AD8C12A00F0B58005D8B52AD2
:10D2780000F0A380C02A69D0F9E0C22A00F0B58086
:10D28800C32A40F0F480B549580101EB43114430FA
:10D2980004310422FCF732FF01F0D6B8D42A00F09A
:10D2A800BC8013D8C82A00F0AA80CC2A40F0DF80BE
:10D2B800AA4A580111180E311044081A023300EB1B
:10D2C80043100222FCF71AFF01F0BEB8D62A00F07C
:10D2D800C080C0F0B080FE2A40F0C9809F4C5A013F
:10D2E800A1180C312244881A023300EB43100122A2
:10D2F800FCF704FFB37804EB4314207BFBF7C6FD6F
:10D3080001F0A2B818460621FDF726FAAC780020ED
:10D31800610141F0060101F0E601FDF732F9904B99
:10D328008D4A43F82400AB780021D15401F08CB821
:10D338008A4A5C01111909311444081B023300EBB5
:10D348004310FCF7D5FE607201F07EB8834A5C0199
:10D3580011190A311444081B023300EB4310FCF77F
:10D36800C7FEA07201F070B818460421FDF7F4F961
:10D3780001F06AB8794C5A01A1180B312244881A75
:10D38800023300EB43100122FCF7B8FEB07804EB3F
:10D398004014E17AC1F10801C9B2FDF7DDFD01F0E1
:10D3A80053B818461A21FDF7D7F901F04DB81846B9
:10D3B8001821FDF7D1F901F047B8580100F118021A
:10D3C8006649101A0233114400EB43100422FCF79B
:10D3D80095FE01F039B85801604C483004EB43140D
:10D3E800FCF786FE207201F02FB85C49981C4001BA
:10D3F80001EB43110422FCF781FE01F025B8574ADE
:10D40800580111181F311044081A023300EB431059
:10D418000122FCF773FE01F017B8504A58011118A1
:10D4280014311044081A023300EB43100422FCF7AD
:10D4380065FE01F009B8494A580111181E31104417
:10D44800081A023300EB43100122FCF757FE00F0E4
:10D45800FBBF424A580111181C311044081A023304
:10D4680000EB43100222FCF749FE00F0EDBF032356
:10D47800237000F0E9BFFEF79FFF00F0E5BFBA7820
:10D48800384B022A00F0AE80032A00F0B080002A50
:10D4980040F008815B78502B75D027D8462B55D0A3
:10D4A8000FD8422B4BD006D8402B43D0412B40F00D
:10D4B800F7802D4B8EE0442B2B4A43D044D8137968
:10D4C800ECE04B2B56D008D8482B4FD040D3492BF3
:10D4D80040F0E680244BDB7D80E04D2B50D04CD3D0
:10D4E8004F2B40F0DD80204B5B7ED7E0812B5BD05B
:10D4F80012D8542B4ED005D8522B1B4A46D047D8A9
:10D50800137DCBE0572B48D0802B4AD0552B40F0C9
:10D51800C780154BDB7EC1E0852B4FD004D8832B09
:10D5280048D049D80C4BA6E0FE2B52D054D8F02B4B
:10D538004FD0B5E040F2FF70FCF7DAFD89E00A4B06
:10D548005B78ABE0D369A9E05379A7E0064B75E0B7
:10D55800054B70E0F05400201C470020A84C002028
:10D56800FC580020C8530020040000208D4B93F87D
:10D57800263093E08B4BDB7890E08A4B9B788DE0EC
:10D58800884B5B7D8AE0874B9B7D87E0136A85E04B
:10D59800136983E0834B9B7E80E0824B93F82730AE
:10D5A8007CE0814B1B7E79E07F4B1B7E181F43423A
:10D5B800434173E07C4B3BE07C4B36E07A4A7C4944
:10D5C80093684B4303F540533933936023F000438A
:10D5D80064E0784B1B7861E0774B1B78003318BF09
:10D5E80001235BE05A78754B53F8223056E05B789C
:10D5F8002E2B55D8DFE803F0181B1E5454545454EE
:10D608005421242754545454545454545454545462
:10D618005454542A2F313335375454545454543BAA
:10D628003E4144474A4D5000654B1B6836E0644B09
:10D638005B6833E0624B9B6830E0614BDB682DE050
:10D648005F4B1B692AE05E4B5B6927E00020FDF712
:10D6580032F9606028E0002006E00120F7E70120A9
:10D6680002E00220F3E70220FDF73AF9F1E7544B14
:10D678009B6913E0524BDB6910E0514B1B6A0DE0CC
:10D688004F4B5B6A0AE04E4B9B6A07E04C4BDB6AE8
:10D6980004E04B4B1B6B01E0494B5B6B636003E0A1
:10D6A800032300E004232370464B1B78002B00F073
:10D6B800CB86454B62681A60444B2AB91A6842F017
:10D6C80008021A6000F0C0BE1A6822F008021A6048
:10D6D80000F0BABEBB78022B15D17B78372B0ED859
:10D6E800364903F5A770800001EB83010422FCF79B
:10D6F8007AFC00F0A9BE7B78142B40F2E982032360
:10D70800237000F0A1BE042388F8003000F09CBE0E
:10D71800BB78022B0ED12E4B5B78372BEFD82749DD
:10D7280003F5A770800001EB83010422FCF7E6FCF7
:10D7380000F08ABE0423237000F086BEB878022861
:10D748003FF698A97B78012B23D006D3022B24D14E
:10D7580001F0B8FE606000F077BE01F0A3FE1C4B3C
:10D768009A7800239A4209D01A4800EB4311897F1E
:10D7780051B100EB4210807F884205D10A4901204F
:10D7880058541549002058540133032BEAD100F0AE
:10D798005BBE01F08FFE00F057BE0323237000F03C
:10D7A80053BE00BF040000201C470020E0540020A6
:10D7B8006D4EC641504D0020DE540020FC54002020
:10D7C800144D0020DF540020D0540020D0530020F6
:10D7D800C8530020A84C00201F4C0020BB7813B170
:10D7E800022B05D01DE03046FAF70CFF00F02CBEE6
:10D7F800974B5878072808D81EB9FAF712FE00F098
:10D8080023BEFAF733FE00F01FBEFF287FF477AF80
:10D81800711C0ABF8F4BF0B21878FAF74BFE00F074
:10D8280013BE0423237000F00FBEBB78012B1CD05D
:10D8380005D3022B1DD17878FAF784FE0EE07878AC
:10D84800082802D8FAF747FE08E00A2802D1002380
:10D85800636010E00B2803D1FAF772FF60600AE0FA
:10D86800FF2808D1FAF7A2FEF8E77878FCF76CFAF7
:10D87800F4E704232370784B1B78002B00F0E48531
:10D88800744B62681A60754B2AB91A6842F008022C
:10D898001A6000F0D9BD1A6822F008021A6000F078
:10D8A800D3BD7A786B4B092A27D8DFE802F0050840
:10D8B8000B0E12181B1E21251A6816441CE01A6844
:10D8C800961B19E01A68564316E01A6892FBF6F69A
:10D8D80012E01A6892FBF6F106FB11260CE01A68B2
:10D8E800164009E01A68164306E01A68564003E035
:10D8F8001A68D2431A6000E01E601A68574B2AB9AA
:10D908001A6842F008021A6000F09EBD1A6822F0F8
:10D9180008021A6000F098BD4E4B1A684F4BB2428D
:10D92800196804DD21F0030141F0040108E00BBF90
:10D9380021F0060121F0050141F0010141F0020149
:10D9480019602AB91A6842F008021A6000F07CBD12
:10D958001A6822F008021A6000F076BD7B780C2B5A
:10D9680000F27285DFE803F0071019222B343E47D6
:10D978005059626B7E00394B1B681A0740F1648569
:10D98800374BDE6100F060BD344B1B681B0700F1AC
:10D998005B85334BDE6100F057BD304B1B68DF07FA
:10D9A80040F152852E4BDE6100F04EBD2B4B1B68BB
:10D9B800DD0700F149852A4BDE6100F045BD274BA4
:10D9C8001B685C0740F14085254BDE6100F03CBDDB
:10D9D800224B1B6813F0050F00F03685204BDE61E3
:10D9E80000F032BD1D4B1B68980740F12D851C4B7C
:10D9F800DE6100F029BD194B1B68990700F02485EA
:10DA0800174BDE6100F020BD144B1B68DA0640F1AD
:10DA18001B85134BDE6100F017BD104B1B689B067E
:10DA280040F112850E4BDE6100F00EBD0B4B1B68FA
:10DA38005F0640F109850A4BDE6100F005BD074B22
:10DA48001B681D0640F10085054BDE6100F0FCBC3B
:10DA5800C8530020D0540020DF540020D0530020A9
:10DA68001C470020AA4B1B68DC0540F1ED84A94B3C
:10DA7800DE6100F0E9BC1A6A072A00F2E584511C4D
:10DA88001962D96903EB82025162DE6100F0DCBCE5
:10DA98001B6AA04A002B00F0D784013B136202EBFB
:10DAA80083035B6AD36100F0CFBC7B782E2B04D84C
:10DAB800994A0121D15400F0C7BCFF2B7FF41FAE57
:10DAC800944B012283F8442000F0BEBC7B782E2BB7
:10DAD80004D8914A0021D15400F0B6BCFF2B7FF442
:10DAE8000EAE8C4B002283F8442000F0ADBC894C6C
:10DAF80094F8453083B9701C4FF00A0304D1874A63
:10DB080016687343A36401E05E43A664FAF7AAFBB0
:10DB18000123E06484F845306B78042B00F2948488
:10DB2800DFE803F0034372A51900FAF79BFBE26CE8
:10DB3800A16C801A80EAE072A2EBE0728A42754B0F
:10DB480004D9002283F8452000F07EBCDA69013A46
:10DB5800DA6100F079BCA87801F0B4FC40B96C4BEC
:10DB680084F845001A6822F010021A6000F06CBCB4
:10DB7800A36C684DA3B1FAF775FBEB6CAA6CC01ADD
:10DB880080EAE073A3EBE073934209D9002385F898
:10DB980045305F4B1A6842F010021A6000F054BC1E
:10DBA800E369013BE36100F04FBC0020FCF7CDFCCA
:10DBB800AB785B00184110F0010609D0002384F807
:10DBC8004530534B1A6822F010021A6000F03CBC32
:10DBD800A36C504D9BB1FAF745FBEB6CAA6CC01ACD
:10DBE80080EAE073A3EBE073934208D9484B85F8C9
:10DBF80045601A6842F010021A6000F025BCE3691B
:10DC0800013BE36100F020BC01AA00207C21FCF765
:10DC1800A1FCAA780223520003FA02F29DF806300A
:10DC280012EA030709D0002384F84530384B1A68F4
:10DC380022F010021A6000F007BCA16C354D91B1BA
:10DC4800FAF710FBE96CAE6C401A80EAE071A1EBC0
:10DC5800E071B14207D92E4B85F845701A6842F039
:10DC680010021A60F0E3E369013BE361ECE301AA07
:10DC780000207C21FCF76EFCAB789DF806205B0049
:10DC880042FA03F313F0010608D0002384F8453064
:10DC98001F4B1A6822F010021A60D5E3A26C1D4DC2
:10DCA80092B1FAF7DFFAEA6CA96C801A80EAE0729E
:10DCB800A2EBE0728A4207D9154B85F845601A68CD
:10DCC80042F010021A60BFE3E369013BE361BBE382
:10DCD800BA78022A28D85C001149E018104441F8A3
:10DCE80020601048807E002800F0AE83002B00F0F2
:10DCF800AB83581E0C2568432344134400F5C360C6
:10DD080000EB820001EB83010422FCF76CF99BE332
:10DD1800D05300201C470020744D0020D054002010
:10DD2800D453002004000020FF2A7EF4A3AEA54EA1
:10DD380083B90C25002405F20C6071192044214494
:10DD480004220434FCF74FF90C2CF4D10C35FC2DCB
:10DD5800F0D179E300246B780C205A1E504303EB72
:10DD68004303E11800F5C36000EB840006EB810172
:10DD780004220134FCF737F9032CECD164E37B78F7
:10DD8800142B3FF6BCAC904A9278022A19D803EBC0
:10DD980043031A448B498D4B51F822201B7862604B
:10DDA800002B00F051838A4B1A608A4B22B91A68FB
:10DDB80042F008021A6047E31A6822F008021A6063
:10DDC80042E3FF2A7EF456AE7E4E83B90C2500242A
:10DDD80005F20C6071192044214404220434FCF734
:10DDE8008DF90C2CF4D10C35FC2DF0D12CE300244A
:10DDF8006B780C205A1E504303EB4303E11800F5DF
:10DE0800C36000EB840006EB810104220134FCF7B7
:10DE180075F9032CECD117E37F78142F3FF66FAC1C
:10DE2800AE78DFF8A48131062DD50024AB782341E4
:10DE3800DA070FD56101644B41F00201002001F0BF
:10DE4800E2015E78FCF782FD06EB46065D4B264450
:10DE580043F82600604B9B7E8BB16B787BB15A1ED2
:10DE68000C20504303EB4303564A00F5C360E11806
:10DE780002EB810100EB84000422FCF7B4F80134C2
:10DE8800032CD3D1E0E2022E3EF6F4AD710141F04D
:10DE98000201002001F0E201FCF758FD4E4B494A0F
:10DEA80007EB47079B7E3E4442F82600002B00F014
:10DEB800CB8298F80130002B00F0C682591E0C2046
:10DEC800484398F8024003EB4303E11800F5C360A8
:10DED80002EB810100EB84000422FCF784F8B3E232
:10DEE8007A783B4B0A2A42D8DFE802F0060B111673
:10DEF8001C24292E33383C0038491A6809680A441A
:10DF080003E036491A680968521A1A602FE0334943
:10DF18001A6809684A43F8E730491A68096892FBA1
:10DF2800F1F2F2E72D4A1968126891FBF2F002FB50
:10DF38001012EAE7294A11681A680A40E5E7274AF1
:10DF480011681A680A43E0E7244A11681A684A40C7
:10DF5800DBE7224A1168C943116008E01A681F49C3
:10DF68000A6004E01D4A18681168106019601A6890
:10DF7800184B22B91A6842F008021A6064E21A685B
:10DF880022F008021A605FE2114B1B68C7F80330E1
:10DF9800FDF71EFC58E20E4B1B68C7F80330FEF76E
:10DFA8000BFA51E27B78052B00F24E82DFE803F092
:10DFB80003181E242A30074B1A6802F00F021A6051
:10DFC80042E200BFD4530020C8530020DF54002091
:10DFD800D0540020D053002004000020EC5400202E
:10DFE800A74B1A6822F010021A602DE2A44B1A6897
:10DFF80022F020021A6027E2A14B1A6822F04002A0
:10E008001A6021E29E4B1A6822F080021A601BE215
:10E018009B4B1A6822F480721A6015E27B782E2BCB
:10E028003FF66DAB974A02EB83031E650CE2954BF6
:10E038009549D3F80C210A60D3F8102193490A6056
:10E04800D3F814218E49DA61D3F818210A60D3F87D
:10E058001C218F4983F84520D3F82021DA64D3F8AE
:10E0680024219A6493F82821885C08B101208854F7
:10E07800002283F82C21E7E1BA78022A3EF6FAACAE
:10E088007B78142B3FF63BAB03EB43031A447E4BE0
:10E0980080491B6841F82230D6E100F049FFD3E1FE
:10E0A80000F048FFD0E100F046FFCDE100F044FF6A
:10E0B800CAE100F042FFC7E100F040FFC4E17B780D
:10E0C80013B1012B04D00BE06E4B01221A76BBE191
:10E0D800B6F5006FBEF4CEAC6A4A1376D661B3E1EA
:10E0E800032388F80030AFE1664B02221A76ABE1D1
:10E0F800644A4FF0FF3002F1500343F821006448AE
:10E108000023435401312F29F2D11376D3611362CE
:10E1180082F845305C4A13605C4A1360584A1360C1
:10E1280092E15D4B1B7D9B0709D4B6F5006FBEF4E9
:10E13800A1AC544B04221A76C3F8306184E1082359
:10E1480088F8003080E1554B01221A70524B544C2C
:10E158009A78B6F5006F227026D21B7D13F0010560
:10E1680022D1304601A9FBF717FE9DF8043025722D
:10E1780063709DF80530A3709DF80630E3709DF834
:10E188000A3023719DF8093063719DF80830A37136
:10E198009DF80730E3710123E15C227A01330A44D8
:10E1A800082B2272F8D14FE101230021E1540133F9
:10E1B800082B3B4AF9D11378137245E17B7883B970
:10E1C800364A012111703449354A89781170354928
:10E1D80008680133C11811F8011C082BD154F8D173
:10E1E80032E1012B40F030810C2288F8072088F8B2
:10E1F80005302622092388F8062088F8043023E110
:10E208007B78032B00F22081DFE803F0020E191D52
:10E218001C4B1A7EE27193F84520D3F83031A27175
:10E228001A0A627123710FE1164B1A7EE27193F894
:10E238004520DB69A2711A0A6271237104E1124B4D
:10E248001B68636000E1114B1B686360FCE07B782E
:10E25800002B40F0F980144B9978002940F0F480A5
:10E2680040F2D2439E4240F0EF8040F2FF70FBF74D
:10E2780057FEFBF7ADFD0120FAF794FDE4E000BF7F
:10E28800D05300201C470020D0540020EC5400201C
:10E29800744D0020D453002004000020D4540020E2
:10E2A800D554002000000020C85300207A78684B1D
:10E2B80002B101221A70EA78664B1A70664B93F81D
:10E2C8003411664B1970664900230B7065490B7051
:10E2D800654B19780A431A70B6E05F4B012283F840
:10E2E8003521B1E07D7815B1012D11D01DE0042252
:10E2F80040F2FB7001A9FBF701FF019BD7F803204F
:10E308009A4206BF0123C8F80430C8F804509BE0BD
:10E31800BB782A2B06D140F2FB7054490422FBF744
:10E3280062FE91E0032323708EE0032388F8003017
:10E338008AE07B78032B3CD8DFE803F008022D380D
:10E34800454A0023D2F83811144610E0424BD3F85E
:10E358003821092A07D8511CC3F8381103EB820366
:10E36800C3F83C6170E0092323706DE001338B42F0
:10E378006AD03F4A9D0052F82300B042F6D12A44A1
:10E38800481E834204D25068013342F8040BF7E771
:10E39800C4F8380158E0304A0023C2F83831344A0A
:10E3A800002199500433282BF9D14DE00A236360EA
:10E3B8004AE00323237047E07B78812B44D1BA7865
:10E3C8002C4B922A40D19A79A32A3DD15A79B42A62
:10E3D8003AD11A79C52A37D1DB78D62B34D1264BD6
:10E3E8001C221A83FDF7EEF9F9F73CFF0446F9F70A
:10E3F80039FF001B0028B8BF4042B0F57A7FF6DB32
:10E4080072B6FAF7DDFC1D4B00241C6021461C483F
:10E4180002F0B5FD1A4802F0F1FC01F099FF02F094
:10E4280085FE4FF0804003F009FC2046FAF7BAFC5D
:10E438000AE040F2D2439E4206D1074B012283F8FC
:10E44800642101E00223237005B0BDE8F08300BF1A
:10E45800F04B0020234C00201C4700205C4D00207E
:10E46800224C0020A34D0020F14B0020CB5300206C
:10E4780058480020C85300200010024010E000E077
:10E48800106402404649F8B500230B604549464AE6
:10E498000B604649D36113620B6082F8453082F8FD
:10E4A800443082F82C311646414A4FF0FF3142F889
:10E4B8002310404A0024D45401332F2BF4D1650192
:10E4C800EDB245F006010020FCF740FA3A4B45F062
:10E4D8000C0143F824000020FCF738FA374B43F8C6
:10E4E80024000134032CEAD10024354DE0B205EBB9
:10E4F8004413D97A0134C1F10801C9B2FCF72CFDE3
:10E50800032CF2D1287BFAF7C1FC95F82C00FAF716
:10E51800BDFC95F84C00FAF7B9FC0023294A002104
:10E5280099500433B3F5806FF8D1274FBB7E83B180
:10E538000C250024254905F20C6029442044214477
:10E5480004220434FBF7DAFD0C2CF3D10C35FC2D36
:10E55800EFD1FB7E2BB13B7903F0EF02012A0DD1FD
:10E568000EE04FF4A7641A492046214404220434DB
:10E57800FBF7C4FDB4F5C36FF5D1ECE7212B01D14E
:10E58800012300E0002386F865317B7D23B1FAF78B
:10E5980059F808B1012300E000233376F8BD00BF25
:10E5A800D0540020EC5400201C470020D0530020F9
:10E5B8006C470020744D0020FC580020F0540020C7
:10E5C800A84C0020FC54002004000020D453002054
:10E5D800C44F0020F7B50F4E0F4CC6F803300F4B51
:10E5E80086460F46B270002294E803001A708DE840
:10E5F800030086F800E07770FEF71EF9217863685B
:10E60800074A82F866119DE8030084E8030018466B
:10E6180003B0F0BDC8530020E4540020DF540020AC
:10E628001C470020014B93F8660170471C470020E7
:10E63800F7B51F4E024653780C4696E803008DE85E
:10E6480003001C4900270B7093786D464B70D378F4
:10E658008B7013798B7153794B7193790B71D379D3
:10E66800CB70154B1F70FEF7E7F8144B197833463B
:10E6780071B9217032786170A2707278E270F279A3
:10E688002271B27962717279A2713279E27109E00C
:10E69800012907D13A460A4911444978A15401325F
:10E6A800082AF8D195E8030083E8030003B0F0BD19
:10E6B800E4540020C8530020DF540020D454002024
:10E6C800D55400202DE9F04FAF4B95B01B78AF4CD7
:10E6D80013B994F8673163B1AD4B1B78062B08D09A
:10E6E8000A2B06D003F0EF030F2B1CBF002384F87E
:10E6F800343194F83431A54A591E0129A54E3BD826
:10E70800A549012BCA6814BF082307238DF83030A8
:10E7180094F868310D9232788DF8313000238DF8F5
:10E728003230C2B98B688DF83F208DF838309B4B5A
:10E7380019788DF8391059788DF83A10D9798DF8FB
:10E748003B1099798DF83C1059791B798DF83D105B
:10E758008DF83E3009E0012A07D1914901330CAA0E
:10E76800595C1A44082BD171F7D10CA8FAF7F4FFB9
:10E77800002800F0A783ACE0032B2AD192F865515A
:10E788001DBB33788BB9844F844DB87897F80180D6
:10E798002A78804490446A789044EA799044AA7927
:10E7A80090446A7990442A7920E0012B40F09180C6
:10E7B8007B4B585D0135FAF70DFD092DF8D188E03E
:10E7C800072B63D192F8653173B3744801F0FEFCEE
:10E7D8007FE0042BF4D1704F704DB87897F8018022
:10E7E800002301226B702A706B6080449044FAF712
:10E7F800F1FC7878FAF7EEFC2878FAF7EBFC687801
:10E80800FAF7E8FCE879FAF7E5FCA879FAF7E2FC08
:10E818006879FAF7DFFC5FFA88F82879FAF7DAFC02
:10E828004046FAF7D7FC54E032782ABB5A4B93F8A3
:10E8380002E093F801C0594B8DF818E01F785D7815
:10E84800E644D8798DF81A70774499798DF81B5079
:10E858003D445A798DF81C0028441B798DF81D1009
:10E8680001448DF81E200A448DF81F3013448DF89A
:10E8780019C08DF8203028E0012A26D1484A06A977
:10E888009A5CCA540133092BF8D11EE0082B20D119
:10E89800424A002301205370107053603E4A8DF89D
:10E8A8001A00917852788DF818108DF819200A44BA
:10E8B80002448DF81B308DF81C308DF81D308DF812
:10E8C8001E308DF81F308DF8202006A80921FCF78E
:10E8D80027FF344B1A789846002A00F08D80324B77
:10E8E800324D1B78013B062B00F28280DFE803F0F3
:10E8F8000404258080806000274A297893688DF871
:10E908004E108DF8483080238DF849308A238DF8D1
:10E918004A3000238DF84B308DF84C308DF84D304F
:10E928008DF841308DF84230D368072110A88DF852
:10E9380040101193FAF710FF5AE0174F2A78B87869
:10E9480097F80190814409F10A099144FAF742FCC9
:10E958007878FAF73FFC8020FAF73CFC8A20FAF72F
:10E9680039FC0020FAF736FC0020FAF733FC0020C7
:10E97800FAF730FC5FFA89F92878FAF72BFC484651
:10E98800FAF728FC34E000BFDE5400201C470020C2
:10E99800C8530020D454002004000020E454002070
:10E9A800D5540020A34D00205C4D0020224C0020AF
:10E9B800B54B2A789878597880238DF8251001442A
:10E9C8000A318DF826308A238DF824008DF82730F7
:10E9D8008DF82B2000230A4409A809218DF8283036
:10E9E8008DF829308DF82A308DF82C20FCF798FE08
:10E9F80000232B7088F80030002384F834313370FA
:10EA080084F8673194F8643113B10120FAF7CAF930
:10EA180094F835219D4B52B193F86521D2F101024A
:10EA280038BF002283F86521002283F835210CA81D
:10EA3800FAF7E0FE00283FD09DF83030062B3BD98E
:10EA4800934B9DF838201A709DF839205A709DF81C
:10EA58003A209A709DF83B209A719DF83C205A7193
:10EA68009DF83D201A719DF83E20DA709DF83130EE
:10EA780084F86831844B1A690D9B934203D1834B08
:10EA8800012283F86721F9F7EDFB824B0022186019
:10EA9800814B1A709DF83030227E072B0CBF012362
:10EAA800022384F83431531E012B7C4B02D9052AEA
:10EAB80040F0C9800022E4E094F86551002D70D13F
:10EAC80009A8FAF7A1FB00286BD0FAF7BBFB10B135
:10EAD8006E4B83F8695194F869119DF824004A1C1B
:10EAE800D2B22144092A694B84F8692181F86A0164
:10EAF80040F0DC80002283F86921634A93F86A3188
:10EB08005178994207D092F82710002900F0CE805A
:10EB18008B4240F0CB8092F827209A4204BF012311
:10EB280084F8673100231A46584D05F5B571595CCC
:10EB380001330A44082BD2B2F6D195F872319342C8
:10EB48002BD1534B95F86B211A7095F86C215A709C
:10EB580095F86D219A7095F86E219A7195F86F2144
:10EB68005A7195F870211A7195F87121DA70F9F7D0
:10EB780079FB4B4B4B4A1860297E00231370032204
:10EB880085F834214A1E012A85F86931434A02D999
:10EB9800052918BF0123137088E0042385F8343150
:10EBA80084E094F86531394D7BB1394801F0C1F9F9
:10EBB80058B1F9F757FB3A4B3A4A186000231370DB
:10EBC800032285F834212A7E36E094F86561002E08
:10EBD80040D110AD2846FCF7CDFD00283AD0334689
:10EBE8003246E95C01330A44082BD2B2F9D19DF8C8
:10EBF800481091422BD1264B9DF841201A709DF860
:10EC080042205A709DF843209A709DF844209A71CA
:10EC18009DF845205A719DF846201A719DF84720A5
:10EC2800DA70F9F71FFB1E4B1E4A18600023137099
:10EC3800072284F83421227E511E01291946174BD8
:10EC480003D9052A01D001221BE019702EE084F8AF
:10EC580034312BE0237E0D4D013B012B26D8EB6987
:10EC6800B3F5006F20D2F9F7EDFCE8B1E86908497F
:10EC7800431CEB61FBF790F8092385F83431074B07
:10EC880001221A7012E000BF040000201C47002077
:10EC9800C85300204C4D0020E04B0020DF540020DA
:10ECA800544D00205B4D002000232376237E874DA2
:10ECB800042B04D1864E3278130640F1D98094F89B
:10ECC800343113F0FB0F05D0082B03D0062B01D0ED
:10ECD800FDF7B2FD94F83431092B0BD07B4B93F838
:10ECE8003401092840F0AA801A7E022A04BF0522AE
:10ECF8001A76A3E0F9F7B6FA744A764DD2682B680B
:10ED0800801A80EAE072A2EBE0729A4208D9724B4C
:10ED18001A78012A04BF02221A70F9F7A3FAE060F0
:10ED2800F9F7A0FA23696A68C01A80EAE073A3EBCE
:10ED3800E073934208D9684B5A78012A04BF02222B
:10ED48005A70F9F78FFA2061F9F78CFA6369AA68A3
:10ED5800C01A80EAE073A3EBE073934208D95E4BD4
:10ED68009A78012A04BF02229A70F9F77BFA606147
:10ED780094F84420554B002AB0D093F82C21002A4F
:10ED8800ACD15649DC6C0968049401915449D3F814
:10ED98001C410968D3F80C9102915249D3F81081AB
:10EDA8000968D8690391996CD3F814C10591D3F80F
:10EDB800187193F845100094D3F82061D3F82451C2
:10EDC80093F828411346DFF810A11AF803B0BBF1F5
:10EDD800020F18D1DFF814B15BF823B0BBF1FF3F85
:10EDE8000DD000918446DCB2059D049E039F5846D1
:10EDF800DDF80880DDF804900122002103E04FF0DF
:10EE0800000B0AF803B001332F2BDCD12F4B83F80A
:10EE180045100099C3F80C91C3F81081D861C3F864
:10EE280014C1C3F81871C3F81C11C3F82061C3F8E2
:10EE3800245183F8284183F82C214FE7D3F838214F
:10EE48002249002A3ED009283CD10B7E012B39D11A
:10EE5800C86900231D4901F59E7454F82340A04257
:10EE680002D105230B762DE001339342F2D129E03C
:10EE780095F8343113F0FB0F24D0082B22D0062B41
:10EE880020D0D5F83001184CD6F80330B0F5006F13
:10EE98006270636012D23146FBF77CF8D5F8300116
:10EEA8003146FAF7E5FF30B1D5F830310133C5F80E
:10EEB8003031652300E00723237003E00723237024
:10EEC80000232B7615B0BDE8F08F00BF1C4700204B
:10EED800C8530020144D0020744D0020D054002049
:10EEE800EC540020D0530020E45400206C4700204C
:10EEF800704710B5F9F7B6F9074C2368C01AB0F592
:10EF0800FA7F07D9054B5A6982F040025A61F9F72E
:10EF1800A9F9206010BD00BF085900200010024068
:10EF280008B5F9F70BFF014B586008BDE454002001
:10EF3800704770477047704770477047704700BF09
:10EF48002DE9F04F470187B0FDB2044645F07C013A
:10EF580005AA0020FBF7FEFAB74B9DF81610DA1940
:10EF68006300029392F808B0029E02231BF0400F40
:10EF7800506803FA06F30CD003EA01020123B340F8
:10EF880001EA0309AC4BC0F10008D9594942039181
:10EF980008E00122B24003EA0109A74B0A40DB5905
:10EFA80080460393022C94BF601CA01CC0B201923F
:10EFB800F9F791FAA0490BF03F0B394491F9081081
:10EFC80082460029019A04DAD0F1010A38BF4FF0CD
:10EFD800000A0BF1FF31072900F25D82DFE811F02A
:10EFE80008000800080008001401140114011401A5
:10EFF800924E315D0F2900F24E82DFE811F04C028B
:10F0080010004C013C007901480051005D0070007F
:10F018009F00D100D6004C02F000F900360245F0FE
:10F02800140105AA0020FBF795FA45F006059DF89E
:10F03800153006EB8406294600207360FBF7A1FA19
:10F048002146306102220020FBF7B3FA002029464E
:10F0580040F2FF72FBF7D7F9002021460322FBF7A5
:10F06800CAFAABF1020BBBF1010F744F94BF022334
:10F0780004233B550FE2002A00F00D82002045F0E2
:10F088000201FBF763FC6E4B43F8240025E1B9F15C
:10F09800000F00F000822046FBF7A4FB0623F9E1ED
:10F0A800214600200322FBF7A6FA002045F00801BC
:10F0B8004246FBF7A8F948E1B9F1000F40F0EB81AF
:10F0C80045F00805484629464A46FBF79CF9484654
:10F0D8002946C8F10002FBF796F90823DAE1B9F1ED
:10F0E800000F00F0D88145F002010020FBF72EFC4C
:10F0F80081460020024645F00801FBF784F9504B91
:10F10800002053F824202146C9EB020243F82420AA
:10F118000322FBF770FA002045F006014246FBF790
:10F1280072F9002007F0E0014A46FBF77EF900205B
:10F1380021460246FBF73DFA0923ABE10020FBF725
:10F1480004FA029A1041C10740F1A581002045F058
:10F15800080902464946FBF756F9002021460222D3
:10F16800FBF727FA0020024645F00201FBF75DF99C
:10F178000020024607F0E001FBF757F9ABF1030B5B
:10F1880020460021F9F7A6FABBF1010F00F27881B9
:10F19800002021460222FBF70CFA0020494606E12E
:10F1A800B9F1000F40F0148175E1B9F1000F40F09A
:10F1B800728145F002014846FBF7C8FB45F008019B
:10F1C80080464A464846FBF71EF90222484607F0A1
:10F1D800E00198FBF2F2FBF728F948461AE1002013
:10F1E800FBF7B3F9029B1841C20740F1548147E18C
:10F1F80006EB8407002045F006013A69FBF703F99E
:10F20800002021463A7942E10C4E315D0F2900F287
:10F218004281DFE811F0400117003D005A006A0002
:10F22800880040019C0040014001D200DF00B50089
:10F23800050137012A0100BFA84C00209048002092
:10F24800E44B002045F0140105AA0020FBF782F9E1
:10F258009DF8152006EB84035A60002021460222FF
:10F26800FBF7A7F9002045F0060140F2FF72FBF713
:10F27800CAF8002021460322FBF7BDF9BBF1060FAF
:10F288005BD0BBF1080F58D0844B04221A5502E119
:10F29800BBF1060F09D106EB84035A68002002F07F
:10F2A8000402214642F0010205E0BBF1080F04D137
:10F2B800002021460322FBF79EF9002045F00801B3
:10F2C800039AFBF7A0F80323E4E0ABF10503012B55
:10F2D80005D822B1BBF1060F31D10423DAE0BAF127
:10F2E800000F00F0D8800C23D4E0BBF1050F09D142
:10F2F80006EB84035A68002002F00402214642F01B
:10F30800020205E0BBF1070F04D1002021460322C9
:10F31800FBF771F9039B00205A4245F00801FBF7FF
:10F3280072F80523B6E0ABF10502012A09D8B9F154
:10F33800000F06D0BBF1050F01D10223AAE00F236D
:10F34800A8E0BAF1000F00F0A6800723A2E0BAF106
:10F35800000F40F0A080ABF1070BBBF1010F0AD9F9
:10F3680006EB84035A68504602F00402214642F034
:10F378000102FBF740F9002045F00801424618E079
:10F38800BAF1000F40F08780ABF1070BBBF1010F1A
:10F398000AD906EB84035A68504602F00402214653
:10F3A80042F00202FBF727F9002045F00801C8F1F6
:10F3B8000002FBF728F80A236CE0BAF1000F6AD0C4
:10F3C800002045F00201FBF7C1FA06EB8403D8617F
:10F3D8000B235FE0BAF1000F5DD145F00201504602
:10F3E800FBF7B4FA2E4B81463B4483F80DA05046F8
:10F3F80045F006014246FBF718F806EB8403DB6983
:10F4080002229944504607F0E00199FBF2F2FBF71B
:10F418000CF8504621460246FBF7CBF80D2339E09D
:10F428000020FBF792F8029A1041C30733D5002059
:10F438000E2345F0080102463355FAF7E4FF21464A
:10F4480000200222FBF7B5F8002045F00201024631
:10F45800FAF7EBFF002007F0E0010246FAF7E5FFB4
:10F4680020460021F9F736F915E00020214602224E
:10F47800FBF79FF8002045F008010246FAF7C3FFA2
:10F488000E2307E006EB84031A7900202146FBF7D8
:10F49800B2F80023335507B0BDE8F08F904800203C
:10F4A800A84C0020024B1A5C0AB901221A54704772
:10F4B80090480020024B1A5C0AB10F221A54704778
:10F4C80090480020014B185C704700BF904800200E
:10F4D80010B50024064B0022E254064BE0B203EBC1
:10F4E8004413997A0134F8F799FF032CF2D110BD2F
:10F4F8005D4D0020A84C00202DE9F04F964C85B0BA
:10F50800237833B96FF000436360A360E36001239D
:10F518002370257C914F4DB9E8B2F8F7DCFF785598
:10F528000135082DF8D18C4B01221A7427250026A5
:10F53800F0B2F8F7D0FFBB5D83421AD0874BB21DFB
:10F54800F054874B53F82230022B05D0032B0AD0F6
:10F55800012B0ED168B106E058B9824A515D0129E4
:10F5680007D1535505E07F4B5A5D012A04BF02229B
:10F578005A550136082E05F10105D9D17A4EF3699D
:10F58800C3B17A4D2F78AFB9F8F76CFE784B1B688A
:10F59800C01AF3690028B8BF404298420AD93846D1
:10F5A800FBF720F90120FBF71DF90220FBF71AF9F8
:10F5B80001232B70336AD3B16E4D2E78BEB9F8F79C
:10F5C80051FE6D4B684A1B68126AC01A80EAE073E4
:10F5D800A3EBE07393420AD93046FBF703F9012005
:10F5E800FBF700F90220FBF7FDF801232B70607E82
:10F5F800624D594F05EB4012167B002E00F0F78044
:10F608005F4A604E0244604B00920021821903EB6E
:10F61800800301920A46FBF7BFFE787E4301EA1891
:10F62800127B013A042A00F2D980DFE802F0033D98
:10F63800B13DB100F9F710FC544EA0B1607E23181B
:10F648009B7E022B03D1335C002B00F0C78005EBB7
:10F658004015697AF8F7E2FE607EFBF70DFF637EDE
:10F668000221E2181CE0607E23189B7E012B03D147
:10F67800335C002B00F0B28005EB4013997AF8F761
:10F68800CDFE607E05EB4015AB7A13B9FBF7E6FEBD
:10F6980003E0335C0BB1FBF7EFFE637E0121E21858
:10F6A80091760022F25499E03256384E002A19DB3E
:10F6B8002218927E022A01D1325C62B12B44597A17
:10F6C800F8F7ACFE607EFBF7D7FE637E0221E218F6
:10F6D80091760022F254667EF8F7C4FD04EB8603A7
:10F6E800586032E02044837E1B4F012B03D1637E98
:10F6F800F35C93B929E0F8F7B5FD7B7E0A2107EBA7
:10F70800830705EB43139B8B7A684B43801A80EA87
:10F71800E072A2EBE0729A42E9DD607E05EB4013ED
:10F72800997AF8F77BFE607E05EB40139B7A13B954
:10F73800FBF794FE03E0335C0BB1FBF79DFE637EA1
:10F748000121E21891760022F254607E05EB401503
:10F758002B7B042B35E000BFB8480020C9480020A7
:10F76800144D0020744D0020040000205B4D002043
:10F77800544D0020E04B00204C4D0020A84C0020A8
:10F78800004C0020A34C0020244C0020584D0020A1
:10F798002218927EA84E022A01D1325C62B12B4413
:10F7A800597AF8F73BFE607EFBF766FE637E02211E
:10F7B800E21891760022F254607E05EB40152B7B0F
:10F7C800052B0BD1F9F748FB9C4B5B7E18B118460B
:10F7D800FBF752FE02E01846FBF740FE627E974BAD
:10F7E8000132D2B2022A88BF00225A761DE3F8F706
:10F7F80039FD3B6AC01A80EAE073A3EBE0730A2B79
:10F8080040F31383797E3046490141F00A0101F043
:10F81800EA01FAF7B6FE0646787EFBF721F9787E0C
:10F828000C2242438649874F8B18D3F804808A58A4
:10F838001B7A002B18BF90463B5C032B00F2AE806E
:10F84800DFE803F0025C153B002E00F0A78005EB13
:10F858004013D97F21B1F8F7E1FD637E032204E06C
:10F86800597AF8F7DBFD637E0222FA5496E04EB926
:10F87800400140F0080101F0E8013046FAF781FE46
:10F88800002845D086EAE672A2EBE672B8F1000FCE
:10F89800B8BFC8F100084245607E01D0002E6DD186
:10F8A800694B53F830108A4272D203EBC0031979BE
:10F8B800F8F7B4FD614B5B7E17E086EAE672A2EBCF
:10F8C800E672B8F1000FB8BFC8F10008424501D090
:10F8D800002E5DD15C4B53F830108A4207D203EBFF
:10F8E800C0031979F8F79AFD637E01224FE005EB12
:10F8F8004013597AF8F792FD637E3DE01EBB400144
:10F9080040F0080101F0E8013046FAF73AFED0B9B4
:10F91800F8F7A8FC637E4FF00A0E04EB83025268E6
:10F92800801A05EB4312918B0028B8BF40420EFBAA
:10F9380001F1884232DD1846917AF8F76FFD3F4BA6
:10F948005B7EFE542AE086EAE673A3EBE673B8F121
:10F95800000FB8BFC8F100084345607E00D06EB9FB
:10F96800394A52F83020934212D305EB4013597AA2
:10F97800F8F754FD314B5B7E022208E005EB40139B
:10F98800D97F29B1F8F74AFD2C4B03225B7EFA5444
:10F99800677EF8F767FC04EB87077860607E2B4B7F
:10F9A8000021034400932A4B0A4603440193294B40
:10F9B800DFF8888003EB8003FBF7EEFC607E264FC0
:10F9C80005EB40139B69002B4CD0F8F74FFE00283D
:10F9D80048D098F8190086EAE672A2EBE67207EBBF
:10F9E80040139B699A423DD9FAF7FCFE98F8193002
:10F9F8001A4A012107EB4317D154BB7F43B9637EF1
:10FA0800174A0F33D15C01292CD10221D15429E0A6
:10FA18000027627E05EB471305EB4212927F9B7F1E
:10FA28009A4205D13846FAF7DDFEF8B2FFF742FDF3
:10FA38000137032FEDD1E2E7584D0020B8480020E8
:10FA4800584C00205D4D0020044C0020004C002044
:10FA5800A34C0020244C0020A84C0020A04C0020DF
:10FA6800744D00200020FAF770FD94F82420C10797
:10FA780002F0F802B74B48BF42F0010247078DF881
:10FA8800080083F8242005D594F8243043F00203B5
:10FA980084F82430C10605D594F8243043F00403D3
:10FAA80084F82430DFF8C082DFF8C0C2DFF8C0E293
:10FAB800DFF8A8B2A84B94F8249098F800109CF8A6
:10FAC80000209EF800009BF8007093F800A0002327
:10FAD80041FA03FB1BF0010F16D049FA03FB1BF098
:10FAE800010F11D042FA03FB1BF0010F0CD10127C3
:10FAF80007FA03FBBAF1000F5FFA8BFB4BEA000031
:10FB08004BEA020208BF00210133032BE0D1934BDB
:10FB18008CF800201F7094F8243088F80010DA0759
:10FB28008EF800000AD58B4A92F82520D70705D40D
:10FB38008B4AD178012904BF0221D170980709D5D1
:10FB480094F82520910705D4854A1179012904BF25
:10FB5800022111715A0709D594F82520570705D4B1
:10FB68007F4A5179012904BF02215171627E84F8CC
:10FB780025300323B2FBF3F304A90B4413F9083C23
:10FB8800002B43DA520142F01601002001F0F60181
:10FB980003AAFAF7DFFC9DF80E30580609D56D4A1E
:10FBA8006F49527E52001B32885C012804BF022034
:10FBB8008854190609D5617E694A0E3112F8110078
:10FBC800012804BF022002F81100DA0608D5627E77
:10FBD800634952001B32885C012804BF0220885404
:10FBE8009B0609D5627E5E4B0E3213F8121001296E
:10FBF80004BF022103F81210617E0020490141F080
:10FC0800160101F0F60103AAFAF7D8FB627EDFF8C5
:10FC1800448151016B185B69DFF858A1002B00F093
:10FC28008A80504B9F5C9946002F40F08480002EBC
:10FC380000F0828041F0020101F0E2013846FAF753
:10FC480085FE834698F81900F8F728FD98F81910EA
:10FC5800C0EB0B000AEB41135B6980EAE07BABEB7E
:10FC6800E07B83EAE372A2EBE372934540F384807E
:10FC7800002B25DD0846FAF7B5FD98F819300AEB90
:10FC880043139B7F63B9607E354A00F11503D15C4D
:10FC980001294AD10221D15447E00137032FF2D07C
:10FCA800627E05EB471305EB4212927F9B7F9A42D7
:10FCB800F3D13846FAF796FDF8B2FFF7FBFBECE70D
:10FCC80038460222FAF775FC98F8191038464901A7
:10FCD80041F0080101F0E801FAF720FC98F8193022
:10FCE8000AEB43139B7F002BCDD0627E05EB4713B5
:10FCF80005EB4212927F9B7F9A4212D15FFA87F8F6
:10FD0800002041460222FAF754FC4FEA481141F01C
:10FD18000801002001F0E801FAF700FC4046FFF76F
:10FD2800C9FB0137032FE0D1ADE7012309F8003003
:10FD3800FFF7C0FB20E0FEB941F00801002001F008
:10FD4800E801FAF71EFCB8B9637E05EB4312D289C5
:10FD5800F2B120E0B8480020F04B0020A34D00206D
:10FD6800744D00201F4C0020234C0020F14B002034
:10FD7800224C0020A84C0020677E2D4BDB5D002B19
:10FD8800E2D1F8F76FFA2B4B03EB8707B8621EE056
:10FD9800274AD35CDBB1F8F765FA637E04EB83028C
:10FDA800926A05EB4315801AE98980EAE072A2EBB2
:10FDB800E0720A2041438A4209DD1F4DEA5C32B9EC
:10FDC8001846FBF74BFB1B4B01225B7EEA54607E17
:10FDD8001A4D002EB8BF764255F83030154F9E4266
:10FDE8000AD2FBF701FA7B7E05EBC3056A798242EA
:10FDF8000DD11846002108E0FBF7F6F97B7E05EBEC
:10FE0800C3056979884202D01846FBF7C1F9607EBC
:10FE1800FFF796F8637E074D0133DBB2022B88BFEC
:10FE280000236B76F8F71EFA206205B0BDE8F08F64
:10FE3800604D0020B8480020634D0020044C00208D
:10FE4800074B10B518681C4601460A780B46013165
:10FE58001AB12C2AF9D100221A700133236010BD7F
:10FE6800EC48002070B50646F9F7CEF90D4C05466A
:10FE780018B100232371012070BDA368E268934282
:10FE880007D25A1C23441B7C012033702071A260C6
:10FE980070BD04F11000FBF75BFCA560E06028462C
:10FEA80070BD00BFEC48002010B50D4C0246237908
:10FEB8001BB9BDE81040F9F78DB9206D0D2A00F186
:10FEC80001032044236580F8542002D03F2B00D83A
:10FED80029B919460348FBF723FC0023236510BD05
:10FEE800EC4800204049002070B50121044686B046
:10FEF8002020FFF7D9FF002C04DA2D200121FFF77D
:10FF0800D3FF644200230A2194FBF1F201FB124162
:10FF180001AE30311D46995514460133002AF2D1FD
:10FF2800705D0121FFF7C0FF15F1FF35F8D206B06B
:10FF380070BD2DE9F34105460DF10700FFF792FF6B
:10FF4800974C002800F0C88094F894309DF807007A
:10FF5800944E03BB7378403398420DD1D4F898304F
:10FF6800002B40F0B9803179012331F0010184F888
:10FF7800943040F0B180ADE00D2801D01B2801D1AC
:10FF8800002305E0D4F898307E2B00F2A5800133D9
:10FF9800C4F89830A0E0317931F0010101D1FFF7C0
:10FFA80083FF9DF807301F2B0CD9D4F898207C4983
:10FFB8007E2A00F28280501C0A44C1F8980082F818
:10FFC8009C307AE0082B08D1D4F89830002B74D0F4
:10FFD800734A013BC2F898306FE00D2B6DD1D4F80D
:10FFE8009830002B69D03379112B16D16D4B012134
:08FFF800587800274030C0B228
:020000040801F1
:10000000FFF756FFD4F898309F4206D2684B012183
:10001000D85DFFF74DFF0137F4E70D200121FFF711
:1000200047FF0023D4F898802768C4F81C311A468B
:100030001946424537D0012911D002D3022925D0D3
:100040002FE0DFF864C10CF19C00105C202828D060
:100050000CEB030181F820010133012121E052481A
:1000600000F19C0C12F80CC0BCF1200F0AD1012B3E
:1000700004D91844002180F8201101334D4F02218A
:100080001F440EE0184480F820C109E0DFF818C1D1
:100090000CF19C00105C202803D09C448CF82001BB
:1000A00001330132C5E70022C4F81C31234483F830
:1000B00020210123276084F89F3184F89420C4F81C
:1000C00098209DF807301B2B0AD133790021012B92
:1000D000C4F8981084F8941002D10D20FFF7E8FEC0
:1000E00094F89F01002600285AD02F4B83F89F6177
:1000F000F7B2DFF8DC80C7EBC70708EB07042D4831
:10010000214605F0FBFC28B9A6796379F1072B702D
:1001100036D506E018F807300136002BE8D12B70F1
:100120003DE0FFF791FE2B780446042B14D12249C1
:1001300005F0E4FC08B900230CE020461F4905F057
:10014000DDFC08B9012305E01D49204605F0D6FC79
:1001500090B902236B7013E00D2B0ED1194905F0F5
:10016000CDFC0028E7D02046174905F0C7FC002841
:10017000E8D020461549E9E7204605F0BBFC687049
:10018000B20704D5FFF760FE05F0B4FCA870730752
:1001900005D5FFF759FE05F0ADFCC5F803000120B9
:1001A00002B0BDE8F08100BFEC4800200400002050
:1001B000884900200C4A0020316401083564010898
:1001C000396401083F640108456401084A64010874
:1001D000F762010838B50D4D0446A878012140307A
:1001E000C0B2FFF765FE687801214030C0B2FFF76A
:1001F0005FFE2078FFF77CFE6068FFF779FEBDE8C0
:1002000038400D200121FFF753BE00BF040000203D
:100210007047FEE7FEE7FEE7FEE77047704770476E
:10022000704700002F4B82B01A6842F001021A603A
:1002300000229A60196821F0847121F480311960DC
:1002400029495960196821F480211960DA60009207
:1002500001921A6842F480321A60224B1A6802F442
:1002600000320192009A01320092019A1AB9009A62
:10027000B2F5A06FF1D11B6813F4003318BF01234E
:100280000193019B012B04D0184B194A9A6002B0CC
:100290007047144B9A689A609A6842F400429A60D8
:1002A0009A6842F4A0529A60124A5A601A6842F060
:1002B00080721A6019680B4A8901FBD50E4B40F217
:1002C00003711960936823F003039360936843F00C
:1002D00002039360034B9B6803F00C03082BF9D1D6
:1002E000D2E700BF003802401030002400ED00E0EB
:1002F00000800008081E4005003C0240134A10B56B
:100300009068134B00F00C000428124913D0082801
:1003100011D154685068526800F03F00C2F388124F
:10032000B1FBF0F15143094A5268C2F30142013274
:100330005200B1FBF2F1054A19609268C2F3031250
:100340001A4411791A68CA401A6010BD0038024078
:10035000BC0000200024F40008B54FF48070012197
:1003600001F0E4F9BDE808404FF48070002101F08D
:10037000DDB943680A6823F0407323F480731343A4
:100380000A7910B543EA02234360CA680B6984689E
:100390001A438B681A43084B234013434A7943EAB4
:1003A000420383600B7DC26A013B22F47002DBB220
:1003B00042EA0353C36210BDFDF7FFC00023036090
:1003C000037143718360C360036101230375704748
:1003D000074A084B516810B50B4090E812000C43D7
:1003E0008168C068214301430B43536010BD00BFC7
:1003F00000230140E030FCFF002303604360836082
:10040000C3607047836811B143F0010301E023F03A
:10041000010383607047436823F4400323F40073AF
:10042000194341607047416282627047436823F01C
:100430001F03194341607047044B5A6810B142F4DE
:10044000000201E022F400025A60704700230140DC
:10045000044B5A6810B142F4800201E022F4800299
:100460005A60704700230140092970B50DD9A1F1E8
:100470000A0404EB44040725A540A340C66826EA05
:10048000050545EA0304C4600BE001EB41040725C0
:10049000A54003FA04F4066926EA050545EA0403C3
:1004A0000361062A0CD8013A02EB82021F23934013
:1004B00001FA02F2446B24EA03031A43426370BD5B
:1004C0000C2A0CD8073A02EB82021F23934001FA50
:1004D00002F2046B24EA03031A43026370BD0D3A6F
:1004E00002EB82021F23934001FA02F2C46A24EA5B
:1004F00003031A43C26270BD836843F08043836084
:1005000070478068C0F380507047836811B143F42E
:10051000806301E023F4806383607047836811B1D6
:1005200043F0020301E023F0020383607047436855
:10053000013923F4604343EA413343607047436821
:1005400011B143F4006301E023F40063436070479A
:10055000C06C80B27047014B186870470823014097
:10056000836811B143F4807301E023F480738360E6
:100570007047836811B143F4007301E023F4007302
:1005800083607047044B5A6810B142F4005201E096
:1005900022F400525A60704700230140092970B5C7
:1005A0000DD9A1F10A0404EB44040725A540A3409A
:1005B000C66826EA050545EA0304C4600BE001EBC2
:1005C00041040725A54003FA04F4066926EA050557
:1005D00045EA04030361846B931CC4F301555B1B60
:1005E000DBB203EB83031F229A40994024EA020402
:1005F00044EA0103836370BD836B013923F4401324
:1006000043EA01538363704782B000230193019052
:10061000019B19440191019B1A6002B070478368E5
:1006200023F47023194381607047836823F44013D7
:10063000194381607047836843F480038360704787
:100640008068C0F380507047436811B143F4806301
:1006500001E023F4806343607047436811B143F4C1
:10066000805301E023F480534360704782B000233D
:1006700001930190019B283319440191019B186853
:1006800080B202B070470123C9B203FA01F1436896
:100690000AB1194301E023EA010141607047036890
:1006A00019420CBF002001207047C9430160704708
:1006B0004368006810EA112007D0C9B2012202FA8B
:1006C00001F119420CBF0020012070476FEA11218F
:1006D0000160704708B50B4B984207D14FF000708E
:1006E000012101F017F84FF0007006E04FF0806034
:1006F000012101F00FF84FF080600021BDE80840B3
:1007000001F008B800640040036823F002030360AE
:10071000036843F0010303604FF480334268D2075B
:1007200001D4013BFAD1436813F0010355D08B7912
:10073000012B03680CBF43F0800323F080030360A8
:10074000CB79012B03680CBF43F0400323F0400337
:1007500003600B7A012B03680CBF43F0200323F0E6
:10076000200303604B7A012B03680CBF43F0100396
:1007700023F0100303608B7A012B03680CBF43F056
:10078000080323F008030360CB7A012B03680CBF36
:1007900043F0040323F0040303608B78CA789B07BB
:1007A00043EA02630A7943EA02434A7943EA02537D
:1007B0000A88013A1343C361036823F0010303600D
:1007C0004FF480334268D20701D5013BFAD140682B
:1007D00000F0010080F00100704718467047837AEE
:1007E00001219940344B70B5D3F80022CC4342F03C
:1007F0000102C3F80022D3F81C222240C3F81C22B5
:10080000027BA2B9D3F80C22C6882240C3F80C227E
:10081000827A4588483245EA064543F832500388D3
:100820008288857A43EA0242244BED005A51037BC9
:10083000012B15D1204B0688D3F80C2245880A439A
:10084000C3F80C22827A45EA0645483243F8325012
:10085000C3888288857A43EA0242184BED005A51D8
:10086000C37A154A1BB9D2F80432234002E0D2F809
:1008700004320B430589C2F804320F4B2DB9D2F86C
:1008800014522C40C2F8144206E0012D04D1D3F8D2
:1008900014220A43C3F81422427B012A04D1D3F85C
:1008A0001C221143C3F81C12D3F8002222F00102CB
:1008B000C3F8002270BD00BF0064004044660040E1
:1008C00000238371C371037243728372C372837096
:1008D000C370032303710223437101230380704714
:1008E0000D4BD3F8002242F00102C3F80022D3F8E6
:1008F000002222F47C5222F00E02C3F80022D3F828
:10090000002242EA0020C3F80002D3F8002222F0BD
:100910000102C3F80022704700640040036811B16F
:1009200043F4803301E023F48033036070470368AD
:1009300099B143F080030360D0F8843143F48073AD
:10094000C0F88431D0F8943143F48073C0F8943106
:10095000D0F8A43143F4807312E023F080030360E5
:10096000D0F8843123F48073C0F88431D0F8943106
:1009700023F48073C0F89431D0F8A43123F4807349
:10098000C0F8A43170478368F0B55C01024607D413
:100990008368180106D49368DB0005D40420F0BDF9
:1009A000002002E0012000E0022005015319D3F8E5
:1009B000804104F00104C3F880410C7A4E7A44B9B6
:1009C0000C68D3F8807146EA44543C43C3F8804134
:1009D00009E04F68D3F880C144EAC70444EA0C0434
:1009E0002643C3F880618C7A2A4404F00F048C7289
:1009F000D3F8844124F00F04C3F884418E7AD3F8ED
:100A000084413443C3F884414E7B8C7B360446EAF0
:100A10000466CC7A26430C7B46EA0426C2F8886139
:100A200002F5C4744A7C8D7C120442EA0562CD7BD7
:100A3000097C2A4342EA01226260D3F8802142F015
:100A40000102C3F88021F0BD012908D004D3022996
:100A500016D182680C4B04E082680C4B01E082687E
:100A60000B4B1340094A934208D001D853B907E011
:100A7000074A934202D0044A934203D101207047AF
:100A8000022070470020704700000310030000049C
:100A900000030008012907D002D3022908D07047BB
:100AA000836843F0800306E0836843F4004302E078
:100AB000836843F400038360704730B50C01031969
:100AC000D3F8B05105F00405EDB2157225B9D3F88D
:100AD000B0516D0D156003E0D3F8B051ED085560CD
:100AE000D3F8B05105F002055572D3F8B45105F0B2
:100AF0000F059572D3F8B4311B0AD3740319D3F8D8
:100B0000B85103F5DC74D572D3F8B8512D0A1573BA
:100B1000D3F8B8512D0C5573D3F8B8311B0E93731D
:100B20006368D37363681B0A137463681B0C537484
:100B300063681B0E937421B9C36843F02003C3603C
:100B400030BD036943F02003036130BD21B9C368A0
:100B500043F02003C3607047036943F0200303613F
:100B6000704709B9C06802E0012903D1006900F0AB
:100B7000030070470020704799B9036823F003030E
:100B800043F0010303604FF48033426802F0030234
:100B9000012A01D0013BF8D1406800F00300012890
:100BA00028E0012911D1036823F0030303604FF407
:100BB00080334268920701D0013BFAD1436813F0B9
:100BC000030F14BF002001207047022916D10368CB
:100BD00023F0030343F0020303604FF480334268C1
:100BE00002F00302022A01D0013BF8D1406800F074
:100BF0000300022814BF0020012070470020704726
:100C0000036823F0030343F002030360406800F02D
:100C10000300831E584258417047036823F00203C3
:100C200003604FF480334268920701D5013BFAD14B
:100C3000406880F00200C0F340007047806900F017
:100C4000700070478069000E70478069C0F30740EC
:100C5000704743690AB1194301E023EA0101416188
:100C6000704711F4700F01D083690BE0CB0101D5FF
:100C7000436807E00A0101D5836803E08B014CBF9C
:100C8000C3680369C3F313030B420CBF00200120A8
:100C900070470A4B994202D10023836170478A0151
:100CA000C1F3130301D5C36070474A0101D5036145
:100CB00070470A014CBF8360436070477000F0309A
:100CC00043690B405CD0402942D010D8042933D06E
:100CD00005D8012927D0022954D1C0682FE0102956
:100CE0002CD0202930D008294CD1C06835E0B1F58E
:100CF000006F3BD00CD8B1F5007F31D0B1F5806FDB
:100D000032D0B1F5807F3DD1806900F0010070479D
:100D1000B1F5803F1ED0B1F5003F1DD0B1F5004FB9
:100D200030D1406829E0806800F0013020F0807008
:100D3000003018BF01207047C06806E0006910F05D
:100D4000030018BF012070470069C0F3C00070475E
:100D5000006902E04068F8E74068C0F3001070479F
:100D60008069C0F340007047806906E0836913F032
:100D7000700F0CBF002001207047C0F38000704747
:100D80001846704700207047B1F5807F35D00CD8E9
:100D9000082924D004D801291CD004291DD070476B
:100DA00020291FD040291FD07047B1F5006F22D0F5
:100DB00006D8B1F5007F20D0B1F5806F1DD0704707
:100DC000B1F5803F13D0B1F5003F12D0B1F5004F1F
:100DD00015D110E00A4B83607047082300E0102310
:100DE000C3607047082300E01023036170470823A5
:100DF00004E0102302E00023836104234360704772
:100E000001010100036823F0010303600023036074
:100E100043608360C360036121234361294B98428F
:100E200017D0294B98421BD0284B984220D0284BF2
:100E3000984225D0274B98422AD0274B98422ED053
:100E4000264B984232D0264B984236D0254B9842BA
:100E500003D13D2243F8082C7047234B984204D11C
:100E60004FF4746243F8202C7047204B984204D111
:100E70004FF4741243F8382C70471D4B984204D13C
:100E80004FF0746243F8502C70471A4B984203D1CC
:100E9000194A43F8642C7047184B984203D1184AFA
:100EA00043F87C2C7047174B984203D1164A43F8FD
:100EB000942C7047154B984203D14FF03D5243F8A4
:100EC000AC2C704710600240286002404060024035
:100ED000586002407060024088600240A06002409A
:100EE000B86002401064024028640240406402403E
:100EF00058640240706402403D0000208864024053
:100F0000400F0020A064024000003D20B864024071
:100F10000268134B10B51340CC680A6814434A6941
:100F200014438A691443CA6914430A6A14434A6A17
:100F300014438A6A14434A6B14438A6B2243134353
:100F4000036044690A6BCB6A24F00704134323430C
:100F500043610B6943604B6883608B68C36010BD5D
:100F60003F801CF00023036043608360C360036123
:100F700043618361C361036243628362C36203634B
:100F8000436383637047036811B143F0010301E0D9
:100F900023F0010303607047036811B143F4004379
:100FA00001E023F4004303607047036811B143F08C
:100FB000200301E023F02003036070474160704785
:100FC000406880B27047036812B143F4002301E027
:100FD00023F40023036001617047036811B143F4F7
:100FE000802301E023F48023036070470AB101618C
:100FF0007047C16070470068C0F3C0407047006828
:1010000000F001007047406900F0380070470A4B5B
:1010100010B50A4A0A4CA0428CBF104618468B00F5
:101020004CBF4368036821F0F02121F0821119427E
:101030000CBF0020012010BD00600240006402408F
:101040000F64024010B5084B084A094CA0428CBFFF
:101050001046184611F0005F21F0F02121F08211B6
:1010600014BFC160816010BD006002400064024096
:101070000F6402400B0611D543694AB143F0800367
:101080008029436114D0036801F01E0119430EE06A
:1010900023F080038029436104D17047802907D061
:1010A000002AF0D1036801F01E0123EA010101606A
:1010B000704730B5104B114A114D21F0F024A84271
:1010C0008CBF15461D4624F0C3132BB1026802F0F5
:1010D0001E0202EAD12202E0426902F080028B0085
:1010E0004CBF6B682B6824F08210184002D0101C93
:1010F00018BF012030BD00BF006002400064024004
:101100000F64024010B5084B084A094CA0428CBF3E
:101110001046184611F0005F21F0F02121F08211F5
:1011200014BFC160816010BD0060024000640240D5
:101130000F640240044B00221A605A609A60DA6021
:10114000024A5A61704700BF003C0140FFFF7F0028
:10115000837930B50168027943B3194BCC431D68DC
:1011600002F1804225401D605D6802F59E322C40F0
:101170005C6014682143116002689C68D1430C4094
:101180009C60DC682140D9604179102906D19968BA
:1011900011439960D9680A43DA6030BD01F1804398
:1011A00003F59E3319680A431A6030BD02F180438B
:1011B00003F59E331A6822EA0101196030BD00BFB1
:1011C000003C014000230C220360037142718371D3
:1011D0007047024B1A69104318617047003C014088
:1011E000034B5B6918420CBF00200120704700BF11
:1011F000003C0140014B5861704700BF003C01407A
:10120000054B1A685B69034004D010420CBF0020F4
:101210000120704718467047003C0140014B58615F
:10122000704700BF003C014008B52C4B984205D1E7
:101230000120014600F04AFA012048E0284B98427C
:1012400005D10220012100F041FA02203FE0254BA8
:10125000984205D10420012100F038FA042036E03C
:10126000214B984205D10820012100F02FFA0820D7
:101270002DE01E4B984205D11020012100F026FAE6
:10128000102024E01A4B984205D12020012100F0C3
:101290001DFA20201BE0174B984205D14020012168
:1012A00000F014FA402012E0134B984205D1802040
:1012B000012100F00BFA802009E0104B98420BD17D
:1012C0004FF48070012100F001FA4FF4807000218A
:1012D000BDE8084000F0FAB908BD00BF00000240B8
:1012E0000004024000080240000C024000100240CE
:1012F0000014024000180240001C0240002002407E
:101300002DE9F0410F68002301229A4002EA070507
:10131000954230D15A00032494400668E4432640A5
:1013200006600E79D0F800C006FA02F8013E48EADD
:101330000C0C012EC0F800C014D891F805C08668C6
:101340000CFA02FC2640866086684CEA0606866037
:10135000466826EA050545608D7946689D40ADB230
:1013600035434560C5682C40CD79C46005FA02F26A
:10137000C4682243C2600133102BC5D1BDE8F0819F
:101380004FF6FF7303600023037143718371C371D0
:10139000704782B04FF480330193019B0B4301935C
:1013A000019BC361C161019BC361C3690193C369AF
:1013B000019302B07047036919420CBF002001205D
:1013C0007047006980B27047436919420CBF002022
:1013D00001207047406980B27047018370474183A4
:1013E00070470AB10183704741837047416170477C
:1013F000436959404161704701F00703C90800EB98
:1014000081009B000F2199409A4010B5046A24EA9C
:1014100001010162016A1143016210BD0A4B002102
:101420001A6842F001021A6099601A6822F0847208
:1014300022F480321A60054A5A601A6822F4802227
:101440001A60D960704700BF003802401030002495
:10145000024B00221A701870704700BF0238024019
:10146000034B1A6822F0F80242EAC0001860704785
:1014700000380240014B1860704700BF000047422F
:10148000064B002201281A701A7002D0042802D0DC
:1014900070471870704705221A7070477038024004
:1014A000014B1860704700BF800E474210B5029C88
:1014B0005B0840EA04600143013B41EA821242EAD0
:1014C0000344014B5C6010BD00380240014B1860C2
:1014D000704700BF600047420907034B41EA801094
:1014E000C3F88400704700BF00380240014B186009
:1014F000704700BF68004742014B1860704700BF4B
:101500004C004742034B9A6822F0EC6211430843B7
:101510009860704700380240034B9A6822F0784286
:10152000114308439860704700380240034B9A68A3
:1015300022F0030210439860704700BF0038024059
:10154000024B986800F00C00704700BF0038024062
:10155000034B9A6822F0F00210439860704700BF76
:1015600000380240034B9A6822F4E052104398601E
:10157000704700BF00380240034B9A6822F4604273
:1015800042EAC0009860704700380240194B10B51D
:101590009968194A01F00C01042913D0082911D1C6
:1015A0005C6859685B6801F03F01C3F38813B2FBC4
:1015B000F1F25A430F4B5B68C3F3014301335B0005
:1015C000B2FBF3F20B4902608B680C4AC3F30313BE
:1015D000D45C0368E34043608C68C4F38224145DE8
:1015E00023FA04F484608968C1F34231525CD34029
:1015F000C36010BD003802400024F400D000002079
:1016000000F44073B3F5407F084B08D1996820F08F
:10161000704221F4F81122F440720A439A601A6F62
:10162000C0F30B0010431867704700BF003802403A
:10163000014B1860704700BF3C0E4742014B1860D9
:10164000704700BF400E4742014B1860704700BF13
:101650005C014742044B1A6B09B1104301E022EAD6
:1016600000001863704700BF00380240044B5A6BFB
:1016700009B1104301E022EA00005863704700BF3F
:1016800000380240044B9A6B09B1104301E022EA92
:1016900000009863704700BF00380240044B1A6C8A
:1016A00009B1104301E022EA00001864704700BF4E
:1016B00000380240044B5A6C09B1104301E022EAA1
:1016C00000005864704700BF00380240044B1A699C
:1016D00009B1104301E022EA00001861704700BF21
:1016E00000380240044B5A6909B1104301E022EA74
:1016F00000005861704700BF00380240044B9A69EF
:1017000009B1104301E022EA00009861704700BF70
:1017100000380240044B1A6A09B1104301E022EA82
:1017200000001862704700BF00380240044B5A6A3C
:1017300009B1104301E022EA00005862704700BF7F
:1017400000380240044B1A6D09B1104301E022EA4F
:1017500000001865704700BF00380240044B5A6D06
:1017600009B1104301E022EA00005865704700BF4C
:1017700000380240044B9A6D09B1104301E022EA9F
:1017800000009865704700BF00380240044B1A6E95
:1017900009B1104301E022EA00001866704700BF5B
:1017A00000380240044B5A6E09B1104301E022EAAE
:1017B00000005866704700BF00380240044B1A789A
:1017C00009B1104301E022EA00001870704700BF21
:1017D0000D3802404309012B074A01D1136803E089
:1017E000022B0CBF136F536F00F01F0023FA00F0A1
:1017F00000F00100704700BF0038024007B5002329
:1018000001933120FFF7E6FF019B01330193019B18
:10181000B3F5A06F01D00028F3D03120FFF7DAFF35
:10182000003018BF012003B05DF804FB024B5A6F73
:1018300042F080725A67704700380240034BDB6801
:1018400018420CBF00200120704700BF0038024042
:10185000014B1870704700BF0E38024008B5154B99
:1018600098420BD14FF480500121FFF75FFFBDE894
:1018700008404FF480500021FFF758BF0E4B9842AC
:1018800007D14FF480400121FFF744FF4FF480401F
:1018900009E00A4B98420BD14FF400400121FFF7B9
:1018A00039FF4FF400400021BDE80840FFF732BF88
:1018B00008BD00BF0030014000380040003C00403F
:1018C0000B8810B54C88028823438C8802F441525F
:1018D0002343CC8823430C8923434C8923438C899D
:1018E0002343CC89234313439BB20380838B23F48C
:1018F00000631B041B0C83830B8A038210BD838B44
:10190000F0B523F47B6323F00F031B041B0C8383CC
:10191000022303848B68858B022BADB238D08A8872
:10192000002A294A14BF022601269468240203D5FE
:10193000946824F400049460D2F88440D2F884704F
:101940005268DFF888C002F03F02BCFBF2F2C4F339
:1019500088145443C7F30272B4FBF2F4CA88B2F598
:10196000007F18BF76014FF00A020CBF240AB4FBB7
:10197000F6F46243B2FBF3F305330A229BB2B3FBE6
:10198000F2F303F001021202C3F34F0392B200E03C
:1019900000229C1EA4B2FE2C28BF0022CC8828BFA7
:1019A0000223134323430A889BB2038445EA0203BC
:1019B0004A8843F4006313438A8813438A89134394
:1019C0009BB28383F0BD00BF003802400024F400C6
:1019D0000023038043808380C3800381438183810C
:1019E000C3810723038270470023022203804380C0
:1019F0008380C380826083817047038819B19BB262
:101A000043F0400303E023F040031B041B0C03805E
:101A10007047838B19B19BB243F4806303E023F4D6
:101A200080631B041B0C83837047038823F40063CB
:101A30001B041B0C038003889BB219430180704771
:101A4000B1F5804F038803D19BB243F4804303E098
:101A500023F480431B041B0C038070474FF6FF6385
:101A60009942038803D09BB243F4807303E023F4CC
:101A700080731B041B0C03807047838819B19BB2D1
:101A800043F0040303E023F004031B041B0C8380D6
:101A90007047838819B19BB243F0100303E023F031
:101AA00010031B041B0C83807047808980B2704731
:101AB00081817047038819B19BB243F4005303E05E
:101AC00023F400531B041B0C0380704703889BB254
:101AD00043F4805303807047012914BF008B808A30
:101AE00080B27047008A80B2704783889BB20AB187
:101AF000194301E023EA01018180704709090123AC
:101B00008B409BB21AB1828892B2134303E0828861
:101B100092B222EA030383807047038919420CBF03
:101B2000002001207047C94389B20181704701F04C
:101B30000F02012303FA02F210B584880089A4B2CF
:101B400080B2104005D009098B401C420CBF002018
:101B5000012010BD01F00F0101238B40DB439BB23C
:101B60000381704708B54FF480400121FFF7DEFD87
:101B7000BDE808404FF480400021FFF7D7BD014B7E
:101B8000186070470038014001F003039B000F22EA
:101B90009A40984001F0FC0101F1804101F59C312F
:101BA00010B58C6824EA02028A608A6802438A605F
:101BB00010BD014B18607047DC002742014B1860D4
:101BC000704700BF00042742024B186AC0F3002090
:101BD000704700BF0038014030B5048C24F0010488
:101BE0002404240C0484058B048CADB225F0F30589
:101BF000A4B22A4324F00A0442EA031344F0010485
:101C00009DB221430583018430BD30B5048C24F09E
:101C100010042404240C0484058B048C25F44075E2
:101C2000A4B22D052D0D24F0A00444F0100445EAC3
:101C3000022242EA033344EA01119BB28CB20383CD
:101C4000048430BD08B5474B984205D101200146B8
:101C5000FFF76CFD01203DE0B0F1804F05D1012080
:101C60000146FFF757FD012076E03F4B984205D132
:101C700002200121FFF74EFD02206DE03B4B984210
:101C800005D104200121FFF745FD042064E0384B15
:101C9000984205D108200121FFF73CFD08205BE0B8
:101CA000344B984205D110200121FFF733FD10205D
:101CB00052E0314B984205D120200121FFF72AFD47
:101CC000202049E02D4B984209D102200121FFF745
:101CD0002DFD02200021BDE80840FFF727BD284B5D
:101CE000984207D14FF480300121FFF71FFD4FF4D8
:101CF0008030EFE7234B984207D14FF400300121A9
:101D0000FFF714FD4FF40030E4E71F4B984207D172
:101D10004FF480200121FFF709FD4FF48020D9E71F
:101D20001A4B984205D140200121FFF7F3FC4020D7
:101D300012E0174B984205D180200121FFF7EAFC01
:101D4000802009E0134B98420BD14FF480700121A1
:101D5000FFF7E0FC4FF480700021BDE80840FFF77A
:101D6000D9BC08BD0000014000040040000800404C
:101D7000000C00400010004000140040000401402E
:101D8000004001400044014000480140001800406C
:101D9000001C0040002000401C4A038890429BB277
:101DA00012D002F5806290420ED0B0F1804F0BD07D
:101DB000A2F58032904207D002F58062904203D0B3
:101DC00002F58062904203D14A8823F070031343E6
:101DD0000F4A904208D002F58062904204D023F46A
:101DE00040730A899BB2134303804B68C3620B881C
:101DF0000385064B984203D003F58063984201D1D6
:101E00008B7A038601238382704700BF0000014064
:101E1000001000404FF0FF33436000230380038134
:101E2000438083727047018582827047038823F064
:101E300070031B041B0C19430180704741627047FB
:101E4000C1627047406A7047008D80B27047038856
:101E500019B19BB243F0020303E023F002031B0419
:101E60001B0C03807047038819B19BB243F0040335
:101E700003E023F004031B041B0C0380704703885A
:101E800019B19BB243F0800303E023F080031B04ED
:101E90001B0C03807047038823F008031B041B0CF2
:101EA000038003889BB2194301807047038823F4A1
:101EB00040731B041B0C038003889BB219430180F1
:101EC0007047038819B19BB243F0010303E023F08C
:101ED00001031B041B0C03807047038C70B523F0B7
:101EE00001031B041B0C0384038C8488028B0D8864
:101EF00022F073021204120C2A434E888D8923F0BB
:101F000002031B043543ADB21B0C2B430E4DA4B290
:101F1000A84203D005F58065A8420ED1CD8923F0F3
:101F200008032B438D8823F004032B434E8A0D8A2C
:101F300024F440743543ADB22C43848002838A6814
:101F40004263038470BD00BF00000140038C30B5C4
:101F500023F010031B041B0C0384038C8288048B66
:101F60000D8824F4E6442404240C23F0200344EADE
:101F700005241B048D891B0C43EA05134D8892B27E
:101F800043EA0513124DA4B2A8429BB203D005F553
:101F90008065A84215D1CD8923F080039BB243EA26
:101FA00005134FF6BF751D408B8822F4406245EA49
:101FB00003130D8A9BB242EA85024D8A42EA8502EA
:101FC00092B282808A6804838263038430BD00BF3A
:101FD00000000140038C30B523F480731B041B0CFC
:101FE0000384038C8288848B0D8824F0730424047A
:101FF000240C23F400732C431B048D891B0C43EA2F
:1020000005234D8892B243EA0523124D9BB2A842A4
:1020100003D005F58065A84215D1CD8923F400636E
:102020009BB243EA05234FF6FF351D408B8822F40F
:10203000405245EA03230D8A9BB242EA05124D8ABB
:1020400042EA051292B282808A688483C263038462
:1020500030BD00BF00000140038C30B523F4805335
:102060001B041B0C0384038C8488828B0D8822F450
:10207000E6421204120C23F4005342EA05221B0428
:102080008D891B0C43EA05334D88A4B243EA05331E
:102090000A4D92B2A8429BB203D005F58065A842D2
:1020A00005D10D8A24F4804444EA8514A4B28480C6
:1020B00082838A680264038430BD00BF000001404F
:1020C000002303804380838083608381C3810382F4
:1020D0004382704730B501248C40058C00F1180311
:1020E000ADB225EA0404048421F0080038B9490897
:1020F0005C584FF68F702040585058580AE0043909
:10210000C1F34E01CC5848F6FF702040C85012026F
:10211000C85892B20243CA5030BD416370478163D0
:102120007047C163704701647047038B23F07003ED
:102130001B041B0C194301837047038B23F4E043FA
:102140001B041B0C43EA01218BB203837047838B72
:1021500023F070031B041B0C194381837047838B8E
:1021600023F4E0431B041B0C43EA01218BB283835D
:102170007047038B23F008031B041B0C19430183D6
:102180007047038B23F400631B041B0C43EA0121FB
:102190008BB203837047838B23F008031B041B0C53
:1021A000194381837047838B23F400631B041B0C4A
:1021B00043EA01218BB283837047038B23F004032E
:1021C0001B041B0C194301837047038B23F48063AA
:1021D0001B041B0C43EA01218BB203837047838BE2
:1021E00023F004031B041B0C194381837047838B6A
:1021F00023F480631B041B0C43EA01218BB283830D
:102200007047038B23F080031B041B0C19430183CD
:102210007047038BC3F30E0343EA01218BB20383A0
:102220007047838B23F080031B041B0C19438183AD
:102230007047838BC3F30E0343EA01218BB2838380
:102240007047038C23F002031B041B0C1943018409
:102250007047038C23F008031B041B0C19430184F3
:102260007047038C23F020031B041B0C43EA01116D
:102270008BB203847047038C23F080031B041B0C78
:1022800043EA01118BB203847047038C23F400737B
:102290001B041B0C43EA01218BB203847047038C9F
:1022A00023F400631B041B0C43EA01218BB203845B
:1022B0007047038C23F400531B041B0C43EA0131C9
:1022C0008BB20384704701238B408A4010B5048C85
:1022D000A4B224EA03030384038C13439BB2038454
:1022E00010BD04238B408A4010B5048CA4B224EAAC
:1022F00003030384038C13439BB2038410BD0023A8
:102300000122038043808280C38003817047406B39
:102310007047806B7047C06B7047006C7047038BD1
:1023200023F00C031B041B0C0383038B9BB2194388
:1023300001837047038B23F440631B041B0C03834E
:10234000038B9BB243EA01218BB203837047F8B53C
:102350000C464988A2880029B4F800E014BF002781
:102360000227012A054614BF012602262389BEF151
:10237000000F11D1FFF730FC2846E188FFF7CFFFAF
:102380002846394632462389FFF73FFC2846E18834
:10239000BDE8F840FFF7CEBFFFF737FC2846E188DD
:1023A000FFF7C8FF2846394632462389FFF714FC59
:1023B0002846E188BDE8F840FFF7B1BF838B23F0E2
:1023C0000C031B041B0C8383838B9BB219438183F7
:1023D0007047838B23F440631B041B0C8383838B24
:1023E0009BB243EA01218BB283837047F8B50E8814
:1023F0000D4604464988AA882B893EB9FFF7ECFBB5
:102400002046E988BDE8F840FFF789BF042E07D1D0
:10241000FFF7FBFB2046E988BDE8F840FFF78ABFDD
:10242000082EB5F806C0078C1CD127F480773F042E
:102430003F0C0784868B058CB6B2ADB226F0F3064E
:1024400025F4206546EA031345EA01219BB289B2CF
:102450001A4341F480718283BDE8F84001846146EB
:10246000FFF7ACBF27F480573F043F0C0784868BEF
:10247000058C26F4407625F4005536056D046D0C68
:10248000360D46EA022645EA013146EA033389B2AF
:102490009BB241F4805183830184BDE8F8406146DA
:1024A000FFF797BF4A880B8813438A881343CA886B
:1024B00013430A8913434A8913438A8913439BB2FE
:1024C000A0F8443070470023038043808380C3809A
:1024D0000381438183817047B0F8443029B16FEAAA
:1024E00043436FEA53439BB201E0C3F30E03A0F8EA
:1024F00044307047838819B19BB243F0040303E072
:1025000023F004031B041B0C83807047838819B1DC
:102510009BB243F0010303E023F001031B041B0CF7
:102520008380704783899BB20AB1194301E023EA93
:1025300001018181704781827047038A19420CBF73
:10254000002001207047C94389B201827047038A85
:10255000828911EA030092B203D011420CBF00201D
:1025600001207047C94389B2018270470A43A0F82D
:102570004820704783899BB20AB1194301E023EADE
:10258000010181817047838819B19BB243F0080330
:1025900003E023F008031B041B0C838070470389AE
:1025A00023F007031B041B0C03817047038923F0EE
:1025B00070031B041B0C1943018103899BB243F078
:1025C00007030381704738B50D46602D1146044658
:1025D0004FF0010202D1FFF718FB01E0FFF7FCFA10
:1025E000238923F070031B041B0C2B4323812389B5
:1025F0009BB243F00703238138BD038923F07003A6
:102600001B041B0C194301817047838823F070035E
:102610001B041B0C838083889BB219438180704705
:10262000038923F007031B041B0C038103899BB25E
:10263000194301817047038923F080031B041B0C9D
:10264000038103899BB219430181704710B5048946
:10265000E4B221430A4342EA03239CB2048110BD41
:1026600010B50446FFF7F2FF238923F077031B041C
:102670001B0C43F07703238110BD10B50446FFF710
:10268000E5FF23899BB243F48043238110BD70B5DD
:102690000589048B068C24F44074B6B224F003043C
:1026A00026F0220625F00705240432432D04240CCD
:1026B0002D0C44F4807442EA0313294344F00104CE
:1026C0009EB201810483068470BD838819B19BB2D8
:1026D00043F0800303E023F080031B041B0C838082
:1026E0007047A0F85010704708B5234B984205D1A9
:1026F00010200121FFF71AF8102037E01F4B9842F5
:1027000007D14FF400300121FFF704F84FF40030F7
:1027100009E01B4B98420BD14FF480200121FEF7BA
:10272000F9FF4FF480200021BDE80840FEF7F2BF1A
:10273000144B984207D14FF400200121FEF7EAFF25
:102740004FF40020EFE7104B984207D14FF4801070
:102750000121FEF7DFFF4FF48010E4E70B4B9842B6
:1027600009D120200121FEF7E1FF20200021BDE852
:102770000840FEF7DBBF08BD0010014000440040E8
:1027800000480040004C0040005000400014014050
:10279000038ACA889BB223F4405330B513430D46D5
:1027A00003820989AB8882890B43698992B20B4302
:1027B00022F4B05222F00C029BB213438381838A2D
:1027C000AA899BB223F44073134385B083820446E5
:1027D0006846FEF7DBFE194B9C4203D003F580638D
:1027E0009C4201D1039B00E0029BA289192112B2F5
:1027F0005943002A2A684FF06403B4BF5200920084
:10280000B1FBF2F1B1FBF3F21201100903FB10115D
:10281000A08900B2002806DAC9003231B1FBF3F317
:1028200003F0070305E009013231B1FBF3F303F0D4
:102830000F031A4392B2228105B030BD001001404F
:102840004FF4165303600C2200238380C38003815E
:102850004281838170470B8810B54C88028A2343DC
:102860008C88C988234392B20B4322F470629BB2D6
:102870001343038210BD0023038043808380C38001
:102880007047838919B19BB243F4005303E023F4EA
:1028900000531B041B0C83817047038B03F47F439D
:1028A0000383038B9BB2194301837047838929B14A
:1028B0006FEA43436FEA53439BB201E0C3F30E0355
:1028C00083817047838A19B19BB243F4006303E0AC
:1028D00023F400631B041B0C83827047C1F30801BF
:1028E000818070478088C0F308007047038A23F016
:1028F0000F031B041B0C0382038A9BB21943018242
:102900007047838919B19BB243F0020303E023F0BF
:1029100002031B041B0C83817047838923F400632B
:102920001B041B0C838183899BB2194381817047EF
:10293000038A23F020031B041B0C0382038A9BB22F
:10294000194301827047038A19B19BB243F4804353
:1029500003E023F480431B041B0C0382704783892C
:102960009BB243F0010383817047838A19B19BB204
:1029700043F0080303E023F008031B041B0C8382CD
:102980007047038BDBB20383038B9BB243EA0121C5
:1029900001837047838A19B19BB243F0200303E09F
:1029A00023F020031B041B0C83827047838A19B118
:1029B0009BB243F0100303E023F010031B041B0C35
:1029C00083827047838A23F004031B041B0C8382D9
:1029D000838A9BB2194381827047838A19B19BB263
:1029E00043F0020303E023F002031B041B0C838269
:1029F0007047838A9BB20AB1194301E023EA0101BF
:102A000081827047C1F3421310B5012401F01F0108
:102A1000A34204FA01F101D10C3003E0022B0CBFF8
:102A20001030143003680AB1194301E023EA0101B0
:102A3000016010BD038819420CBF002001207047BF
:102A4000C94389B20180704710B5C1F3421401F047
:102A50001F030122012C02FA03F201D1838903E052
:102A6000022C0CBF038A838A9BB21340028892B265
:102A700043B10123090A03FA01F111420CBF0020FE
:102A8000012010BD184610BD090A01238B40DB430D
:102A90009BB20380704700BF40F0BF60024B40F420
:102AA0000030D860704700BF00ED00E0C27810B57C
:102AB00003780AB3164A4478D26803F16043D243DC
:102AC000C2F30222C2F10401C9B204FA01F10F24D7
:102AD00044FA02F28478C9B222400A431201D2B207
:102AE00003F5614383F8002303780122590903F0B9
:102AF0001F0302FA03F306E05909012203F01F0342
:102B000002FA03F32031034A42F8213010BD00BF1E
:102B100000ED00E000E100E021F0604121F07F01E4
:102B2000014B08439860704700ED00E0044B1A69C0
:102B300009B1104301E022EA00001861704700BFAC
:102B400000ED00E0044B04281A680CBF42F00402B8
:102B500022F004021A60704710E000E010B5D0F8CF
:102B6000E83504461B699847032384F81231002096
:102B700010BD08B590F8123180F81331042380F8A5
:102B80001231D0F8E835DB689847002008BD08B559
:102B9000D0F8E435DB6903B19847002008BD08B5DB
:102BA000D0F8E4351B6A9847002008BD08B5D0F876
:102BB000E4355B6A9847002008BD10B5D0F8E835C9
:102BC00004465B699847012384F81531002010BD45
:102BD000D0F8E83510B59B6904469847D4F8E43539
:102BE00020465B6800219847002084F8150110BD3D
:102BF000002110B50B460446402201F053F9802114
:102C000040222046002301F04DF9012384F81231BF
:102C1000D4F8E835A0785B689847002010BD13B55C
:102C20006946044600F078FA9DF8001001F01F0391
:102C3000012B0CD006D3022B0ED12046694600F0A2
:102C4000DFFB0EE02046694600F096FA09E02046D8
:102C5000694600F0BDFB04E0204601F0800101F070
:102C60008EF9002002B010BD70B50446002947D18E
:102C700090F81131022B37D1D0F83821D0F8243117
:102C80009A4211D9C178D21A0129C0F8382104D149
:102C9000D0F828110B44C0F828312046D4F8281168
:102CA00092B200F0F2F91FE0D0F83C51B5FBF3F618
:102CB00003FB16565EB99D4209D3D0F840319D42C0
:102CC00005D2324600F0E1F9C4F840610CE0D4F8D6
:102CD000E435DB682BB194F81221032A01D1204698
:102CE0009847204600F003FA94F81631012B10D1D2
:102CF000094A236912685A60002384F8163108E0F3
:102D0000D0F8E4355B6923B190F81221032A00D191
:102D10009847002070BD00BF0C59002010B5044634
:102D200059BB90F81131032B30D1D0F89023D0F853
:102D30007C339A4214D9C178D21A0129C0F8902361
:102D400004D1D0F880131944C0F880139A4228BFE8
:102D50001A462046D4F8801392B200F0B0F915E07C
:102D6000D0F8E4351B6923B190F81221032A00D171
:102D70009847204600F0ACF908E0D0F8E4359B69AC
:102D800023B190F81221032A00D19847002010BDEA
:102D90002DE9F041069F0446164698460D46F8F781
:102DA0003DFC20462946C4F8E485C4F8E875C4F81B
:102DB000EC6501F02BF8D4F8E8351B6898472046FD
:102DC000BDE8F041F8F77CBC00207047D0F8E4354E
:102DD00010B51B6804469847D4F8E8359B689847B7
:102DE000002010BD08B5D0F8E4355B689847002096
:102DF00008BD00BF10B5074C2068FF2807D0064B60
:102E0000064A9B68064912689847FF232360002002
:102E100010BD00BF10010020A80000208C4A002037
:102E20009359002043230B80004870471401002071
:102E30001D4B70B55A681946052A02F1010401D0EC
:102E40005C602EE00A7A0023012A4B6029D0CA6810
:102E5000B2F5006F08BFCB60CC680A69124B944290
:102E600002D100221A721CE08CBFC4F50062C4EBD0
:102E700002025A614E690C4D402EA2B205D940346F
:102E8000403EEC606E61402304E03444EC6000247A
:102E9000B3B26C6101240C72044C8121224401F014
:102EA00055F8002070BD00BF8C4A00209B590020BF
:102EB00038B5282303FB0101074C084B05461B6965
:102EC0002046B1F88C13984728460121224640231A
:102ED00001F021F8002038BD53590020A80000203F
:102EE00070B50B78064613F060050C4627D0202DF0
:102EF00021D1CD884A78BDB11B060BD5214B104698
:102F00009B682A462049984730461F49E28800F0CE
:102F1000ABF807E01D4B1C491A601D4B2A461D608B
:102F200000F0BCF800252BE0164B10469B682946A4
:102F30002A46984724E000F011F9022520E04B785A
:102F40000A2B11D00B2B14D0062B19D14B881B0A3E
:102F5000212B05D1CA880F493A2A28BF3A2201E01D
:102F60000D493A22304601E00C49012200F07CF87C
:102F700006E08B7813B9064B9D6101E000F0EEF896
:102F8000284670BDA80000209359002010010020A1
:102F90008C4A0020260100201D010020A44A0020A8
:102FA00010B58121044600F09EFF2046012100F06B
:102FB0009AFF8221204600F096FF024B5B689847FB
:102FC000002010BDA800002038B581210446402211
:102FD000022300F067FF204601214022022300F077
:102FE00061FF822120460822032300F05BFF084B8B
:102FF000022200251A715D71064B1B689847204616
:103000000121054A402300F086FF284638BD00BF55
:1030100044000020A80000205359002038B5104972
:103020000B7A012B19D14C690CB90C7215E0402CAC
:1030300007D9CB68403C9AB24033CB604C61402307
:1030400006E0CD68A3B22C44CC600024AAB24C6147
:10305000044C8121224400F079FF002038BD00BFDC
:103060008C4A00209B59002038B50446C4F83C2106
:10307000C4F838210D461346022280F811210021A0
:103080002A4600F063FF002038BD10B50C461346F9
:103090000021224600F05AFF002010BD38B504463A
:1030A000C4F89423C4F890230D461346032280F8F5
:1030B000112100212A4600F02EFF002038BD10B556
:1030C0000C4613460021224600F025FF002010BDCB
:1030D00010B50021042304460A4680F811310B463E
:1030E00000F034FF204600F0C5FD002010BD10B5F3
:1030F0000021052304460A4680F811310B4600F0F2
:103100000AFF204600F0B6FD002010BD282303FB77
:103110000101B1F88C03704790F8CC350B7090F832
:10312000CD354B7090F8CF2590F8CE3503EB0223C8
:103130004B8090F8D12590F8D03503EB02238B809B
:1031400090F8D32590F8D23503EB02239BB2CB80C5
:10315000C0F84031012380F81131704710B580214B
:10316000044600F00CFF2046002100F008FF204636
:10317000BDE8104000F07EBD73B54B7804460D46A7
:10318000092B00F21681DFE813F0C70002011401D9
:10319000DA0014016E000A001401B9008D006B887A
:1031A0001A0A013A062A00F20481DFE812F0070049
:1031B0001A0027000201020102010201D0F8EC35D9
:1031C0000DF106011B6880789847EB880146402B7B
:1031D00003D094F81231012B35D10823ADF8063015
:1031E00031E0D0F8E4350DF106019B6A807898470C
:1031F000022343700146C4F8F00524E0DBB2052B3E
:1032000000F2D780DFE803F003070B0F1317D0F8A5
:10321000EC355B6812E0D0F8EC359B680EE0D0F836
:10322000EC35DB680AE0D0F8EC351B6906E0D0F835
:10323000EC355B6902E0D0F8EC359B690DF10601D5
:10324000A07898470146BDF80630002B00F0B58005
:10325000EA88002A00F0B1809A4228BF1A46ADF8E9
:103260000620204668E0AB88002B40F0A280EB8867
:10327000002B40F09E8090F81231AE78032B06F0C0
:103280007F0600F0968080F81461314600F0B7FEAA
:103290002046FFF71DFF0EB1022300E0012384F852
:1032A00012318AE0A978464E0129317000F28180FE
:1032B00090F81231022B02D0032B09D079E00029BB
:1032C00061D00121032380F8101180F8123111E040
:1032D00039B9022380F8123180F81011FFF782FD0E
:1032E00051E090F8101101294DD0FFF77BFD3178A6
:1032F00084F810112046FFF769FD44E0EA88012AAE
:1033000057D190F81231022B04D0032B51D100F584
:10331000887111E02B490FE090F81231023B012B2C
:1033200047D8274B01229A60D0F818210AB103220E
:103330009A60254920460222FFF796FE3DE06B8801
:10334000012B2DD0022B38D1AA8812F0FF0F34D1D7
:103350000369120A013A5B68042A0FD8DFE802F019
:10336000030507090B00012206E0022204E0032204
:1033700002E0042200E0052262F30613134A136000
:10338000012384F816312046FFF7A2FE15E090F8DD
:103390001231023B012B0CD86B88012B0DD100237D
:1033A000C4F81831D4F8E43520469B68294698477C
:1033B000E9E720462946FFF7D1FE002002B070BDA4
:1033C000A84A0020AC4A0020B04A00200C59002036
:1033D00038B590F812310446032B0D460CD10B7909
:1033E000012B09D8D0F8E4359B689847EB882BB9B6
:1033F0002046FFF76DFE01E0FFF7B0FE002038BD6C
:1034000070B54E788A88012E04460D46D3B210D08E
:1034100027D3032E50D190F81221022A28D0032A54
:1034200048D14A889AB95E0611D0194600F0A7FD26
:103430000DE090F81221022A1AD0032A3AD14A88C4
:10344000002A39D1590608D0194600F0B2FDD4F847
:10345000E43520469B68294698472046FFF738FE0A
:103460002AE090F81251022D02D0032D06D021E05F
:103470005A0621D0194600F082FD1DE012F0800F9F
:103480004FF028010D4A10D003F07F0301FB030128
:1034900091F81E310BB1012300E00023D3602046D8
:1034A00007490222FFF7E0FD06E001FB030393F862
:1034B0007633EFE7FFF752FE002070BDA84A0020E8
:1034C000B44A002030B5D0B10023DCB20133C518B6
:1034D00015F8015C002DF8D1631C5B0013800B70A4
:1034E00003234B700138022310F8012F3AB15C1C02
:1034F000CA54E4B202330022DBB20A55F4E730BD0D
:1035000037B50023104C054601930320F8F7EEF879
:103510002B68013C1A69019213D0019A002AF4DA4F
:10352000019A42F001020192019A1A61064A196950
:10353000013A019102D00199C907F8D40320F8F7A4
:10354000D5F8002003B030BD410D030030B5C4787C
:103550006CB900EB82000333D0F8D0509B102246A8
:103560009A4204D051F8220001322860F8E7002086
:1035700030BD10B50332D0F8D040921000239342F2
:103580004FEA830004D0206841F823000133F6E7B6
:10359000084410BD0122F0B50023827001294FF0CC
:1035A0004002C37082800CD108230370042343704F
:1035B0004FF4A073C38002230372C1724FF0A04383
:1035C00009E041B90C230370062343704FF4A06354
:1035D000C380234BC17203F5006245780261C3606A
:1035E000024619460024AC4201F1200602F1040211
:1035F00008D201F5106701F530611165576101349A
:103600003146F0E7047803F58062426103EB44152C
:1036100003F58862C0F8CC2005F5A06503F5A0622B
:103620000146AA4201F1040103D0C1F88C202032E6
:10363000F7E703EB043403F5805204F580540146A8
:10364000A24201F1040104D0C1F8CC2002F580525D
:10365000F6E703F56063C0F80C310020F0BD00BF51
:103660000000044038B5037A0546012B4FF00004F2
:1036700050F80C2F1ED1936B697A64F3104309B193
:1036800043F480139363D3686FF386136FF39653F9
:103690006FF351436FF3D343D360FFF731FFEB7800
:1036A000012B19D1052363F34404EB6844F0200493
:1036B0009C6011E0D36843F04003D360FFF720FF24
:1036C0006B7AEA68002B0CBF4FF450234FF4E813D9
:1036D00093631420F8F714F8EB78012B07D1EB680B
:1036E00005229C6862F3440444F020049C6000209E
:1036F00038BDC36800209A6842F001029A607047A2
:10370000C36800209A6822F001029A60704707B5EA
:1037100000230193019B43F020030193019B61F37C
:103720008A130193019BC2681361074B1169013B26
:10373000019102D001998906F8D40320F7F7D6FF4A
:10374000002003B05DF804FB410D030007B5002322
:103750000193019B43F010030193019BC268136125
:10376000074B1169013B019102D00199C906F8D4B8
:103770000320F7F7BBFF002003B05DF804FB00BF98
:10378000410D0300C26808B5D36801296FF35D736A
:103790006FF39E7302D143F0005302E009B943F086
:1037A0008043D3603220F7F7ABFF002008BDC36829
:1037B000586900F001007047C368586900F00100C3
:1037C00080F001007047C368586900F0010070473D
:1037D000C3685A69986910407047C3685868704751
:1037E00003691A6861F301021A60704710B5C26874
:1037F00000236FF080414FF0FF34936151615460BA
:10380000516109499161C1780020994208BF102394
:1038100043F0804343F47013916943F4605343F0E1
:103820000C030B43936110BD0008008038B5D0F83D
:103830000C3100221A60036915461A68044665F3C4
:10384000CC221A60C37A012B21D10321FFF7C8FFD4
:10385000E36880214FF4001261F30F0259629A620B
:10386000A02262F30F0561F31F454FF49072C3F875
:10387000045162F30F05C0F220054FF4A072C3F8A3
:10388000085162F30F056FF31F45C3F80C51102167
:103890002046FFF73CFF2046FFF758FF2369002230
:1038A0004FF0FF311A615A619961DA6161788A4299
:1038B0000FD204EB82018969013208680028ACBF8D
:1038C00000204FF09040086000200861FF208860D1
:1038D000ECE7002261788A420FD204EB8201496D45
:1038E000013208680028ACBF00204FF0904008600B
:1038F00000200861FF208860ECE71A6942F48072BA
:103900001A61E278012A04D1044A402161F3594244
:103910001A632046FFF76AFF002038BD030101004B
:1039200003699B68C3F34103022B05D0032B05D029
:10393000012B03D0032070470120704702207047FD
:10394000036910B59C688169C4F341000A680228C4
:1039500006BF032060F30A026FF30A020A605A6886
:10396000002042F480725A6010BD30B54D780B785B
:10397000012D4FF0000200EB830405D105FA03F39B
:10398000A46963F30F0205E0012505FA03F3646DF2
:1039900063F31F4223681D040DD48D6865F30A0389
:1039A000CD78C98865F3934361F3995343F080530D
:1039B00043F40043236003690020D9690A43DA61B4
:1039C00030BD30B54D780B780024012D224600EB38
:1039D000830105D105FA03F3896963F30F0205E05A
:1039E000012505FA03F3496D63F31F4203696FF381
:1039F000CF340C60D969002021EA0202DA6130BDBF
:103A0000F8B54E780A460978012E536900EB81011A
:103A100045D18D6929682C6963F3120413B966F3E3
:103A2000DC440BE096689F19013FB7FBF6F666F39E
:103A3000DC44D678012E08BF66F35E742C61C4782E
:103A40001578012C05D100EB8505AD6914696C6111
:103A50000AE0D478012C07D033B1012707FA05F525
:103A60000469666B35436563D478012C07D104691A
:103A7000A468E40554BF41F0005141F0805114782E
:103A800041F0044100EB8404A4692160D17801294C
:103A900036D1D1689BB21278FFF758FD30E04E6DF9
:103AA0009568316834692BB965F31204012363F317
:103AB000DC440AE02B44013BB3FBF5F363F3DC4445
:103AC000C3F309035D4365F312043461C378012B2A
:103AD00005D1137800EB83035C6D13696361D378C0
:103AE000012B06D1537913B141F0005101E041F0AF
:103AF0008051137841F0044100EB8300436D19605D
:103B00000020F8BDF7B591F801C04A69BCF1010F7A
:103B10003DD18469236826690096F5B2C6F307474C
:103B200042B962F306056CF3C4078DF800508DF8B6
:103B300002700FE08E68B2428ABF66F3060562F338
:103B400006054E6101223E4662F3C4068DF8005020
:103B50008DF80260009A2261C278012A05D10A78A4
:103B600000EB820295690A696A6143F004432360AD
:103B7000C378002B3FD14B69002B3CD00A78012140
:103B800001FA02F20369586B02435A6333E00B787F
:103B900000EB83035C6D236825690095EFB2C5F3E4
:103BA00007468D684AB9012265F3060762F3C40629
:103BB0008DF800708DF802600BE03A4665F306025E
:103BC0004D618DF800203546012262F3C4058DF861
:103BD0000250009A2261C278012A05D10A7800EBCE
:103BE0008202546D0A6962610A7843F0044300EB73
:103BF0008200426D1360002003B0F0BD4B78012BB2
:103C00000B7800EB830006D182691368002B04DA7D
:103C100043F0804301E0426D136843F400131360E6
:103C2000002070474B78012B0B78C97800EB83009C
:103C30000CBF8269426D0239136801296FF3555335
:103C400098BF43F0805313600020704703699A695E
:103C5000D8691040000C704700EB81014B6D026980
:103C60009B6850691840704703699869DB69184080
:103C700080B2704782B000230093C0238DF80330D8
:103C800001224FF0000362F3C4038DF802301823C1
:103C90008DF80030009A436D1A61C278012A06D16E
:103CA00000F2CC5058611A684FF080221A6002B0BE
:103CB0007047D0F8183110B50446D3B103699A683B
:103CC000D20716D5827A42B1D0F80C21D0F80C1167
:103CD0006FF341026FF300020A605A68052042F058
:103CE00001025A60F7F70CFD23695A6822F00102BD
:103CF0005A6010BD837A63B103699B68DB0708D5FE
:103D0000D0F80C31D0F80C216FF341036FF30003AE
:103D100013607047012310B5002280F81231044669
:103D20000346617804338A4206D25869FF218160D4
:103D3000186D01328160F4E7236900221A615A612B
:103D4000DA614FF0FF3220469A61FFF7FFFC204610
:103D50001021BDE81040FFF7DABC4B78012B0B783F
:103D600000EB830009D183691B68990211D413F415
:103D7000003F0CBF302020207047436D1B689A0223
:103D800009D413F4003F0CBF4FF440504FF40050DF
:103D90007047102070474FF48050704730B54D7811
:103DA0000C46012D0D7800EB85030BD19D69102A7F
:103DB0002B6803D1BDE83040FFF720BF202A0CD08C
:103DC000302A0FE05D6DB2F5805F2B6802D143F4BD
:103DD000001318E0B2F5005F02D143F0006312E077
:103DE000B2F5405F0CD19A0205D500236371BDE89E
:103DF0003040FFF717BF43F0044343F4004302E0B1
:103E00000AB962F3CF332B6030BD00BF10B5044652
:103E1000FFF7C0FB0123002284F8123184F814213B
:103E20002346617828338A4212D2012183F8F510A3
:103E30004020002183F8F420A3F8FA2083F8F7103B
:103E4000C3F8FC00C3F80011C3F808110132E8E719
:103E500023460022617828338A4211D20021402073
:103E600083F84C23A3F8522383F84D1383F84F13A0
:103E7000C3F85403C3F85813C3F860130132E9E7D9
:103E80002046FFF73DFC2046FFF7ECFB20460021D3
:103E9000FFF778FC2046FFF7C9FC2046BDE810403C
:103EA000FFF727BC70B5CDB215F0800F01F07F048D
:103EB0004FF0280615BF06FB040106FB010101F5C2
:103EC0008E7101F55D71E4B2ED090C704D708A6080
:103ED000CB7005B1CC80022B04BF00230B71FFF720
:103EE00044FD002070BDCBB213F0800F01F07F02C3
:103EF00010B54FF0280415BF04FB020104FB0101BB
:103F000001F58E7101F55D71DB090A704B70FFF7E9
:103F100058FD002010BD38B501F07F04282505FBB1
:103F2000040505F55D714B610023CA608B614B7020
:103F300085F87443C378012B08BF0A6114B9FFF7F1
:103F4000E1FD01E0FFF75CFD002038BD70B501F038
:103F50007F04282505FB0405012605F58E714E70AA
:103F600085F81C41CA600A6100228A614B6114B95C
:103F7000FFF7C8FD01E0FFF743FD002070BDCBB2A5
:103F800013F0800F01F07F0210B54FF0280415BF29
:103F900004FB020104FB010101F58E7101F55D7165
:103FA000DB0901248C700A704B70FFF727FE00209C
:103FB00010BDCBB213F0800F01F07F0210B54FF0AF
:103FC000280415BF04FB020104FB010101F58E71F9
:103FD00001F55D710024DB098C700A704B70FFF7EE
:103FE00021FE204610BD08B50B0604D501F07F0167
:103FF000FFF78DFB01E0FFF7A9FB002008BD026978
:10400000002361F30A1311680B43136070470369BF
:1040100003205A686FF341025A60F7F771BB0369D6
:1040200003205A6842F002025A60F7F769BB11F0A8
:10403000800F4FF0280306D001F07F0103FB010140
:1040400001F58E7103E003FB010101F55D71FFF7DE
:1040500084BE11F0800F4FF0280306D001F07F01DD
:1040600003FB010101F58E7103E003FB010101F582
:104070005D71FFF793BE00002DE9F04F85B0044657
:10408000FFF79AFB08B900201DE22046FFF7A0FBCE
:1040900006460028F7D0C0F3C04000284FD0204685
:1040A000FFF7D4FD27468046A1464FF0000AB8F13D
:1040B000000F43D018F0010F38D05FFA8AFB594641
:1040C0002046FFF7C9FDC107054620D57B6D0125B8
:1040D0009D60E278AA4207D11A69D9F87C33C2F30D
:1040E00012029B1AC9F88C33A64B20461B6859460E
:1040F0001B689847E378012B09D1BAF1000F06D16C
:1041000094F81131052B02D12046FFF7B3FDAA0721
:1041100002D57B6D02259D602B0707D5994B204664
:104120001B6808259B6898477B6D9D600AF1010A12
:104130004FEA5808043709F12809B8E70120750348
:1041400040F1A3802046FFF78FFDA0468246274618
:104150004FF00009BAF1000F00F096801AF0010F3D
:1041600000F08A8023695FFA89FB19695D6B04EBB3
:104170008B0225FA0BF59269ED019268EDB20D43C1
:104180001540E8071CD5012505FA09F15A6B2046B0
:1041900022EA01025A63D8F8183059469D60794BDB
:1041A0001B685B689847E378AB4209D1B9F1000F0F
:1041B00006D194F81131042B02D12046FFF75AFDA5
:1041C000290703D5D8F8183008259D60EA0603D5DD
:1041D000D8F8183010259D606B0603D5D8F8183034
:1041E00040259D60A80703D5D8F8183002259D60AA
:1041F000290641D5D7F83431D7F83021D21AD7F86B
:1042000024319A4238BF134603F1030CD8F8183012
:104210004FEA9C0C9B699BB2634529D9D7F834516E
:10422000D7F830319D4223D213B3D7F824215D1B38
:10423000954228BF154605F1030C4FEA9C0CABB222
:10424000D7F8281120465A46CDF804C0FFF77EF96A
:10425000D7F828312B44C7F82831D7F834311D441A
:10426000C7F83451D8F81830DDF804C09B69D2E79C
:10427000D8F8183080259D6009F101094FEA5A0AE3
:1042800008F10408283765E70120B20702D5E36882
:1042900002225A61002E19DAA37A43B1D4F80C3104
:1042A000D4F80C216FF341036FF30003136023690B
:1042B00020465A6822F001025A60324B1B689B6903
:1042C0009847E3684FF000425A61012033052DD52D
:1042D00000238DF80F3094F8123120468DF80F30FE
:1042E000284B1B685B69984723694FF400619A6803
:1042F000E3685961A37AC3B1D70716D594F815318D
:10430000012B12D19DF80F30032B0ED1D4F80C31B4
:104310001A6842F001021A601A6842F003021A6039
:10432000194B1A6942F006021A610120350708D5B7
:10433000144B20461B68DB689847E36808225A61E3
:104340000120F10636D5E36828259A6922F010028B
:104350009A611F6A07F00F0305FB0345C7F3434348
:10436000022B05F55D7511D0062B1DD1204604F2F8
:10437000CC510822FFF7FDF8AB69C7F30A173B449D
:10438000AB6111E0E000002000ED00E0C7F30A1788
:1043900057B13A462046E968FFF7EBF8EB683B4433
:1043A000EB60AB691F44AF61E36801209A6942F09A
:1043B00010029A61F20434D5236900255A68204618
:1043C00022F001025A602946FFF7A1F923462A4646
:1043D000617804338A4206D25869FF218160186DE2
:1043E00001328160F4E7236901274FF0FF3267F360
:1043F0000F059A6167F31F450B22DD615A611A614F
:104400001A6820466FF30A121A60FFF733FCE3685C
:104410004FF480525A612D4B20461B681B69984708
:104420003846B3041DD52046FFF78AFAE3682046D4
:10443000DD68FFF775FA032806D10023A3704FF457
:104440000073A380092304E00123A3704023A38009
:10445000052363F38D25E3684FF40052DD600120EE
:104460005A61F70209D5194B20461B68DB6998474A
:10447000E3684FF480125A610120B50209D5134B4D
:1044800020461B681B6A9847E3684FF400125A6184
:104490000120710009D50D4B20461B685B6A9847C7
:1044A000E3684FF080425A61012072070BD5E36840
:1044B0005D686B0704D5054B20461B689B6A9847CF
:1044C000E36801205D6005B0BDE8F08FE0000020EA
:1044D00081F0004102E000BF83F0004330B54FEAB5
:1044E00041044FEA430594EA050F08BF90EA020F22
:1044F0001FBF54EA000C55EA020C7FEA645C7FEAB5
:10450000655C00F0E2804FEA5454D4EB5555B8BFD7
:104510006D420CDD2C4480EA020281EA030382EA48
:10452000000083EA010180EA020281EA0303362DDA
:1045300088BF30BD11F0004F4FEA01314FF4801CAD
:104540004CEA113102D0404261EB410113F0004FBF
:104550004FEA03334CEA133302D0524263EB430376
:1045600094EA050F00F0A780A4F10104D5F1200E14
:104570000DDB02FA0EFC22FA05F2801841F100016F
:1045800003FA0EF2801843FA05F359410EE0A5F143
:1045900020050EF1200E012A03FA0EFC28BF4CF074
:1045A000020C43FA05F3C01851EBE37101F000452A
:1045B00007D54FF0000EDCF1000C7EEB00006EEB37
:1045C0000101B1F5801F1BD3B1F5001F0CD34908C1
:1045D0005FEA30004FEA3C0C04F101044FEA445218
:1045E00012F5800F80F09A80BCF1004F08BF5FEA9F
:1045F000500C50F1000041EB045141EA050130BD7F
:104600005FEA4C0C404141EB010111F4801FA4F121
:104610000104E9D191F0000F04BF01460020B1FA76
:1046200081F308BF2033A3F10B03B3F120020CDAAE
:104630000C3208DD02F1140CC2F10C0201FA0CF08C
:1046400021FA02F10CE002F11402D8BFC2F1200CF1
:1046500001FA02F120FA0CFCDCBF41EA0C019040A7
:10466000E41AA2BF01EB0451294330BD6FEA0404F0
:104670001F3C1CDA0C340EDC04F11404C4F12002DB
:1046800020FA04F001FA02F340EA030021FA04F3ED
:1046900045EA030130BDC4F10C04C4F1200220FA44
:1046A00002F001FA04F340EA0300294630BD21FA82
:1046B00004F0294630BD94F0000F83F4801306BF48
:1046C00081F480110134013D4EE77FEA645C18BF3C
:1046D0007FEA655C29D094EA050F08BF90EA020FD3
:1046E00005D054EA000C04BF1946104630BD91EACB
:1046F000030F1EBF0021002030BD5FEA545C05D1CE
:104700004000494128BF41F0004130BD14F580040C
:104710003CBF01F5801130BD01F0004545F0FE4180
:1047200041F470014FF0000030BD7FEA645C1ABFB5
:10473000194610467FEA655C1CBF0B46024650EAEC
:10474000013406BF52EA033591EA030F41F4002118
:1047500030BD00BF90F0000F04BF0021704730B59E
:104760004FF4806404F132044FF000054FF0000173
:1047700050E700BF90F0000F04BF0021704730B534
:104780004FF4806404F1320410F0004548BF404209
:104790004FF000013EE700BF42004FEAE2014FEA5E
:1047A00031014FEA02701FBF12F07F4393F07F4F39
:1047B00081F06051704792F0000F14BF93F07F4F6B
:1047C000704730B54FF4607401F0004521F00041AE
:1047D00020E700BF50EA010208BF704730B54FF034
:1047E00000050AE050EA010208BF704730B511F039
:1047F000004502D5404261EB41014FF4806404F171
:1048000032045FEA915C3FF4DCAE4FF003025FEAF2
:10481000DC0C18BF03325FEADC0C18BF033202EB7A
:10482000DC02C2F1200300FA03FC20FA02F001FAD4
:1048300003FE40EA0E0021FA02F11444C1E600BF73
:1048400070B54FF0FF0C4CF4E06C1CEA11541DBF26
:104850001CEA135594EA0C0F95EA0C0F00F0DEF8F1
:104860002C4481EA030621EA4C5123EA4C5350EAD6
:10487000013518BF52EA033541F4801143F4801327
:1048800038D0A0FB02CE4FF00005E1FB02E506F0B8
:104890000042E0FB03E54FF00006E1FB03569CF00D
:1048A000000F18BF4EF0010EA4F1FF04B6F5007F13
:1048B00064F5407404D25FEA4E0E6D4146EB060685
:1048C00042EAC62141EA55514FEAC52040EA5E500E
:1048D0004FEACE2EB4F1FD0C88BFBCF5E06F1ED8B8
:1048E000BEF1004F08BF5FEA500E50F1000041EBEF
:1048F000045170BD06F0004646EA010140EA02009C
:1049000081EA0301B4EB5C04C2BFD4EB0C0541EABD
:10491000045170BD41F480114FF0000E013C00F3D2
:10492000AB8014F1360FDEBF002001F0004170BDF6
:10493000C4F10004203C35DA0C341BDC04F114040F
:10494000C4F1200500FA05F320FA04F001FA05F29B
:1049500040EA020001F0004221F0004110EBD37068
:1049600021FA04F642EB06015EEA430E08BF20EA94
:10497000D37070BDC4F10C04C4F1200500FA04F337
:1049800020FA05F001FA04F240EA020001F00041C9
:1049900010EBD37041F100015EEA430E08BF20EA3C
:1049A000D37070BDC4F1200500FA05F24EEA020E84
:1049B00020FA04F301FA05F243EA020321FA04F0B3
:1049C00001F0004121FA04F220EA020000EBD3706A
:1049D0005EEA430E08BF20EAD37070BD94F0000F6A
:1049E0000FD101F00046400041EB010111F4801F9E
:1049F00008BF013CF7D041EA060195F0000F18BF4F
:104A0000704703F00046520043EB030313F4801F8A
:104A100008BF013DF7D043EA0603704794EA0C0F44
:104A20000CEA135518BF95EA0C0F0CD050EA41065A
:104A300018BF52EA4306D1D181EA030101F00041D7
:104A40004FF0000070BD50EA410606BF10461946FF
:104A500052EA430619D094EA0C0F02D150EA01360B
:104A600013D195EA0C0F05D152EA03361CBF10464C
:104A700019460AD181EA030101F0004141F0FE41EB
:104A800041F470014FF0000070BD41F0FE4141F46F
:104A9000780170BD70B54FF0FF0C4CF4E06C1CEA6F
:104AA00011541DBF1CEA135594EA0C0F95EA0C0F24
:104AB00000F0A7F8A4EB050481EA030E52EA0335DF
:104AC0004FEA013100F088804FEA03334FF0805500
:104AD00045EA131343EA12634FEA022245EA11152D
:104AE00045EA10654FEA00260EF000419D4208BFDE
:104AF000964244F1FD0404F5407402D25B084FEA8B
:104B00003202B61A65EB03055B084FEA32024FF436
:104B100080104FF4002CB6EB020E75EB030E22BF93
:104B2000B61A754640EA0C005B084FEA3202B6EB53
:104B3000020E75EB030E22BFB61A754640EA5C0002
:104B40005B084FEA3202B6EB020E75EB030E22BF92
:104B5000B61A754640EA9C005B084FEA3202B6EB93
:104B6000020E75EB030E22BFB61A754640EADC0052
:104B700055EA060E18D04FEA051545EA16754FEAB4
:104B800006164FEAC30343EA52734FEAC2025FEAD2
:104B90001C1CC0D111F4801F0BD141EA00014FF061
:104BA00000004FF0004CB6E711F4801F04BF014332
:104BB0000020B4F1FD0C88BFBCF5E06F3FF6AFAE4E
:104BC000B5EB030C04BFB6EB020C5FEA500C50F1DE
:104BD000000041EB045170BD0EF0004E4EEA113161
:104BE00014EB5C04C2BFD4EB0C0541EA045170BD68
:104BF00041F480114FF0000E013C90E645EA060EAC
:104C00008DE60CEA135594EA0C0F08BF95EA0C0FD9
:104C10003FF43BAF94EA0C0F0AD150EA01347FF421
:104C200034AF95EA0C0F7FF425AF104619462CE7F8
:104C300095EA0C0F06D152EA03353FF4FDAE10465B
:104C4000194622E750EA410618BF52EA43067FF4AC
:104C5000C5AE50EA41047FF40DAF52EA43057FF43C
:104C6000EBAE12E74FF0FF3C06E000BF4FF0010C47
:104C700002E000BF4FF0010C4DF804CD4FEA410CAB
:104C80007FEA6C5C4FEA430C18BF7FEA6C5C1BD078
:104C900001B050EA410C0CBF52EA430C91EA030FF9
:104CA00002BF90EA020F0020704710F1000F91EA56
:104CB000030F58BF994208BF90422CBFD8176FEA24
:104CC000E37040F0010070474FEA410C7FEA6C5CF2
:104CD00002D150EA013C07D14FEA430C7FEA6C5CF9
:104CE000D6D152EA033CD3D05DF8040B704700BF25
:104CF0008446104662468C461946634600E000BF73
:104D000001B5FFF7B7FF002848BF10F1000F01BD44
:104D10004DF808EDFFF7F4FF0CBF012000205DF80F
:104D200008FB00BF4DF808EDFFF7EAFF34BF012094
:104D300000205DF808FB00BF4DF808EDFFF7E0FF2D
:104D400094BF012000205DF808FB00BF4DF808ED7E
:104D5000FFF7CEFF94BF012000205DF808FB00BFE5
:104D60004DF808EDFFF7C4FF34BF012000205DF8C7
:104D700008FB00BF4FEA410212F5001215D211D50F
:104D80006FF47873B3EB625212D94FEAC12343F048
:104D9000004343EA505311F0004F23FA02F018BFCA
:104DA000404270474FF00000704750EA013005D193
:104DB00011F0004008BF6FF0004070474FF0000056
:104DC000704700BF4FEA4102B2F1E04324BFB3F5A0
:104DD000001CDCF1FE5C0DD901F0004C4FEAC00272
:104DE0004CEA5070B2F1004F40EB830008BF20F056
:104DF0000100704711F0804F21D113F13872BCBF10
:104E000001F00040704741F480114FEA5252C2F164
:104E10001802C2F1200C10FA0CF320FA02F018BFAD
:104E200040F001004FEAC1234FEAD32303FA0CFC00
:104E300040EA0C0023FA02F34FEA4303CCE77FEA8F
:104E4000625307D150EA01331EBF4FF0FE4040F4D9
:104E50004000704701F0004040F0FE4040F4000088
:104E6000704700BF80F0004002E000BF81F00041C9
:104E700042001FBF5FEA410392EA030F7FEA226C00
:104E80007FEA236C6AD04FEA1262D2EB1363C1BF90
:104E9000D218414048404140B8BF5B42192B88BFFF
:104EA000704710F0004F40F4000020F07F4018BF22
:104EB000404211F0004F41F4000121F07F4118BF42
:104EC000494292EA030F3FD0A2F1010241FA03FCEA
:104ED00010EB0C00C3F1200301FA03F100F00043D2
:104EE00002D5494260EB4000B0F5000F13D3B0F19A
:104EF000807F06D340084FEA310102F10102FE2A09
:104F000051D2B1F1004F40EBC25008BF20F0010078
:104F100040EA03007047490040EB000010F4000F26
:104F2000A2F10102EDD1B0FA80FCACF1080CB2EBB9
:104F30000C0200FA0CF0AABF00EBC2505242184318
:104F4000BCBFD0401843704792F0000F81F40001BD
:104F500006BF80F400000132013BB5E74FEA410390
:104F60007FEA226C18BF7FEA236C21D092EA030FFC
:104F700004D092F0000F08BF0846704790EA010F76
:104F80001CBF0020704712F07F4F04D1400028BFA3
:104F900040F00040704712F100723CBF00F5000085
:104FA000704700F0004343F0FE4040F400007047BB
:104FB0007FEA226216BF08467FEA23630146420267
:104FC00006BF5FEA412390EA010F40F4800070477A
:104FD0004FF0000304E000BF10F0004348BF404220
:104FE0005FEA000C08BF704743F0964301464FF05C
:104FF00000001CE050EA010208BF70474FF00003B8
:105000000AE000BF50EA010208BF704711F00043F8
:1050100002D5404261EB41015FEA010C02BF8446C8
:105020000146002043F0B64308BFA3F18053A3F527
:105030000003BCFA8CF2083AA3EBC25310DB01FA6E
:1050400002FC634400FA02FCC2F12002BCF1004FF2
:1050500020FA02F243EB020008BF20F00100704783
:1050600002F1200201FA02FCC2F1200250EA4C00D7
:1050700021FA02F243EB020008BF20EADC7070471D
:105080004FF0FF0C1CEAD0521EBF1CEAD15392EA2B
:105090000C0F93EA0C0F6FD01A4480EA010C400207
:1050A00018BF5FEA41211ED04FF0006343EA501061
:1050B00043EA5111A0FB01310CF00040B1F5000FA3
:1050C0003EBF490041EAD3715B0040EA010062F152
:1050D0007F02FD2A1DD8B3F1004F40EBC25008BF3C
:1050E00020F00100704790F0000F0CF0004C08BF5A
:1050F00049024CEA502040EA51207F3AC2BFD2F127
:10510000FF0340EAC250704740F400004FF0000334
:10511000013A5DDC12F1190FDCBF00F0004070476E
:10512000C2F10002410021FA02F1C2F1200200FAAC
:1051300002FC5FEA310040F1000053EA4C0308BF73
:1051400020EADC70704792F0000F00F0004C02BFC4
:10515000400010F4000F013AF9D040EA0C0093F03F
:10516000000F01F0004C02BF490011F4000F013B99
:10517000F9D041EA0C018FE70CEAD15392EA0C0F07
:1051800018BF93EA0C0F0AD030F0004C18BF31F072
:10519000004CD8D180EA010000F00040704790F048
:1051A000000F17BF90F0004F084691F0000F91F0EC
:1051B000004F14D092EA0C0F01D142020FD193EAB2
:1051C0000C0F03D14B0218BF084608D180EA01003A
:1051D00000F0004040F0FE4040F40000704740F016
:1051E000FE4040F4400070474FF0FF0C1CEAD052E4
:1051F0001EBF1CEAD15392EA0C0F93EA0C0F69D040
:10520000A2EB030280EA010C49024FEA402037D0AA
:105210004FF0805343EA111143EA10130CF00040A1
:105220008B4238BF5B0042F17D024FF4000C8B4291
:1052300024BF5B1A40EA0C00B3EB510F24BFA3EB71
:10524000510340EA5C00B3EB910F24BFA3EB910341
:1052500040EA9C00B3EBD10F24BFA3EBD10340EA9B
:10526000DC001B0118BF5FEA1C1CE0D1FD2A3FF6E1
:1052700050AF8B4240EBC25008BF20F00100704796
:105280000CF0004C4CEA50207F32C2BFD2F1FF0339
:1052900040EAC250704740F400004FF00003013A6A
:1052A00037E792F0000F00F0004C02BF400010F40E
:1052B000000F013AF9D040EA0C0093F0000F01F022
:1052C000004C02BF490011F4000F013BF9D041EA44
:1052D0000C0195E70CEAD15392EA0C0F08D1420277
:1052E0007FF47DAF93EA0C0F7FF470AF084676E74A
:1052F00093EA0C0F04D14B023FF44CAF08466EE723
:1053000030F0004C18BF31F0004CCAD130F00042F0
:105310007FF45CAF31F000437FF43CAF5FE700BF48
:105320004FF0FF3C06E000BF4FF0010C02E000BF71
:105330004FF0010C4DF804CD4FEA40024FEA410313
:105340007FEA226C18BF7FEA236C11D001B052EAC9
:10535000530C18BF90EA010F58BFB2EB030088BF8F
:10536000C81738BF6FEAE17018BF40F001007047FE
:105370007FEA226C02D15FEA402C05D17FEA236CE0
:10538000E4D15FEA412CE1D05DF8040B704700BF27
:10539000844608466146FFE70FB5FFF7C9FF0028BE
:1053A00048BF10F1000F0FBD4DF808EDFFF7F4FFF7
:1053B0000CBF012000205DF808FB00BF4DF808ED90
:1053C000FFF7EAFF34BF012000205DF808FB00BFB3
:1053D0004DF808EDFFF7E0FF94BF012000205DF8D5
:1053E00008FB00BF4DF808EDFFF7D2FF94BF012086
:1053F00000205DF808FB00BF4DF808EDFFF7C8FF7F
:1054000034BF012000205DF808FB00BF42000ED22F
:10541000B2F1FE4F0BD34FF09E03B3EB126209D4EF
:105420004FEA002343F0004323FA02F070474FF0A5
:105430000000704712F1610F01D1420202D14FF01A
:10544000FF3070474FF00000704700BF73B96AB972
:10545000002908BF0028BCBF00204FF00041C4BF96
:105460006FF000414FF0FF3000F03CB882B0EC46E6
:105470002DE9005000F006F8DDF804E002B00CBCA5
:10548000704700BF2DE9704F089E14461D468046A8
:10549000894600F029F804FB01F3A4FB00AB00FBF4
:1054A00005329344B8EB0A0869EB0B09C6E9008999
:1054B000BDE8708F2DE9704F089E14461D4680464A
:1054C000894600F061F900FB05F5A0FB04AB04FB85
:1054D0000154A344B8EB0A0869EB0B09C6E900893B
:1054E000BDE8708F704700BF00292DE9F00FC0F2B2
:1054F000A1800024002BC0F29880154606460F4676
:10550000002B3FD18A4258D9B2FA82F34BB1C3F192
:10551000200201FA03F720FA02F29D4000FA03F696
:105520001743290CB7FBF1F201FB1277A8B200FB7D
:1055300002F34FEA164C4CEA0747BB4209D97F19E0
:1055400002F1FF3C80F00581BB4240F20281023A49
:105550002F44FF1AB7FBF1F301FB137100FB03F0BB
:10556000B6B246EA0141884208D9491903F1FF372A
:1055700080F0F180884240F2EE80023B43EA024232
:10558000002303E08B420AD900231A46104619462D
:1055900014B1404261EB4101BDE8F00F7047B3FA2E
:1055A00083F8B8F1000F40F088808B4202D382422A
:1055B00000F2E28000230122E8E712B90123B3FBE5
:1055C000F2F5B5FA85F2002A3AD17F1B280C1FFAB2
:1055D00085FC0123B7FBF0F100FB11770CFB01F216
:1055E0004FEA164848EA0747BA4207D97F1901F13E
:1055F000FF3802D2BA4200F2C4804146BF1AB7FB5C
:10560000F0F200FB12700CFB02FCB6B246EA00405E
:10561000844507D9401902F1FF3702D2844500F2D0
:10562000AE803A4642EA0142B0E7E443524263EBBD
:10563000430362E7404261EB41014FF0FF3459E719
:105640009540C2F1200927FA09F126FA09F9974095
:10565000280CB1FBF0F800FB18111FFA85FC0CFBBD
:1056600008F349EA07094FEA194747EA01418B4223
:1056700006FA02F608D9491908F1FF327AD28B42AC
:1056800078D9A8F102082944C91AB1FBF0F300FB4C
:1056900013170CFB03F21FFA89F949EA0747BA42CC
:1056A00007D97F1903F1FF3160D2BA425ED9023BBC
:1056B0002F44BF1A43EA08438CE7C8F1200225FAB9
:1056C00002F103FA08FC27FA02F320FA02F207FAC1
:1056D00008F741EA0C0C4FEA1C49B3FBF9F109FB4E
:1056E00011331FFA8CFA0AFB01FB17433A0C42EA0A
:1056F00003439B4505FA08F008D913EB0C0301F1AD
:10570000FF3235D29B4533D902396344CBEB0303D7
:10571000B3FBF9F209FB12330AFB02FABFB247EA04
:105720000347BA4508D917EB0C0702F1FF331BD228
:10573000BA4519D9023A674442EA0145A5FB00017E
:10574000CAEB07078F424FF000030AD305D02A4661
:105750001CE76246FDE63B4610E706FA08F686427D
:10576000F5D26A1E002311E71A46E5E70B46A0E7CB
:105770001146CBE7904687E74346424606E7023AA2
:1057800050E702392F4439E72DE9F00F144605465A
:105790000E46002B43D18A4253D9B2FA82F757B151
:1057A000C7F1200620FA06F601FA07F302FA07F419
:1057B00000FA07F51E43210CB6FBF1F201FB12665D
:1057C000A0B200FB02F32F0C47EA0646B34209D908
:1057D000361902F1FF3780F0FD80B34240F2FA80C3
:1057E000023A2644F61AB6FBF1F301FB136100FB03
:1057F00003F0ADB245EA0141884208D9091903F125
:10580000FF3680F0E980884240F2E680023B43EABE
:105810000242002310461946BDE8F00F70478B4244
:105820004CD8B3FA83F6002E4FD18B4202D382427A
:1058300000F2DD80BDE8F00F00230122104619467A
:10584000704712B90124B4FBF2F4B4FA84F2002ACE
:1058500040F08280091B260CA7B20123B1FBF6F0B1
:1058600006FB101107FB00F24FEA154C4CEA014110
:105870008A4207D9091900F1FF3C02D28A4200F29C
:10588000C8806046891AB1FBF6F206FB121107FBCD
:1058900002F7ADB245EA0145AF4208D92C1902F131
:1058A000FF3180F09B80A74240F29880023A42EAA2
:1058B000004210461946BDE8F00F704700231A4613
:1058C00010461946BDE8F00F7047C6F1200522FAD0
:1058D00005F703FA06F421FA05F301FA06FB20FAAC
:1058E00005F53C434FEA1448B3FBF8FC08FB1C33B6
:1058F0001FFA84F909FB0CFA45EA0B0B4FEA1B452A
:1059000045EA03439A4502FA06F204D91B190CF141
:10591000FF356FD3AC46CAEB0303B3FBF8F508FBC6
:10592000153309FB05F91FFA8BFB4BEA0347B94511
:1059300004D93F1905F1FF3362D31D4645EA0C4CEB
:10594000ACFB0223C9EB07079F424FF000054AD387
:1059500046D062462B465DE79440C2F1200921FA09
:1059600009FC914020FA09F9260CBCFBF6F806FB6D
:1059700018CCA7B207FB08F349EA01094FEA19411D
:1059800041EA0C4C634500FA02F509D91CEB040C02
:1059900008F1FF323BD2634539D9A8F10208A4448B
:1059A000C3EB0C0CBCFBF6F306FB13C107FB03F2C5
:1059B0001FFA89F949EA01418A4207D9091903F115
:1059C000FF3022D28A4220D9023B2144891A43EA7D
:1059D000084343E73A4605E7334618E70A4666E7D1
:1059E000B0409042B5D20CF1FF32002312E73346AB
:1059F00032460FE79A458DD9ACF1020C23448AE771
:105A0000B9459AD9023D274498E70346DEE7904618
:105A1000C6E70238214435E7002100F004B80C4BFA
:105A20005B58435004310B480B4B42189A42FFF429
:105A3000F6AF0A4A00F003B8002342F8043B084BD3
:105A40009A42FFF4F9AFFAF7EDFB00F00DF870475A
:105A50009465010800000020BC050020C00500205E
:105A60009C620020FFF7FEBF08B562B6F2F704FCA7
:105A7000F3F7E6FEF2F7E6FBF4F7BAF8F4F750FBBB
:105A8000F3F760F9194C28B1F3F75CF96070F3F79C
:105A900059F9A0602078F3F781FA22696079A1684A
:105AA000F3F70CFDF5F77EFEF4F7A2FFF5F7FAF930
:105AB000F2F7FEFEF8F7EAFCF9F71EFAF9F70CFD2B
:105AC0000B4B1C225A83F8F701FEF9F716FAF9F787
:105AD00017FDF2F7A5FDF2F7C3FD0028F3D0F5F7A7
:105AE000E1F9F8F7D3FCF9F7F7FCECE70400002044
:105AF0000010024000210A2200F0ACB80F4B30B475
:105B000005461C6802E0D01A16D1ABB115F8013B6E
:105B1000E21850781A4600F00300012808BF03F18C
:105B2000200211F8013BE018407800F00300012842
:105B3000E9D12033D01AE9D030BC7047B405002039
:105B40002DE9F00F424C82B0D4F800C001900E460F
:105B500000E02646344614F8015B0CEB0500407863
:105B600000F0080000F0FF0A0028F2D12D2D5BD0D4
:105B70002B2D04BF7578B41C33F010003CD099462F
:105B8000BAF1000F0CBF6FF0004B4FF0004BBBFBA6
:105B9000F9F8002709FB18BB38460CE0303DAB4252
:105BA00019DD7E1C05D0404523D820D009FB0050CC
:105BB000012714F8015B0CEB0506767816F0040F4C
:105BC000ECD116F0030606D0012E14BF5726372657
:105BD000AD1BAB42E5DC7B1C15D0BAF1000F21D127
:105BE0000AB1EFB9116002B0BDE8F00F70475D4532
:105BF000DCDD4FF0FF37DCE7302D1AD0002BBED1B3
:105C00000A239946BCE70199BAF1000F4FF022032D
:105C10000CBF6FF000404FF000400B60002AE2D054
:105C2000611EDFE74042DBE7B41C75784FF0010AE4
:105C3000A2E7207800F0DF00582803D0002B9ED187
:105C400008239CE7102365789946023498E700BF43
:105C5000B405002030B4044C0D46134601462A46D4
:105C6000206830BCFFF76CBFB0050020024B13B1B9
:105C7000024800F005B87047000000008D5C010884
:105C8000014600200246034600F018B838B5094D19
:105C9000094C641BA41018BF05EB840505D0013C1A
:105CA00055F8043D9847002CF9D1BDE8384000F084
:105CB00061BC00BF9065010894650108F0B5274CF0
:105CC00085B026680746D6F84841002C40D0656864
:105CD0001F2D1EDD224818B94FF0FF3005B0F0BD72
:105CE0004FF4C870039102920193AFF300800399BF
:105CF0000446029A019B0028EED0D6F848510020B5
:105D0000256060600546C6F84841C4F88801C4F8BB
:105D10008C013FB96B1C00200235636044F82510EC
:105D200005B0F0BD0126AE4004EB8500C0F8882028
:105D3000D4F88821022F42EA0602C4F88821C0F86C
:105D40000831E7D1D4F88C311E43C4F88C61E1E707
:105D500006F5A674C6F84841B9E700BF58640108C3
:105D6000000000002DE9F0418AB004460D4600F025
:105D70006BF8DFF8D080064698F900300F46013303
:105D80000BD02046294600F057FA30B1204629466C
:105D900000220023FEF7E4FF20B1304639460AB066
:105DA000BDE8F081234B98F800600890CDE90245EA
:105DB000CDE90445019346BB1F4B4FF06042CDE94E
:105DC00006232046294600220023FEF7A1FF70B1DA
:105DD00002239E42009322D0684600F055FAF0B1AB
:105DE000089B0BBBDDE906010AB0BDE8F081012389
:105DF000022E00930ED0684600F046FA50B10F48CC
:105E000000F044FACDE90601EAE70D4B0022CDE9A6
:105E10000623D6E700F040FA21230360EFE700F005
:105E20003BFA22230360DBE700F036FA089B0360AD
:105E3000D8E700BF60650108FFFFEFC76465010890
:105E40000000F0FFB80500202DE9F04FB1F5801FEC
:105E500087B002460B460F465BDA21F00046064348
:105E600000F0F5800029C0F2A4810022B24BFEF7B9
:105E7000E7FC0F460B46B14902468F426FF03505ED
:105E80004BDCC7F3130606F5152101F6647101F426
:105E9000801484F07F5181F4401141EA06031046DA
:105EA00019460022A64BFEF717FB4FEA2758B31CF2
:105EB000A8F2FF38C3F31303A844022B08EB1458CD
:105EC00082468B464FF000022EDC0023FEF720FFB7
:105ED000002800F0C580B8F1000F00F07181404645
:105EE000FEF748FC80A3D3E9002306460F46FEF7E1
:105EF000A7FC7FA3D3E9002304460D46304639466C
:105F0000FEF79EFC02460B4620462946FEF7E6FABF
:105F100007E08A4900258F42B3DD10461946FEF797
:105F2000DDFA07B0BDE8F08F4FF08043FEF7D6FAF8
:105F300002460B4650465946FEF7ACFDCDE902013C
:105F40004046FEF717FCCDE90401DDE902010246F7
:105F50000B46FEF775FC02460B46CDE90001FEF745
:105F60006FFC65A3D3E9002304460D46FEF768FCE9
:105F700063A3D3E90023FEF7B1FA22462B46FEF7CE
:105F80005FFC61A3D3E90023FEF7A8FA22462B4663
:105F9000FEF756FC5EA3D3E90023FEF79FFADDE986
:105FA0000023FEF74DFC5CA3D3E90023CDE90001FB
:105FB00020462946FEF744FC59A3D3E90023FEF707
:105FC0008DFA22462B46FEF73BFC57A3D3E900236C
:105FD000FEF784FA22462B46FEF732FC0B460246B9
:105FE000DDE90001FEF77AFAA6F5C223C6F5D72649
:105FF000A3F27A4351361E43002E04460D4657DD68
:106000000022504B50465946FEF71AFC52465B465A
:10601000FEF716FC06460F46B8F1000F40F09680DA
:1060200022462B46FEF75AFADDE90223FEF708FC6A
:1060300002460B4630463946FEF74EFA02460B46FC
:1060400050465946FEF748FA07B0BDE8F08F0022E7
:10605000002300203C49FEF71DFD07B0BDE8F08F8E
:1060600052465B4650465946FEF7EAFB30A3D3E959
:10607000002304460D4650465946FEF7E1FB024612
:106080000B4600202F49FEF727FA02460B46204612
:106090002946FEF7D5FB04460D46B8F1000F40F047
:1060A00092805046594622462B46FEF715FA38E7AD
:1060B000B8F1000F00F0AB800BA3D3E90023DDE9BA
:1060C0000401FEF7BDFB22462B4606460F4650460E
:1060D0005946FEF701FADDE90223FEF7B1FB04465B
:1060E0000D46DDE904017CE00000E0FE422EE63FC3
:1060F000763C7935EF39EA3D44523EDF12F1C23F3A
:10610000DE03CB966446C73F599322942449D23F7D
:10611000935555555555E53F9FC678D0099AC33FCD
:10612000AF788E1DC571CC3F04FA97999999D93FE4
:10613000555555555555D53F00005043FFFFEF7F4E
:106140000000F03F0000E03F000050C336A3D3E959
:106150000023DDE90401FEF773FB224680468946F1
:106160002B4630463946FEF7B9F9DDE90223FEF742
:1061700067FB2FA3D3E9002304460D46DDE90401A4
:10618000FEF75EFB02460B4620462946FEF7A6F9BF
:1061900002460B4630463946FEF79EF952465B46AC
:1061A000FEF79AF902460B4640464946FEF794F937
:1061B000B7E6FEF791F900220023FEF76BFCB0E68C
:1061C00000200021ADE64046FEF7D4FA16A3D3E93D
:1061D000002380468946FEF733FB06460F464046BD
:1061E000494613A3D3E90023FEF72AFB02460B46D8
:1061F00020462946FEF770F952465B46FEF76CF9D9
:1062000002460B4630463946FEF766F989E60246F5
:106210000B4650465946FEF75FF9DDE90223FEF7CB
:106220000FFB0BE7AFF300800000E0FE422EE63FDD
:10623000763C7935EF39EA3D31F0004310B408D0AF
:106240000F4AA3F5801494420AD804205DF8044B49
:10625000704700280CBF022003205DF8044B7047F4
:10626000B3F5801F01D20320F7E7064A934201D01D
:106270000020F2E7D0F1010038BF0020EDE700BFB9
:10628000FFFFDF7F0000F07F002070470020014902
:10629000704700BF0000F87F014B1868704700BFCF
:1062A000B0050020F401000064000000018008082F
:1062B00000000000000001000000000000000000DD
:1062C000C80000000000000000000000010003E81A
:1062D0000000000000000003E800000000000200D1
:1062E000FA0600030000000000370600000000006E
:1062F00000000000010203524F5200000106524FFD
:106300004C000002064D5354000003024D5650004D
:1063100000040753415000000507474150000006A4
:106320000353544150000703525341500008035394
:1063300047500000090747475000000A03535447DD
:1063400050000B0352534750000C035246530000B9
:106350000D0353494F00000E0747494F00000F033C
:1063600053414300001D0753434F00001E0747439E
:106370004F00001F0343434F0000200341434F00E1
:1063800000270355463000004007554631000041C4
:106390000755463200004207554633000043075573
:1063A000463400004407554635000045075546363B
:1063B000000046075546370000470752554E00007B
:1063C000810553544F5000800042494E00008B001D
:1063D0000000000000000033313130563130390008
:1063E000544D434D2D333131302028766972747508
:1063F000616C20434F4D29005472696E616D696371
:10640000204D6F74696F6E20436F6E74726F6C00F5
:10641000544D43333131300056435020436F6E6644
:1064200069670056435020496E7465726661636502
:10643000004142530052454C00434F4F52440053D9
:10644000544152540053544F5000535441545553E7
:1064500000000000430000008801002000202020F0
:106460002020202020202828282828202020202004
:1064700020202020202020202020202020881010D4
:106480001010101010101010101010101004040430
:1064900004040404040404101010101010104141EE
:1064A00041414141010101010101010101010101DC
:1064B00001010101010101011010101010104242F0
:1064C00042424242020202020202020202020202AC
:1064D000020202020202020210101010200000004C
:1064E00000000000000000000000000000000000AC
:1064F000000000000000000000000000000000009C
:10650000000000000000000000000000000000008B
:10651000000000000000000000000000000000007B
:10652000000000000000000000000000000000006B
:10653000000000000000000000000000000000005B
:10654000000000000000000000000000000000004B
:10655000000000000000000000000000000000003B
:106560006C6F670000000000F8B500BFF8BC08BC05
:106570009E467047F8B500BFF8BC08BC9E46704701
:0865800068EFFF7F010000003D
:086588006D5C0108AD81000803
:0465900089810008F5
:10659400D7630108000102000008000001000000A8
:1065A40002000000000000000000000000000000E5
:1065B40000000000000000000000000000000000D7
:1065C40000000000000000000000000000000000C7
:1065D400000000001201000202000040D016CC06A8
:1065E40000020102030104030904000000C20100C7
:1065F40000000800EFB40008FDB4000859B5000815
:106604003DB5000875B5000891B50008ADB50008A2
:10661400E1B40008E3B40008E5B40008E7B40008F6
:10662400E9B40008EBB40008EDB400080A0600025F
:10663400000000400100000009B500080DB5000885
:10664400C9B5000811B5000815B50008000E2707E4
:10665400000000000000000001020304060708090E
:1066640000000000010203040102030406070809F4
:10667400E40000201D2D0108692C01081F2C0108CD
:106684008F2B0108F12B0108732B01085D2B0108E6
:106694009F2B0108AD2B0108BB2B0108D12B01084E
:1066A400FF00000009024300020100C03209040097
:1066B400000102020100052400100105240100016B
:1066C400042402020524060001070582030800FFD2
:1066D40009040100020A000000070501024000004D
:1066E4000705810240000000C92F0108A12F0108FD
:1066F400E12E010800000000F52D01081D300108FD
:10670400B12E0108312E0108000000000000000035
:10671400252E010800000000000000007404002081
:10672400DC040020440500200000000000000000FC
:106734000000000000000000000000000000000055
:106744000000000000000000000000005464010884
:106754000000000000000000000000000000000035
:106764000000000000000000000000000000000025
:106774000000000000000000000000000000000015
:106784000000000000000000000000000000000005
:1067940000000000000000000000000000000000F5
:1067A40000000000000000000000000000000000E5
:1067B40000000000000000000000000000000000D5
:1067C40001000000000000000E33CDAB34126DE672
:1067D400ECDE05000B0000000000000000000000DB
:1067E40000000000000000000000000000000000A5
:1067F4000000000000000000000000000000000095
:106804000000000000000000000000000000000084
:106814000000000000000000000000000000000074
:0C6B4400880100205C64010801000000D2
:0400000508015A197B
:00000001FF
